:020000040800F2
:10000000687B01206902000869310008A92B0008FB
:100010004D310008A10400088D38000800000000E0
:10002000000000000000000000000000AD0100081A
:100030005105000800000000010200089932000884
:10004000830200088302000883020008830200087C
:10005000830200088302000883020008830200086C
:10006000830200088302000883020008830200085C
:10007000830200088302000883020008830200084C
:1000800083020008BD04000883020008000000008D
:1000900000000000000000000000000083020008D3
:1000A000830200088302000883020008830200081C
:1000B000830200088302000883020008830200080C
:1000C000830200088302000883020008B13100089F
:1000D0008302000883020008813800080000000045
:1000E0008302000883020008830200080000000069
:1000F0000000000000000000000000008302000873
:100100000000000083020008830200088302000848
:1001100000000000000000000000000000000000DF
:100120008302000883020008C90400088302000853
:100130008302000800000000000000000000000032
:100140000000000000000000000000008302000822
:10015000830200088302000883020008830200086B
:100160008302000883020008000000000000000075
:10017000000000000000000000000000000000007F
:1001800000000000830200080000000000000000E2
:100190008302000883020008DFF80CD000F030F979
:1001A0000048004735480008687B01202B4B196840
:1001B0000868B0E8F04F80F30988BFF36F8F4FF005
:1001C000000080F3118870470000000006480068B6
:1001D000006880F3088862B661B6BFF34F8FBFF343
:1001E0006F8F00DF00BF00BF08ED00E0DFF80C00FC
:1001F000016841F470010160704700BF88ED00E0C4
:10020000EFF30980BFF36F8F144B1A681EF0100FC5
:1002100008BF20ED108A20E9F04F106008B44FF0BD
:10022000500080F31188BFF34F8FBFF36F8F05F03D
:100230004DF94FF0000080F3118808BC1968086878
:10024000B0E8F04F1EF0100F08BFB0EC108A80F33A
:100250000988BFF36F8F704700BF00BFC800002040
:10026000EFF30580704700000648804706480047C6
:10027000FEE7FEE7FEE7FEE7FEE7FEE7FEE7FEE756
:10028000FEE7FEE769330008990100082DE9F05FF9
:100290000546002092469B468846064681464024F5
:1002A0001BE0284641464746224600F099F853464F
:1002B0005A46C01A914110D311461846224600F002
:1002C00080F82D1A67EB01084F46224601200021D5
:1002D00000F077F817EB00094E41201EA4F101044D
:1002E000DFDC484631462A464346BDE8F09FA0F190
:1002F0004101192900D82030704740EA01039B07CB
:1003000003D009E008C9121F08C0042AFAD203E08A
:1003100011F8013B00F8013B521EF9D27047D2B2EE
:1003200001E000F8012B491EFBD270470022F6E7DE
:1003300010B513460A4604461946FFF7F0FF20465B
:1003400010BD421E12F8013F002BFBD111F8013BFA
:1003500002F8013B002BF9D17047421C10F8011B39
:100360000029FBD1801A704710B5002200E0521C12
:10037000835C8C5CA34201D1002BF8D1D8B2E1B2EE
:10038000401A10BD034611F8012B00F8012B002A7A
:10039000F9D11846704730B50B460146002020229F
:1003A000012409E021FA02F59D4205D303FA02F582
:1003B000491B04FA02F52844151EA2F10102F1DCE2
:1003C00030BD202A04DB203A00FA02F100207047F9
:1003D0009140C2F1200320FA03F319439040704783
:1003E000202A04DB203A21FA02F00021704721FA8A
:1003F00002F3D040C2F120029140084319467047F1
:10040000064C074D06E0E06840F0010394E8070061
:1004100098471034AC42F6D3FFF7C2FEE00601085D
:10042000000701080448017BF02904D2034B202275
:100430005A54491C0173704700000020C80C00206A
:100440000448C17A142904D2034B2D225A54491C62
:10045000C172704700000020B40C00200448C17A2B
:10046000142904D2034B2E225A54491CC1727047DE
:1004700000000020B40C0020074A30B1117BF029A5
:1004800003D2064B5854491C11730020D072034804
:1004900014211438FFF74ABF00000020C80C0020C8
:1004A00002A103A000F0EEFCFEE700000000000047
:1004B0004275734661756C7400000000014800F0DD
:1004C0004DBD0000180E0020014800F047BD00009F
:1004D000B80D002001681823CAB2103AB2FBF3F23B
:1004E000054B6FF30901032A9B5CC36500D9091D05
:1004F00081650846704700000006010810B50146F6
:1005000000208B698A6A4FF0C07453B1B3F5005F65
:1005100015D072B1012A0CD0022A0AD0032A09D1BF
:1005200004E01AB1012A06D0022A03D1C96AC9011E
:1005300000D5012010BDC96AA142FAD010BD002A21
:10054000F7D0012AF2D0022AF3D0032AF3D010BD4B
:100550007047000070B505460024FFF7FEFE052831
:1005600014D02846FFF7F9FE042858D02846FFF794
:10057000F4FE03287ED02846FFF7EFFE02287AD04B
:100580002846FFF7EAFE012876D001E1FDA12846C2
:10059000FFF7EAFE00282ED0FCA12846FFF7E4FE74
:1005A00000282AD0FBA12846FFF7DEFE38B3FBA1C6
:1005B0002846FFF7D9FE20B3FAA12846FFF7D4FE5C
:1005C00008B3FAA12846FFF7CFFEF0B1F9A12846FB
:1005D000FFF7CAFED8B1F9A12846FFF7C5FEC0B1A2
:1005E000F8A12846FFF7C0FEA8B1F8A12846FFF7FA
:1005F000BBFE90B1CCE0312070BD322070BD332005
:1006000070BD342070BD352070BD362070BD3720E0
:1006100070BD382070BD392070BD302070BDEDA197
:100620002846FFF7A1FE002841D0ECA12846FFF79D
:100630009BFE002878D0EBA12846FFF795FE98B3E3
:10064000EAA12846FFF790FE78B3EAA12846FFF713
:100650008BFE58B3E9A12846FFF786FE00286ED02E
:10066000E8A12846FFF780FE48B3E8A12846FFF737
:100670007BFE02E02DE065E07FE010B3E5A12846B7
:10068000FFF772FEF8B1E5A12846FFF76DFEE0B175
:10069000E4A12846FFF768FEC8B1E4A12846FFF7A9
:1006A00063FE00287AD073E003E004E005E06220F6
:1006B00070BD662070BD682070BD6A2070BD70205E
:1006C00070BD712070BD762070BD782070BD79201E
:1006D00070BDD8A12846FFF747FE002870D0D6A1EC
:1006E0002846FFF741FE00286BD0D4A12846FFF72B
:1006F0003BFED0B1D2A12846FFF736FEB8B1D1A15A
:100700002846FFF731FEA0B1CFA12846FFF72CFE07
:1007100088B1CEA12846FFF727FE70B1CCA12846AC
:10072000FFF722FE60B133E02BE1642070BD67204B
:1007300070BD6B2070BD722070BD752070BD1EE154
:100740007720FBE7C3A12846FFF70EFE00287DD0E7
:10075000C1A12846FFF708FE58B1C0A12846FFF7FF
:1007600003FE40B1BEA12846FFF7FEFD002871D070
:100770000EE06920E2E76D20E0E78BA12846FFF755
:10078000F3FD002869D080A12846FFF7EDFD88B170
:100790002846FFF7E2FD082814D300E0F0E0B1A1FD
:1007A0002846FFF7E1FD38B1B1A12846FFF7DCFD8F
:1007B00020B161E07420C1E78020BFE78320BDE75E
:1007C000DCE0F2E12846FFF7C8FD062854D1ABA1D2
:1007D0002846FFF7C9FDD0B3AAA12846FFF7C4FDFC
:1007E000B0B3AAA12846FFF7BFFD90B3A9A1284640
:1007F000FFF7BAFD78B3A9A12846FFF7B5FD58B3B6
:10080000A8A12846FFF7B0FD40B39CA12846FFF7FA
:10081000ABFDB8B3A5A12846FFF7A6FD98B3A5A1E7
:100820002846FFF7A1FD78B396A12846FFF79CFD67
:1008300050B3A2A12846FFF797FD70B3A1A12846A7
:10084000FFF792FD50B3A1A1284608E0B8E11CE0F3
:100850001DE01EE0A8E11EE021E0A4E121E0FFF799
:1008600083FD50B391A12846FFF77EFD38B399A1CF
:100870002846FFF779FD20B32846FFF76EFD0528CF
:1008800021D04DE00FE010E011E02E2056E72C20A3
:1008900054E75C2052E7222050E70AE00BE05F209B
:1008A0004CE73A204AE73B2048E73F2046E7212033
:1008B00044E72D2042E7292040E740203EE78420FE
:1008C0003CE788203AE785A12846FFF74DFDE8B3CD
:1008D00084A12846FFF748FDC8B384A12846FFF746
:1008E00043FDA8B383A12846FFF73EFD88B383A14B
:1008F0002846FFF739FD68B382A12846FFF734FD8B
:1009000048B380A12846FFF72FFD98B37FA1284662
:10091000FFF72AFD78B37FA12846FFF725FD58B3DE
:1009200048A12846FFF720FD38B34FA12846FFF71E
:100930001BFD18B379A12846FFF716FDF8B179A180
:100940002846FFF711FDD8B178A105E011E112E1C9
:1009500013E114E115E116E12846FFF705FD78B132
:1009600074A12846FFF700FD58B174A12846FFF78F
:10097000FBFCE7E009E10AE10BE10CE10DE10EE12E
:100980000FE113E12E2D2D2D2D0000002E2E2D2DEB
:100990002D0000002E2E2E2D2D0000002E2E2E2E8E
:1009A0002D0000002E2E2E2E2E0000002D2E2E2E7D
:1009B0002E0000002D2D2E2E2E0000002D2D2D2E70
:1009C0002E0000002D2D2D2D2E0000002D2D2D2D63
:1009D0002D0000002D2E2E2E000000002D2E2D2E7D
:1009E000000000002E2E2D2E000000002E2E2E2E98
:1009F000000000002E2D2D2D000000002E2D2E2E8B
:100A0000000000002E2D2D2E000000002D2D2E2D7B
:100A1000000000002E2E2E2D000000002D2E2E2D69
:100A2000000000002D2E2D2D000000002D2D2E2E5B
:100A3000000000002E2E2E002D2D2D002D2E2E001C
:100A40002D2D2E002D2E2D002E2D2E002E2E2D0084
:100A50002E2D2D002E2D00002E2E00002D2D0000FD
:100A60002D2E00002E2E2E2D2E2E2E2D2E2E2E0033
:100A70002E2E2E2E2E2E2E2E000000002D2E2D2E50
:100A80002D2E00002D2D2E2E2D2D00002E2D2D2D46
:100A90002D2E00002E2D2E2E2D2E00002E2E2D2D33
:100AA0002E2D00002D2D2D2E2E2E00002E2E2D2D24
:100AB0002E2E00002D2E2D2E2D2D00002D2E2E2E13
:100AC0002E2D00002D2E2D2D2E2D00002E2D2D2E05
:100AD0002D2E00002E2E2E2D2E2D00002D2E2E2DF3
:100AE0002E0000002D2E2D2D2E0000002D2E2E2E3E
:100AF0002D0000002E2D2E2E2D0000002D2E2D2E2F
:100B00002D0000002E2D2E2D2E0000002E2E2E2D1D
:100B10002E0000002E2D2E2E2E0000002E2D2D2E0C
:100B20002E2D20002D2D2D2E2E2D00002D2D2E2E84
:100B30002D2E00002D2E2D2E2E0000002E2E2D2EBF
:100B40002E00000078B31FA12846FFF70DFC58B314
:100B50001EA12846FFF708FC38B31EA12846FFF760
:100B600003FC58B31DA12846FFF7FEFB40B3204607
:100B7000E4E52F20E2E52820E0E53D20DEE5092040
:100B8000DCE58120DAE52B20D8E58220D6E585203A
:100B9000D4E58620D2E58720D0E57320CEE56C2011
:100BA000CCE57A20CAE503E004E005E06320C5E572
:100BB0006520C3E56E20C1E56F20BFE58920BDE556
:100BC0006120BBE52D2D2E2D2D0000002D2D2D2E6D
:100BD000000000002D2D2D2D000000002E2D2E2DAB
:100BE0000000000070B5724C86B0A07920B9E079A1
:100BF00010B9207A002875D0E089218A00EB4000E6
:100C0000C00000EB81004EF66021B1FBF0F02085C2
:100C100068A002F0BAFA238D628A218AE08902ADC7
:100C200085E80F00608C1E21CDE90001E38CA28CC9
:100C30006A496B4802F052FE694802F0A6FAE08960
:100C400000284FD0208A00284CD0A079002540B33E
:100C5000A571207808B163A000E065A002F095FAC4
:100C6000A08CE189B0EB410F63480DD9FFF775FB0C
:100C70001D2803D261A16048FFF763FB5FA002F06B
:100C800084FAFFF7DDFB0CE0FFF767FB1D2803D2BA
:100C90005BA15948FFF755FB59A002F076FAFFF720
:100CA000DDFBE079002857D0E57100BF5248FFF71F
:100CB00051FC514E5036307060717570FFF7DCFB9F
:100CC000307880B14FA16846FFF75CFB307884280C
:100CD00056D015DC81285AD00DDC092848D0802850
:100CE00022D147E062E049A16846FFF74BFB42484A
:100CF00048A15030E8E782284BD0832814D107E080
:100D00008538052810D2DFE800F0373905464D0058
:100D100041A100E042A138485030FFF733FB34A135
:100D20004FEA0D00FFF72EFB207818B12DA1684681
:100D3000FFF728FB304B6A4650333BA1A3F132004A
:100D400002F0CCFD2C4926481E31FFF7FAFA2A485A
:100D50000570234802F019FA207A002826D025725F
:100D600034A002F012FA06B0BDE87040FFF75ABB9B
:100D700031A106E031A104E031A102E033A100E09D
:100D800034A11D485030FFF7FDFA34A1C8E735A162
:100D900002E036A100E037A117485030FFF7F2FA21
:100DA00035A1BDE7144836A15030BBE706B070BD91
:100DB000000000201B5B731B5B333B33304820205B
:100DC0002020202020202020202020202020202023
:100DD0002020202020202020202020008006010824
:100DE0009E0100201B5B33383B353B3233386D00AE
:100DF0001B5B33336D000000860500202D000000D2
:100E00002E0000001B5B33326D0000001B5B333192
:100E10006D0000003F3F3F004552524F520000001E
:100E200052494E472E2E2E00092573272573271B66
:100E30005B33376D0D0A000054414200575757008D
:100E4000554E44455253544F4F4400005741495466
:100E50002E2E2E0052455045415400001B5B333767
:100E60006D000000535441525400000053544F5041
:100E700000000000454E44001B5B33366D0000004F
:100E800043480000B2B01E4D0E4604460122D10375
:100E9000284600F05DFC01225103284600F058FC72
:100EA0004FF4804700223946284600F051FC334673
:100EB000224614A1684602F011FD684602F065F969
:100EC000194E0024A8460025184800F0E9FC6D1CC6
:100ED000B542F9D33946404600F00EFC641CE4B23A
:100EE0000A2CF0D3BFF34F8F11480168114A01F467
:100EF000E06111430160BFF34F8F00BFFDE70000C9
:100F0000000402400D0A1B5B33316D47757275207A
:100F10004D656469746174696F6E1B5B33336D2555
:100F20007320257300000000400D0300100C00200A
:100F30000CED00E00400FA0590F83510022903D00A
:100F40008021416501207047052180F83510006837
:100F5000016821F001010160002070472DE9F8438C
:100F600004464FF00009CDF8009063484FF4165145
:100F7000A56D0068B0FBF1F72E6894F85C100820AE
:100F800000FA01F131420FD021680A6852070BD5EF
:100F90000A6822F004020A6094F85C108840A86095
:100FA000606D40F00100606594F85C104FF001083E
:100FB00008FA01F0304208D021684969090604D5D1
:100FC000A860606D40F00200606594F85C10042039
:100FD0008840304208D021680968890704D5A86094
:100FE000606D40F00400606594F85C10102088404B
:100FF000304218D021680968090714D5A860206814
:101000000168490304D50068000308D5A16C07E016
:101010000168C90503D4016821F008010160216C51
:1010200009B12046884794F85C102020884030425F
:1010300031D021680968C9062DD5A86094F835001B
:1010400005282068016806D0490347D500680003D9
:101050001DD4616C1CE021F016010160206841691B
:1010600021F080014161206C08B9A06C20B120689A
:10107000016821F00801016094F85C103F2088406D
:10108000A86084F8349084F83580216D1FE0E16B0E
:1010900009B120468847606D00282BD0606DC007DD
:1010A00014D0052084F835002068016821F0010182
:1010B00001600098401C0090B84203D82068006886
:1010C000C007F6D184F8349084F83580E16C0029AB
:1010D00010D001B02046BDE8F04308470168C905BB
:1010E000D5D4016821F01001016084F8349084F8AF
:1010F0003580CCE7BDE8F883B80000202DE9F04149
:10110000044600F05BFB0546002C7CD0A249206819
:1011100088423ED0A049183188423AD09E493031A9
:10112000884236D09C494831884232D09A49603151
:1011300088422ED09849783188422AD096499031F9
:10114000884226D09449A831884222D093498842C7
:101150001FD09249183188421BD0904930318842C3
:1011600017D08E494831884213D08C49603188426B
:101170000FD08A49783188420BD088499031884213
:1011800007D08649A831884203D0C82184A002F044
:101190006FFD6068C0B1B0F1007F15D0B0F1806F15
:1011A00012D0B0F1C06F0FD0B0F1006F0CD0B0F121
:1011B000206F09D0B0F1406F06D0B0F1606F03D05E
:1011C000C92177A002F054FDA06838B1402805D0AD
:1011D000802803D0CA2172A002F04AFDE068B0F571
:1011E000007F04D018B1CB216DA002F041FD206931
:1011F000B0F5806F04D018B1CC2169A002F038FDA1
:10120000606958B100E071E0B0F5006F06D0B0F54C
:10121000805F03D0CD2162A002F02AFDA06948B111
:10122000B0F5005F06D0B0F5804F03D0CE215CA0B2
:1012300002F01EFDE06940B1B0F5807F05D02028A6
:1012400003D0CF2156A002F013FD206A60B1B0F5A3
:10125000803F09D0B0F5003F06D0B0F5403F03D045
:10126000D0214FA002F004FD606A002832D004288B
:1012700006D0D1214AA002F0FBFC606A002829D0E8
:10128000A06A48B1012807D0022805D0032803D05E
:10129000D62143A002F0ECFCE06A60B1B0F5000F8B
:1012A00009D0B0F1807F06D0B0F1C07F03D0D72144
:1012B0003BA002F0DDFC206B60B1B0F5001F09D04F
:1012C000B0F5800F06D0B0F5C00F03D0D82134A000
:1012D00002F0CEFC002684F83460022084F8350049
:1012E0002068016821F0010101600EE00120BDE8E5
:1012F000F08100BF00F062FA401B052805D92020CC
:101300006065032084F83500F1E720680068C007B5
:10131000F0D12268116830480140D4E90103184334
:10132000D4E903352B43184363691843A369184371
:10133000E3691843236A18430843616A042903D107
:10134000D4E90B1319430843106020684069656AAB
:1013500020F0070128460D43012704280CD1A06A7C
:101360000543E06A40B12046FFF7C8F820B14020AD
:10137000606584F83570B9E7206845612046FFF75D
:10138000A9F894F85C203F2191408160666584F85B
:1013900035700020ABE7000010600240106402408E
:1013A0002E2E2F447269766572732F53544D33324B
:1013B000463478785F48414C5F4472697665722F95
:1013C0005372632F73746D3332663478785F68615B
:1013D0006C5F646D612E63003F8010F02DE9F84F63
:1013E000044691480D46844212D0904884420FD062
:1013F0008F4884420CD08F48844209D08E48844262
:1014000006D08E48844203D0C3218DA002F030FC68
:1014100028680104090C01D0000C03D0C42188A065
:1014200002F026FC6868F8B101281DD011281BD0F5
:10143000022819D0122817D09049884214D0904918
:10144000884211D08F4988420ED08F4988420BD0F4
:101450008E49884208D08E49884205D0032803D09F
:10146000C52177A002F004FCA86838B1012805D096
:10147000022803D0C62172A002F0FAFB00264FF02A
:10148000010B00BF0BFA06F02F6882460740574554
:101490007ED16868022801D0122828D12869C8B1F5
:1014A000092817D0012815D0022813D0042811D0FC
:1014B00005280FD006280DD007280BD0082809D002
:1014C0000A2807D00C2805D00F2803D0D7215CA00C
:1014D00002F0CEFBF00804EB8002106A7107CB0E1D
:1014E0000F2199408843296999400143116220687E
:1014F0007200032101FA02F82979914601F00301F3
:1015000020EA080001FA09F1014321606868012816
:1015100005D0022803D0112801D012281CD1E86878
:1015200048B1012807D0022805D0032803D0EA21BA
:1015300043A002F09DFBA068E96820EA080001FAD8
:1015400009F10143A1606068297920EA0A00C1F32A
:101550000011B14001436160E068A96820EA080019
:1015600001FA09F10143E1606868C00056D54948B5
:10157000016841F480410160006826F0030100F435
:101580008040009044480B18D3F80808B10700E0E9
:1015900044E00A0F0F219140884323498C4201D136
:1015A000002114E021498C4201D101210FE02049A2
:1015B0008C4201D102210AE01E498C4201D1032153
:1015C00005E01D498C4201D1042100E00721914032
:1015D0000143C3F80818314908686A68B843D20360
:1015E00000D5384308602D49091D08686A68B8436A
:1015F000920300D5384308602849083108686A68B2
:10160000B843D20200D53843086024490C31086839
:101610006A68B843920200D538430860761C102EE1
:10162000FFF430AFBDE8F88F000002400004024034
:1016300000080240000C024000100240001C024062
:101640002E2E2F447269766572732F53544D3332A8
:10165000463478785F48414C5F4472697665722FF2
:101660005372632F73746D3332663478785F6861B8
:101670006C5F6770696F2E6300000000000011103E
:101680000000211000003110000012100000221094
:10169000000032104438024000300140003C01405C
:1016A00070B50C00054604D14FF4C77103A002F0D9
:1016B000DFFA2869204000D0012070BD2E2E2F4473
:1016C0007269766572732F53544D3332463478788D
:1016D0005F48414C5F4472697665722F5372632F85
:1016E00073746D3332663478785F68616C5F6770ED
:1016F000696F2E630000000070B50C00054604D130
:101700004FF4E37103A002F0B3FA686960406861C6
:1017100070BD00002E2E2F447269766572732F53B0
:10172000544D3332463478785F48414C5F44726997
:101730007665722F5372632F73746D33326634780B
:10174000785F68616C5F6770696F2E6300000000EE
:1017500070B515460C00064604D140F2AF1108A042
:1017600002F086FA45B1012D04D04FF4D87104A0DF
:1017700002F07EFAB46170BD2004B06170BD00005B
:101780002E2E2F447269766572732F53544D333267
:10179000463478785F48414C5F4472697665722FB1
:1017A0005372632F73746D3332663478785F686177
:1017B0006C5F6770696F2E630000000001488068ED
:1017C00070470000BC00002070B5040033D02449ED
:1017D0002068884203D0AD2122A002F049FA606857
:1017E00078B101280DD002280BD0032809D0042895
:1017F00007D0052805D0062803D0AE2119A002F095
:1018000037FAA068B0F5805F03D3AF2115A002F0CE
:101810002FFA21684CF6CC400860216845F25550FB
:101820000860D4E9000141602168A0688860FFF782
:10183000C5FF054609E0012070BD00BFFFF7BEFFF0
:10184000401B302801D9032070BD2068C0680028E3
:10185000F4D121684AF6AA200860002070BD00007B
:10186000003000402E2E2F447269766572732F531C
:10187000544D3332463478785F48414C5F44726946
:101880007665722F5372632F73746D3332663478BA
:10189000785F68616C5F697764672E6300000000A1
:1018A00000684AF6AA21016000207047024881685A
:1018B0000278114481607047BC0000200B4810B5CD
:1018C000016841F400710160016841F480610160C8
:1018D000016841F480710160032000F0D5F80F2009
:1018E00000F006F800F024F8002010BD003C024093
:1018F00070B50D4D04464FF47A712878B1FBF0F0C5
:101900000A490968B1FBF0F000F060FF48B9102CFB
:1019100007D200222146501E00F066F800206C60BD
:1019200070BD012070BD0000BC000020B800002088
:1019300010B5032000F0A8F8002211466FF00B004C
:1019400000F052F8002211466FF00A0000F04CF847
:10195000002211466FF0090000F046F800221146FF
:10196000501F00F041F800221146101F00F03CF813
:1019700000220F21901E00F037F800220F21BDE851
:101980001040501E00F030B810B5040003D5CE2131
:1019900006A002F06DF904F01F01012088406109E2
:1019A000890001F1E021C1F8000110BD2E2E2F4465
:1019B0007269766572732F53544D3332463478789A
:1019C0005F48414C5F4472697665722F5372632F92
:1019D00073746D3332663478785F68616C5F636FFF
:1019E000727465782E63000070B515460C46064685
:1019F000102A03D3BA2114A002F03AF9102C03D311
:101A0000BB2111A002F034F91E480068C0F3022384
:101A1000C3F107022046042A00D90422191D072910
:101A200001D2002300E0DB1E012404FA02F1491E6A
:101A3000014099409C40641E2C4021433046BDE843
:101A4000704001F092BB00002E2E2F447269766523
:101A500072732F53544D3332463478785F48414C7B
:101A60005F4472697665722F5372632F73746D339E
:101A700032663478785F68616C5F636F7274657822
:101A80002E6300000CED00E010B5044607280BD0D3
:101A9000062C09D0052C07D0042C05D0032C03D02C
:101AA000A22108A002F0E4F8154904F00702086832
:101AB0004FF6FF03184040EA0220124A1043086024
:101AC00010BD00002E2E2F447269766572732F535D
:101AD000544D3332463478785F48414C5F447269E4
:101AE0007665722F5372632F73746D333266347858
:101AF000785F68616C5F636F727465782E63000055
:101B00000CED00E00000FA052DE9F0470E46040058
:101B10007DD02068401E0E2804D94FF414717AA09D
:101B200002F0A6F896B1012E10D0022E0ED0032E90
:101B30000CD0042E0AD0052E08D0062E06D0072E73
:101B400004D040F2512170A002F092F8DFF8F08149
:101B5000D8F80000F7B200F00F00B04207D288F8C2
:101B60000070D8F8000000F00F00B0424FD120689C
:101B7000744D810729D5400703D5286840F4E0500B
:101B800028602078000703D5286840F4604028606A
:101B9000A068A0B1802812D0902810D0A0280ED024
:101BA000B0280CD0C0280AD0D02808D0E02806D011
:101BB000F02804D04FF41D7153A002F059F82868A2
:101BC000A16820F0F000084328602078C00743D0C7
:101BD000DFF870916068A9F1080988B1012822D066
:101BE000022824D0032822D040F27B2146A002F014
:101BF0003FF86068012816D0022818D0032816D0B4
:101C0000D9F800008007002833DA286800E030E0C7
:101C1000616820F0030008432860FFF7CFFD81468C
:101C200041F2883A11E0D9F800008003EBE7D9F8D7
:101C300000008001E7E700BFFFF7C0FDA0EB09014E
:101C4000514502D90320BDE8F0872868616800F09B
:101C50000C00B0EB810FEFD1D8F80010404601F036
:101C60000F01B14207D90770006800F00F00B042C1
:101C700001D00120E7E720784FF4805640074FF469
:101C8000A0574FF4C0584FF4E05914D5E06860B144
:101C9000B0420AD0B84208D0404506D0484504D0EA
:101CA00040F2B92118A001F0E3FF2868E16820F4B0
:101CB000E050084328602078000715D5206960B1FE
:101CC000B0420AD0B84208D0404506D0484504D0BA
:101CD0004FF430710CA001F0CBFF2868216920F48B
:101CE000604040EAC100286000F058F82968164AB0
:101CF000C1F30311515CC840144908600F20FFF77D
:101D0000F7FD00209FE700002E2E2F4472697665B4
:101D100072732F53544D3332463478785F48414CB8
:101D20005F4472697665722F5372632F73746D33DB
:101D300032663478785F68616C5F7263632E63002B
:101D4000003C024008380240E8050108B8000020C5
:101D50000148006870470000B800002004480549A9
:101D600000680968044AC1F38221515CC840704789
:101D7000B800002008380240F80501080448054969
:101D800000680968044AC1F34231515CC840704799
:101D9000B800002008380240F8050108154810B5C1
:101DA000006810F00C02144813D01449042A0FD014
:101DB000082A0ED10F4C241F2268236802F03F022C
:101DC0005B0207D52068C0F38810A0FB010106E084
:101DD000084610BD2168C1F38811A1FB0001002352
:101DE000FEF754FA2168C1F30141491C4900B0FBD8
:101DF000F1F010BD083802400024F40040787D0165
:101E00002DE9F84F04007DD020680F2803D9F82170
:101E1000F2A001F02DFF2078DFF8F8B3FE4DC007E7
:101E200056D060684FF480364FF4A02738B1B042E6
:101E300005D0B84203D0FD21E8A001F019FFDBF87E
:101E400000105846C1F38101012909D00068C0F390
:101E5000810002280BD1EF48001F0068400206D520
:101E60002868800334D560680028CCD030E06068F2
:101E7000B04203D1286840F480300CE0B8422868B2
:101E800003D140F480202860F4E720F480302860FB
:101E9000286820F480202860606860B1FFF78EFC1D
:101EA000064604E0FFF78AFC801B64287ED8286879
:101EB0008003F7D50CE0FFF781FC064605E000BF84
:101EC000FFF77CFC801B6428F0D828688003F7D4D7
:101ED0002078DFF8488380074FF0000956D5E06886
:101EE00030B1012804D040F22F11BCA001F0C0FE97
:101EF00020691F2804D94FF49871B8A001F0B8FEEA
:101F0000584600E092E0DBF8001011F00C0F09D009
:101F10000068C0F38100022811D1BE48001F00688C
:101F200040020CD42868800702D5E06801287DD1E2
:101F30002868216920F0F80040EAC10016E0E06856
:101F4000B0B10120C8F80000FFF738FC064604E0F5
:101F5000FFF734FC801B0228A8D828688007F7D533
:101F6000286820F0F801206941EAC00028600DE0EF
:101F7000C8F80090FFF722FC064604E0FFF71EFCBD
:101F8000801B022892D828688007F7D420780007A1
:101F90002ED5A04EA24F60696C36D0B1012808D072
:101FA0004FF4B8718DA001F063FE00E04DE160696F
:101FB00078B101203860FFF701FC074605E000BF5B
:101FC000FFF7FCFBC01B0228C6D830688007F7D596
:101FD0000EE0C7F80090FFF7F1FB074605E000BFF1
:101FE000FFF7ECFBC01B0228B6D830688007F7D497
:101FF0002078400776D5A068002740B1012806D098
:10200000052804D04FF4CE7174A001F031FEDFF842
:1020100004A20AF1380ADAF80000C0000DD4DAF898
:10202000001041F08051CAF8001000E0D4E0DAF866
:102030000000012700F0805000907A4E3068C00503
:1020400011D4306840F480703060FFF7B7FB009027
:1020500006E000BFFFF7B2FB0099401A022891D8B2
:102060003068C005F6D56B4EA068683601280FD0E1
:102070000528306810D020F001003060306820F072
:1020800004003060A068B8B1FFF798FB00900FE043
:10209000306840F00100F4E740F004003060F7E7FA
:1020A000FFF78CFB0099411A41F2883081428BD8AE
:1020B00030688007F4D50EE0FFF780FB009007E062
:1020C000FFF77CFB0099411A41F2883081428BD89E
:1020D00030688007F4D42FB1DAF8001021F0805175
:1020E000CAF80010A069002875D0012809D002287C
:1020F00007D040F2DF1139A001F0BAFDA069002835
:10210000F2D0DBF80000C0F38100022864D0A0699F
:10211000022805D0C8F86090FFF750FB044697E00E
:10212000E06938B1B0F5800F04D04FF4F4712BA002
:1021300001F09EFD206A3F2804D940F2E91127A052
:1021400001F096FD606AC038F02804D94FF4F571AB
:1021500022A001F08DFDA06A02280AD0042808D030
:10216000062806D0082804D040F2EB111BA001F08D
:102170007FFDE06A801E0D2804D94FF4F67117A088
:1021800001F076FD4746C8F86090FFF717FB06465A
:1021900005E000BFFFF712FB801B022855D8286816
:1021A0008001F7D4D4E907010843A16A1E4A49080F
:1021B00002EB0141626A41EA8211084394F82C1053
:1021C00040EA01611348001F016001203866FFF7F3
:1021D000F5FA04462FE03EE03FE000002E2E2F44AB
:1021E0007269766572732F53544D33324634787862
:1021F0005F48414C5F4472697665722F5372632F5A
:1022000073746D3332663478785F68616C5F7263C3
:10221000632E630008380240003802400000474245
:10222000800E4742007000400000FFFFFFF7C6FA33
:10223000001B022809D828688001F7D50BE000BFF1
:10224000FFF7BCFA001B022802D90320BDE8F88F73
:1022500028688001F4D40020F8E70120F6E77047F1
:1022600038B504460068426881684B0605D4CB0740
:1022700003D0530601D5216C04E08B0707D5130664
:1022800005D5616C01B02046BDE83040084711F427
:10229000B07F48D0930646D54B060AD594F8513006
:1022A000032B3DD0636D43F004036365C36883680B
:1022B00000938B0609D5636D43F001036365836862
:1022C0000093036823F040030360C80506D5606DE2
:1022D00040F008006065206880680090606D00280C
:1022E00021D02068416821F0E0014160012084F89C
:1022F0005100900718D02068416821F00301416027
:102300000B4DE06C18B10565E06CFEF715FEA06C96
:10231000002808D00565A06CBDE83840FEF70CBE6B
:10232000C1688068009038BD2046FFF798FF38BD2F
:10233000DD31000870B504006CD05D49206888422A
:1023400010D05C4988420DD05B4988420AD05B4975
:10235000884207D05A49884204D04FF4877159A067
:1023600001F086FC606838B1B0F5827F04D040F29D
:102370000F1154A001F07CFCA06850B1B0F5806F43
:1023800007D0B0F5004F04D04FF488714DA001F094
:102390006FFCE068B0F5006F05D020B140F211117C
:1023A00048A001F065FCA069B0F5007F08D038B105
:1023B000B0F5802F04D04FF4897142A001F058FC91
:1023C000E06990B1082810D010280ED018280CD041
:1023D00020280AD0282808D0302806D0382804D051
:1023E00040F2131137A001F043FC206A30B180287D
:1023F00004D04FF48A7133A001F03AFC606A58B1FE
:1024000010281BD040F215112EA001F031FC606A9B
:1024100010B113E0012070BD206930B1022804D052
:102420004FF48C7127A001F023FC606930B10128C2
:1024300004D040F2191123A001F01AFC0025A56276
:1024400094F8510020B984F85050204600F056F816
:10245000022084F851002068016821F040010160E9
:10246000D4E901010843D4E9031211430843616927
:102470000843218B01F400710843E1690843216A94
:102480000843A16A084321680860A069042101EAA1
:102490001040616A0843216848602068C16921F4DE
:1024A0000061C1616565012084F85100002070BDA4
:1024B0000030014000380040003C00400034014042
:1024C000005001402E2E2F447269766572732F538F
:1024D000544D3332463478785F48414C5F447269DA
:1024E0007665722F5372632F73746D33326634784E
:1024F000785F68616C5F7370692E630070B5064623
:1025000000681F4986B0884238D11E4800250168FE
:1025100041F4805101600068694600F480500590E4
:10252000E02000900220CDE9010503200390052062
:1025300004901548FEF752FF154C144820604FF0E8
:10254000806060604020C4E902050001C4E9040520
:10255000A561E561256220466562FEF7CFFD18B1F1
:1025600082210CA001F0A0F9B464002205212320EF
:10257000A663FFF739FA2320FFF706FA06B070BD0D
:1025800000300140443802400000024040640240F4
:10259000B80D00202E2E2F5372632F73746D3332BB
:1025A000663478785F68616C5F6D73702E630000CD
:1025B0002DE9F84F04468068994617460D460026D7
:1025C00038B1B0F5004F04D040F2C51158A001F069
:1025D0004FFB94F8500001280ED04FF0010B84F807
:1025E00050B0FFF7EBF8804694F851004FF0000A26
:1025F000012804D0022695E00220BDE8F88F002DC6
:102600007CD0002F7AD0032084F85100C4F854A065
:102610002563A786E786C4F838A0A4F83CA0A4F8F0
:102620003EA0C4F844A0C4F840A0A068B0F5004F94
:1026300004D12068016841F480410160206801688C
:10264000490603D4016841F040010160E068B0F53B
:10265000006F606804D038B3E08E012824D03FE0DA
:1026600010B1E08E01281BD1216835F8020BC8603B
:1026700006E020688168890706D535F8021BC1602D
:10268000E08E401EE0860BE0B9F1000F34D0B9F1C6
:10269000FF3F05D0FFF792F8A0EB080149452BD288
:1026A000E08E0028E5D11EE0216815F8010B0873C3
:1026B00006E020688168890706D515F8011B0173BB
:1026C000E08E401EE0860BE0B9F1000F14D0B9F1A6
:1026D000FF3F05D0FFF772F8A0EB080149450BD288
:1026E000E08E0028E5D14B46012202212046CDF89C
:1026F000008000F07BFD10B1032613E011E042469C
:102700004946204600F05AFD18B101262020606598
:1027100008E0A06818B92068C16880680090606D02
:1027200000B1012684F851B084F850A0304664E727
:102730002E2E2F447269766572732F53544D3332A7
:10274000463478785F48414C5F4472697665722FF1
:102750005372632F73746D3332663478785F6861B7
:102760006C5F7370692E630010B54FF0E02404288D
:1027700009D020B140F2D91105A001F079FA206901
:1027800020F0040002E0206940F00400206110BD48
:102790002E2E2F447269766572732F53544D333247
:1027A000463478785F48414C5F4472697665722F91
:1027B0005372632F73746D3332663478785F686157
:1027C0006C5F636F727465782E63000010B5401EF5
:1027D000B0F1807F01D3012010BD4FF0E024606193
:1027E0000F21601700F0C1FC0020A06107202061CC
:1027F000002010BD7047000070B5026804461068E4
:10280000D168536910F00F0F51D003F0010501F4A6
:10281000907635435DD0C20705D0CA0503D5E26B7B
:1028200042F00102E263420705D5DA0703D0E26B0A
:1028300042F00202E263820705D5DA0703D0E26BB9
:1028400042F00402E263020705D5DA0703D0E26B27
:1028500042F00802E263E26B002A34D0800604D51D
:10286000880602D5204600F0BFFD20684069E16B74
:10287000C0F3801001F008010143204624D000F08D
:10288000A5FD2068416949061AD5416921F040013A
:102890004161606BA0B11B490165606BFEF74CFBA9
:1028A000002810D0606B016DBDE8704008478306BA
:1028B0000FD58B060DD52046BDE8704000F094BDC5
:1028C0002046FFF797FF70BDFFF794FF0020E063FD
:1028D00070BD030606D50B0604D52046BDE8704042
:1028E00000F06ABF4006F3D54806F1D5D16820460E
:1028F00021F04001D160202184F8391000F052F914
:1029000070BD0000BD33000870B504001FD0A06981
:10291000354B00283549364A20681AD08D15984223
:1029200009D0884207D0904205D0294631A001F055
:102930009FF9A069C0B1A069A84215D0B0F5007F89
:1029400012D0B0F5407F0FD040F2011109E0012014
:1029500070BD984208D0884206D0904204D040F220
:10296000051124A001F084F9A06838B1B0F5805FAA
:1029700004D040F207111FA001F07AF9E06938B1E4
:10298000B0F5004F04D04FF484711AA001F070F933
:1029900094F83900002520B984F83850204600F01A
:1029A00047F8242084F839002068C16821F40051D8
:1029B000C160204600F05EFD2068016921F490416D
:1029C00001612068416921F02A0141612068C168E4
:1029D00041F40051C160E563202084F8390084F897
:1029E0003A00002070BD000000100140004400408B
:1029F000001401402E2E2F447269766572732F5396
:102A0000544D3332463478785F48414C5F447269A4
:102A10007665722F5372632F73746D333266347818
:102A2000785F68616C5F756172742E6300000000EE
:102A300070B506460068204986B0884239D11F48E3
:102A40000025016841F4003101600068694600F426
:102A5000003005900C20009002200190012002908F
:102A600003200390072004901548FEF7B7FC164C8E
:102A7000144820604FF0006060604020C4E9020507
:102A80000001C4E90405A561E5612562204665628F
:102A9000FEF734FB18B1D4210CA000F005FF34631D
:102AA000002205212620A663FEF79EFF2620FEF7C2
:102AB0006BFF06B070BD000000440040403802408B
:102AC00000000240A0600240180E00202E2E2F535E
:102AD00072632F73746D3332663478785F68616C1B
:102AE0005F6D73702E63000070472DE9F843044654
:102AF00090F839001F4616460D46202850D1A5B142
:102B00009EB194F8380001284AD0012084F838009A
:102B10004FF00008C4F83C80212084F83900FEF70B
:102B20004DFEA6848146E68426E00120BDE8F883B8
:102B3000E08C401EE084A0684B46B0F5805F4FF00B
:102B400000024FF080012046009703D000F065FEA0
:102B5000E8B90DE000F061FEC8B928882168C0F32B
:102B600008004860206908B16D1C05E0AD1C03E059
:102B7000216815F8010B4860E08C0028D8D14B463D
:102B8000002240212046009700F047FE08B10320B4
:102B9000CCE7202084F8390084F838800020C5E78D
:102BA0000220C3E77047000002A103A0FEF76AF904
:102BB000FEE7000000000000486172644661756C29
:102BC0007400000010B5FDF792FBC0B231287CD034
:102BD00032287BD033287AD0342879D0352878D061
:102BE000362877D0372876D0382875D0392874D051
:102BF000302873D02E2872D02C2871D05C2870D049
:102C000022286FD05F286ED03A286DD03B2866D03E
:102C10003F286AD0212869D02D2868D02B2867D07A
:102C20002F2866D0282865D029286ED03D286DD061
:102C300040286CD009286BD080286AD0812869D0C0
:102C40008228ECD083286ED08428E2D085286BD0EF
:102C500086286AD0872869D0882868D0622867D0FB
:102C600063286ED066286DD068286CD06A286BD037
:102C70006C286AD0702869D0712868D0762867D00F
:102C800078286ED079286DD07A286CD073286BD0D4
:102C90006F286AD0642869D0672868D06B28DAD09A
:102CA00072286FD075286ED077286DD061286CD0CF
:102CB00069286BD06D286AD06E2869D0652868D0E5
:102CC000742867D159A15A4815E018E019E01AE0B4
:102CD00021E022E023E024E02BE02CE02DE02EE0B8
:102CE00037E038E039E03AE042E043E044E045E0F4
:102CF00046E050E051E0BDE81040FDF743BB4DA178
:102D0000E1E74FA1DFE751A1DDE748E049E04AE014
:102D10004BE04CE04DE050A1D5E752A1D3E754A1E0
:102D2000D1E756A1CFE746E047E048E049E04AE076
:102D30004BE055A1C7E757A1C5E759A1C3E75BA180
:102D4000C1E744E045E046E047E048E049E04AE0CA
:102D50004BE05AA1B7E75DA1B5E760A1B3E763A176
:102D6000B1E744E045E046E047E048E049E04AE0BA
:102D700062A1A8E765A1A6E768A1A4E76BA1A2E705
:102D80006EA1A0E741E042E043E044E045E046E0D8
:102D900047E048E049E06CA195E76EA193E770A198
:102DA00091E773A18FE775A18DE778A18BE77AA1F1
:102DB00089E77FA187E781A185E785A183E779A1DD
:102DC00081E77CA17FE785A17DE74DA17BE738A165
:102DD00079E743A177E77BA175E783A173E785A135
:102DE00071E787A16FE742A16DE751A16BE787A16A
:102DF00069E74BA167E746A165E71BA163E70EA161
:102E000061E722A15FE724A15DE74DA15BE713A184
:102E100059E70FA157E737A155E73AA153E729A191
:102E200051E724A14FE711A14DE710BD2D2000006F
:102E3000F00B00202E202D202D202D202D200000F5
:102E40002E202E202D202D202D2000002E202E2063
:102E50002E202D202D2000002E202E202E202E2052
:102E60002D2000002E202E202E202E202E2000008F
:102E70002D202E202E202E202E2000002D202D2033
:102E80002E202E202E2000002D202D202D202E2023
:102E90002E2000002D202D202D202D202E20000062
:102EA0002D202D202D202D202D2000002D202E2006
:102EB0002D202E202D202E20000000002D202D2042
:102EC0002E202E202D202D20000000002E202D2031
:102ED0002D202D202D202E20000000002E202D2022
:102EE0002E202E202D202E20000000002E202E200F
:102EF0002D202D202E202D20000000002D202D2003
:102F00002D202E202E202E20000000002E202E20EE
:102F10002D202D202E202E20000000002D202E20E0
:102F20002D202E202D202D20000000002D202E20D1
:102F30002E202E202E202D20000000002E202D20BF
:102F40002E202D202E2000002D202E202E202D2062
:102F50002E2000002D202E202D202D202E200000A0
:102F60002D202E202D202D202E202D200000000091
:102F70002D202E202E202E202D2000002E202D2032
:102F80002D202E202D202E20000000002E202D2070
:102F90002E202E202D2000002E202E202E202D2011
:102FA0002E202E202E202D202E202E202E20000000
:102FB0002D202E202D202E202D2000002E202E20F2
:102FC0002E202E202E202E202E202E20000000002D
:102FD0002E202E202E202D202E2000002E202E20D0
:102FE0002E202D202E202D002E202D202D202D2096
:102FF000000000002E202D202E202E20000000009A
:103000002E202D202D202E20000000002D202E20EF
:103010002E202D200000000070470000F0B525484C
:1030200087B00024016841F001010160016801F0EE
:1030300001010591016841F00201016000681E4E26
:1030400000F00200059001224FF420413046FEF7C7
:103050007FFB002244F2C0013046FEF779FB174F98
:10306000002271153846FEF773FB012291023846A3
:10307000FEF76EFB41F2080001258DE8310069463C
:103080003046FEF7ABF94EF2C0000090CDE9015496
:10309000694630460394FEF7A1F94FF4C0600090F2
:1030A000CDE90154694638460394FEF797F907B015
:1030B000F0BD000030380240000402400000024031
:1030C000104810B50E4901604FF482714160002133
:1030D0008160C1604FF400720161C0E905120822ED
:1030E000C0E90721416281620A21C162FFF722F92A
:1030F000002804D040F26A51034800F0D5FB10BD0F
:10310000003001401C0C0020484A00080D4810B552
:103110000B4901604FF461214160002181600C2264
:10312000C160C0E904128161C161FFF7EDFB0028B5
:1031300004D040F27D51044800F0B6FB10BD000001
:1031400000440040740C0020484A000802A103A07B
:10315000FDF798FEFEE70000000000004D656D4D94
:10316000616E61676500000070470907090E00285D
:1031700006DA00F00F0000F1E02080F8141D70471F
:1031800000F1E02080F80014704710B50446FDF708
:10319000E4F881B22046BDE8104000F001B800001C
:1031A0000A4601460A230148FFF79FBC740C002021
:1031B0000148FFF755B800001C0C002038B50B463D
:1031C000009204460022802100F010F8002804D06C
:1031D000606D40F020006065032038BD10B5806B45
:1031E0000021C187C186FFF73AF810BD2DE9F041F3
:1031F0001D4617460E460446DDF8188035E0681C6B
:1032000033D02DB1FEF7DAFAA0EB0800A8422CD398
:103210002068416821F0E00141606068B0F5827F7C
:103220000BD1A068B0F5004F02D0B0F5806F04D18B
:103230002068016821F040010160A06AB0F5005FDC
:103240000AD1206801684DF6FF72114001602068C4
:10325000016841F400510160012084F85100002010
:1032600084F850000320BDE8F0812068806836EAC9
:10327000000004D00020B842C1D10020F3E70120B3
:10328000F9E7000030BF0348FEF70AFB642002F0B4
:1032900049F8F7E7100C002010B501F051F9FEF7DE
:1032A00005FBBDE8104001F036BC000030B52848F1
:1032B00093B00024016841F080510160006800F083
:1032C000805011902348016841F44041016000683A
:1032D000102100F4404011900A2000900120CDE917
:1032E00003010225CDE905050820CDE907403C2072
:1032F000CDE9090504200B906846FEF781FD10B169
:1033000040F22C510EE00F20CDE90C054FF4805017
:10331000CDE90E4001210CA81094FEF7F5FB20B179
:1033200040F23A510CA000F0BFFAFEF711FD4FF445
:103330007A71B0FBF1F0FFF749FA0420FFF714FAB5
:1033400000220F21501EFEF74FFB13B030BD0000CE
:1033500040380240007000402E2E2F5372632F6DB4
:1033600061696E2E630000001048016841F470012D
:1033700001600F48016841F0010101600C4A002121
:103380000832116002680B4B1A400260031D0A4AA2
:103390001A60026822F48022026005480C30016045
:1033A00002495806803908607047000088ED00E047
:1033B00000380240FFFFF6FE1030002410B5806B8D
:1033C0000021C185C184FFF715FA10BD0168CA68E4
:1033D00022F49072CA6001684A6922F001024A61CF
:1033E000202180F83A10704710B590F83A10222941
:1033F00001D0022010BD8168B1F5805F11D0016954
:10340000002901681FD0496801F07F03816A4A1CC6
:1034100082620B70C18D491E0904090CC18518D048
:1034200026E00269816A002A0268526805D0D2B299
:103430000A80816A491C8162ECE7C2F308020A80B3
:10344000816A891CF7E74A68816A4B1C83620A70AB
:10345000E0E70168CA6822F49072CA6001684A69AC
:1034600022F001024A61202180F83A10FFF73CFB6C
:10347000002010BD2DE9F04104464068BC49884257
:1034800004D340F68511BBA000F0F2FBE06838B130
:10349000B0F5005F04D040F68611B6A000F0E8FB5E
:1034A000206950B1B0F5806F07D0B0F5C06F04D07F
:1034B00040F68711AFA000F0DBFB60694FF6F371B7
:1034C000084200D120B940F68811AAA000F0D0FB34
:1034D0002268106920F44051E068084310612268B6
:1034E000D06849F20C6188432369A168E5691943F2
:1034F00063692B4319430143D1602268506920F46A
:103500004071A06908435061E2696425B2F5004F3B
:10351000A748A84922684FF032083FD08A4201D01C
:1035200082427CD1FEF72AFC00EBC00101EB0010C7
:1035300061688900B0FBF1F6FEF720FC00EBC001EA
:1035400001EB001061688900B0FBF1F0B0FBF5F011
:103550006FF01801484306EB800108EB0110B0FB47
:10356000F5F000F0F006FEF709FC00EBC00101EBFE
:10357000001061688900B0FBF1F0B0FBF5F006EBDC
:103580000016FEF7FBFB00EBC00101EB00106168C9
:103590008900B0FBF1F7FEF7F1FBD2E08A4201D0DF
:1035A00082423DD1FEF7EAFB00EBC00101EB0010C7
:1035B00061684900B0FBF1F0B0FBF5F00601FEF7E1
:1035C000DDFB00EBC00101EB001061684900B0FBBE
:1035D000F1F7FEF7D3FB00EBC00101EB00106168CF
:1035E0004900B0FBF1F0B0FBF5F06FF01801484373
:1035F00007EB800108EBC100B0FBF5F000F0F8002C
:1036000006EB4006FEF7BAFB00EBC00101EB001031
:1036100061684900B0FBF1F7FEF7B0FB3CE055E014
:10362000FEF79CFB00EBC00101EB00106168490054
:10363000B0FBF1F0B0FBF5F00601FEF78FFB00EBFD
:10364000C00101EB001061684900B0FBF1F7FEF723
:1036500085FB00EBC00101EB001061684900B0FB85
:10366000F1F0B0FBF5F06FF01801484307EB800173
:1036700008EBC100B0FBF5F000F0F80006EB4006E7
:10368000FEF76CFB00EBC00101EB00106168490024
:10369000B0FBF1F7FEF762FB00EBC00101EB00109D
:1036A00061684900B0FBF1F0B0FBF5F06FF0180174
:1036B000484307EB800108EBC100B0FBF5F000F0D8
:1036C0000700216830448860BDE8F081FEF746FBC2
:1036D00000EBC00101EB001061688900B0FBF1F65E
:1036E000FEF73CFB00EBC00101EB001061688900B4
:1036F000B0FBF1F0B0FBF5F06FF01801484306EBBA
:10370000800108EB0110B0FBF5F000F0F006FEF7C9
:1037100025FB00EBC00101EB001061688900B0FBE4
:10372000F1F0B0FBF5F006EB0016FEF717FB00EB2F
:10373000C00101EB001061688900B0FBF1F7FEF7F2
:103740000DFB00EBC00101EB001061688900B0FBCC
:10375000F1F0B0FBF5F06FF01801484307EB800182
:1037600008EB0110B0FBF5F000F00F00A9E7000036
:10377000A137A0002E2E2F447269766572732F53E5
:10378000544D3332463478785F48414C5F44726917
:103790007665722F5372632F73746D33326634788B
:1037A000785F68616C5F756172742E630000000061
:1037B000001401400010014090F83910212901D077
:1037C000022070478168B1F5805F016A0BD04A1C06
:1037D0000262026809785160C18C491E0904090C13
:1037E000C1840ED017E009880268C1F30801516056
:1037F00001690029016A02D0491C0162ECE7891CB9
:10380000FBE70168CA6822F08002CA600068C168EC
:1038100041F04001C160002070472DE9F041984619
:1038200017460E460446069D1DE0681C1BD02DB1B0
:10383000FDF7C4FFA0EB0800A84214D92068C168B6
:1038400021F4D071C1602068416921F0010141611A
:10385000202084F8390084F83A00002084F83800E9
:103860000320BDE8F0812068006836EA000004D03B
:103870000020B842D9D00020F3E70120F9E700008A
:103880000148FEF7B9BF0000740C002002A103A09C
:10389000FDF7F8FAFEE700000000000055736167CD
:1038A000654661756C740000B2B00B46024604A117
:1038B000684600F013F8694604A0FDF7E3FA00003B
:1038C000202573204C696E65202564004572726F57
:1038D000725F48616E646C65720000000FB4084B43
:1038E00010B504A902AA039800F01CF8044602A926
:1038F000002000F0B8F9204610BC5DF814FB000071
:10390000673C000802E008C8121F08C1002AFAD16B
:1039100070477047002001E001C1121F002AFBD14F
:10392000704700002DE9FF4F8BB088460546002602
:1039300006E025280BD0DDE90D1290476D1C761CA2
:1039400028780028F5D10FB03046BDE8F08F00246C
:10395000A146A2460122AE4900E0044315F8013F0A
:10396000203B02FA03F00842F7D128782A2810D029
:103970006FF02F022878A0F13001092915D809EB42
:10398000890102EB410144F0020400EB01096D1CC6
:10399000F0E758F8041B5FEA010903D544F400542A
:1039A000C9F1000944F002046D1C28782E2817D1B3
:1039B00015F8010F44F004042A280ED06FF02F02EE
:1039C0002878A0F1300109290AD80AEB8A0102EB14
:1039D000410100EB010A6D1CF2E758F804AB6D1CC5
:1039E00028786C280FD006DC4C2817D068280DD01A
:1039F0006A2814D104E0742810D07A280FD10DE081
:103A000044F400140AE044F4801401E044F4401447
:103A10006978814202D104F580146D1C6D1C2878F0
:103A2000692865D006DC00288DD0632827D064285B
:103A300006D15DE06E2808D073282AD0752877D08B
:103A4000DDE90D129047761CE0E0C4F30250022835
:103A500009D003280DD0D8F8001004280DD00E602E
:103A600008F10408D2E0D8F80010F217C1E90062AA
:103A7000F6E7D8F800100E80F2E70E70F0E718F8BD
:103A8000041B8DF8001000208DF80100EB4601208A
:103A900003E058F804BB4FF0FF3061074FF0000718
:103AA00001D40AE07F1C57450DDA8742FADB1BF888
:103AB00007100029F6D106E07F1C8742FCDB1BF8CB
:103AC00007100029F8D1DDE90D23A9EB0700814695
:103AD000214600F0B1F83044C61904E0DDE90D12CA
:103AE0001BF8010B90477F1EF8D22146484688E01C
:103AF00058F8040BC4F302514FF00A0B032900D10C
:103B000000B2042900D140B2002802DA40422D213F
:103B100002E0210505D52B218DF82410012104E0B8
:103B200006E0E10710D02021F6E708AF089113E086
:103B300058F8040BC4F302514FF00A0B032900D1CB
:103B400080B2042900D1C0B20021EEE75946FCF74B
:103B500022FC303107F8011D0028F7D1ADEB07003A
:103B600000F1200B600702D524F4803401E04FF00F
:103B7000010ADA4502DDAAEB0B0000E000208246D4
:103B800000EB0B0108980144A9EB01000A90E00347
:103B900006D4DDE90D2321460A9800F04DF80644CD
:103BA0004FF0000908E009A911F80900DDE90D123C
:103BB000904709F10109761C08998945F3DBE00378
:103BC0000CD5DDE90D2321460A9800F035F80644AE
:103BD00004E0DDE90D1230209047761CBAF10001B7
:103BE000AAF1010AF5DC05E0DDE90D1217F8010B79
:103BF0009047761CBBF10001ABF1010BF4DC0A9895
:103C00002146DDE90D2300F005F806446D1C97E61A
:103C1000092801002DE9F041044600251E461746FB
:103C2000880404D405E039462020B0476D1C641E8A
:103C3000F9D52846BDE8F0812DE9F041044600257C
:103C40001E469046C80301D5302700E0202788048F
:103C500004D505E041463846B0476D1C641EF9D5D1
:103C60002846BDE8F0810A68531C0B60107070474D
:103C70007047000010B5074C6389984209DA24891F
:103C8000A14206DA01FB0300B0F5963F01D20249DA
:103C90000A5410BDAA000020780E00201CB50B4A63
:103CA000D180137833B10A464FF496310848FCF7B7
:103CB00036FB09E013891BB2CDE90031518900229E
:103CC0000BB2114600F03AF900201CBDAA000020FA
:103CD000780E00202DE9F843124C80462078F0B190
:103CE000404600F0B4FB2089009000226389114611
:103CF000404600F049FB0C4D0C4E00244FF4963723
:103D0000285D36F81010404600F0A6FB641CBC424B
:103D1000F6D3404600F00AF90020BDE8F883012000
:103D2000FBE70000AA000020780E0020F86F0008D2
:103D30002DE9FF4F774E884681B0B0889146A0F5B7
:103D40008051103917D01846FFF766F94FEAC00ABC
:103D500020287CD070490C5C3078002878D0002571
:103D6000601E00906D480AEB0501002610F801B0B6
:103D70000098C7B293E010255F013078684CA7F532
:103D8000806778B300264FF0010B00BF644807EB53
:103D9000460108440024008890FA90FA291B491E25
:103DA0000BFA01F010EA0A0F07D006EB090001B286
:103DB00004EB080000B20E9A09E01098800708D5BD
:103DC00006EB090001B204EB080000B20F9AFFF7FE
:103DD00051FF641CE4B2AC42E0D3761CF6B2102E64
:103DE000D4D331E0FFE7019800F031FB1020034607
:103DF00000901FFA89F21FFA88F1019800F0C4FAC6
:103E00000026A3464FF0010A07EB460101EB0B0029
:103E10000024008890FA90F9291B491E0AFA01F043
:103E200010EA090F01D00E9900E00F99019800F0F7
:103E300068FB641CE4B2AC42EED3761CF6B2102EE2
:103E4000E2D3019800F072F83648057001E006E010
:103E50002DE008EB050005B080B2BDE8F08F3248D8
:103E6000047879E70120B84010EA0B0F07D005EB82
:103E7000090001B206EB080000B20E9A09E01098A2
:103E8000800708D505EB090001B206EB080000B277
:103E90000F9AFFF7EFFE7F1E761CFFB2F6B2A64226
:103EA000E0D36D1CEDB2082DFFF45CAF2EE001985D
:103EB00000F0CDFA082000901FFA89F21FFA88F16D
:103EC0002346019800F060FA0025A4F1010B00BF21
:103ED00012480AEB05010BF0FF0710F801900026CD
:103EE0000EE00120B84010EA090F01D00E9900E061
:103EF0000F99019800F005FB7F1E761CFFB2F6B209
:103F0000A642EED36D1CEDB2082DE1D3641CE5B2E0
:103F100097E70000AA00002084630008AC5F000857
:103F200017640008A9000020A800002001680968A3
:103F30008968018AC0680122FDF70ABC2DE9F84FA3
:103F400081462D48DDE90A7B46891C461546884690
:103F5000B1423CDA03899D4239DA08EB0401491E7B
:103F60000AB2E919491E09B2002A30DB00292EDB0A
:103F7000B8F1000F03DA541C4FF0000824B2002DF2
:103F800002DA00254F1C3FB2B24202DBA6EB080268
:103F900014B2994201DB591B0FB20078C8B100205E
:103FA00012E009EB080000260FFA80FA07E070190A
:103FB00001B250465A46FFF75DFE761CB6B2BE42CD
:103FC000F5DB09F1010080B28146A042E9DBBDE8E2
:103FD000F88FB8B2009004FB07F6A3B2AAB21FFA9A
:103FE00088F1484600F0D0F9324659464846BDE8C7
:103FF000F84F00F093BA0000AA00002070B50C46FC
:10400000054600F01DFA284600F021FAEF21284667
:1040100000F064FA0321284600F04EFA8021284679
:1040200000F04AFA0221284600F046FACF2128463D
:1040300000F054FA0021284600F03EFAC12128463B
:1040400000F03AFA3021284600F036FAED212846F1
:1040500000F044FA6421284600F02EFA0321284695
:1040600000F02AFA1221284600F026FA812128467B
:1040700000F022FAE821284600F030FA852128468F
:1040800000F01AFA0021284600F016FA7821284696
:1040900000F012FACB21284600F020FA39212846F8
:1040A00000F00AFA2C21284600F006FA00212846E2
:1040B00000F002FA3421284600F0FEF902212846D9
:1040C00000F0FAF9F721284600F008FA20212846E6
:1040D00000F0F2F9EA21284600F000FA0021284613
:1040E00000F0EAF90021284600F0E6F9C021284650
:1040F00000F0F4F92321284600F0DEF9C12128461A
:1041000000F0ECF91021284600F0D6F9C521284628
:1041100000F0E4F93E21284600F0CEF92821284697
:1041200000F0CAF9C721284600F0D8F986212846B0
:1041300000F0C2F93621284600F0D0F9482128467F
:1041400000F0BAF93721284600F0C8F900212846C6
:1041500000F0B2F93A21284600F0C0F9552128466E
:1041600000F0AAF9B121284600F0B8F9002128464C
:1041700000F0A2F91821284600F07AF9B621284665
:1041800000F0ACF90821284600F096F98221284673
:1041900000F092F92721284600F08EF9F2212846F6
:1041A00000F09CF90021284600F086F926212846D7
:1041B00000F094F90121284600F07EF9E02128461C
:1041C00000F08CF90F21284600F076F931212846BD
:1041D00000F072F92B21284600F06EF90C212846D8
:1041E00000F06AF90E21284600F066F908212846F9
:1041F00000F062F94E21284600F05EF9F1212846D0
:1042000000F05AF93721284600F056F907212846D0
:1042100000F052F91021284600F04EF903212846FB
:1042200000F04AF90E21284600F046F909212846F7
:1042300000F042F90021284600F03EF9E12128462D
:1042400000F04CF90021284600F036F90E212846EE
:1042500000F032F91421284600F02EF903212846F7
:1042600000F02AF91121284600F026F907212846F6
:1042700000F022F93121284600F01EF9C12128461C
:1042800000F01AF94821284600F016F908212846BE
:1042900000F012F90F21284600F00EF90C212846F3
:1042A00000F00AF93121284600F006F936212846A7
:1042B00000F002F90F21284600F0FEF811212846EF
:1042C00000F00CF92921284600F008F92846FFF7EC
:1042D0002DFE0021284600F083F821462846FFF7EE
:1042E000DDFC1021084600F071F8002070BD0000D0
:1042F0002DE9FE4F174CDDE90D868346DDF8309041
:1043000067891D469246300608D57F081846FCF797
:1043100024F861784843A7EB500107E0700605D503
:104320001846FCF71AF8617800FB1171A4F80680B2
:1043300009E0CDF80090CDE9018652465846FFF7D6
:10434000F7FC01466D1C2B78002BF2D188B2BDE83A
:10435000FE8F0000AA00002070B5044600F077F838
:104360000421204600F0BAF8218900226068FDF798
:10437000EFF94FF0FF31204600F081F80546204666
:10438000FFF7D4FD284670BD70B5054604980B4470
:1043900010445B1E401E43EA014440EA02462A21C3
:1043A000284600F09BF82146284600F068F82B21AB
:1043B000284600F093F83146284600F060F8284679
:1043C000BDE870402C2100F089B80000034A41EAA2
:1043D000002393805070917070470000AA00002065
:1043E00070B5164A11F003030C460546D3704FF022
:1043F000F0004FF4A07106D0012B06D0022B06D09E
:10440000032B0BD107E0482402E0282404E0882491
:104410005081118102E0E82451811081284600F08A
:1044200016F83621284600F059F82146284600F0B3
:1044300043F82846BDE87040FFF778BDAA00002089
:1044400000680068016841F0400101607047018A1E
:10445000C0680022FDF77CB910B5CBB20446090A4A
:1044600000F006F82046BDE810401946AFF3008082
:104470000068006882689207FCD5C1607047F0B59B
:10448000CDB2C1F30724C1F307430646090E00F07D
:1044900013F807061946304600F00EF847EA0043C5
:1044A0002146304600F008F843EA0023294630460A
:1044B00000F002F81843F0BD02681268D16000688D
:1044C000006800E000BF81688907FBD500E000BFFD
:1044D00081680906FBD4C068C0B2704770B50D464C
:1044E0000446018940680022FDF732F9294620463A
:1044F000FFF7E2FF21896068BDE870400122FDF707
:1045000027B910B50A0ACBB204461146FFF7B0FF2F
:104510002046BDE810401946FFF7AABF70B50C0A47
:104520000546CEB2130009D021462846FFF7A0FF6A
:1045300031462846FFF79CFF5B1EF5D170BD000099
:104540002DE9F843B54C206C616C401C41F1000131
:1045500020646164608B10B1608B401E6083A08B0F
:1045600010B1A08B401EA083A08B002588B94FF40A
:10457000FA70A08300956946206B01F0BFFA00989D
:1045800038B1A7494FF080500860BFF34F8FBFF399
:104590006F8F607AA34F4FF400784FF48069C0B1F9
:1045A000A08DB0B900BFA04EA07A305C2E281AD0E2
:1045B000A07A305C2D2818D0A07A305C202821D039
:1045C000A07A305CFBF793FE70281DD0A07A208B78
:1045D000A085A08D10B1A08D401EA08500BFA08D2C
:1045E000012815D029E0A08A00E0E08AA0850122F8
:1045F00041463846FDF7ACF8002249463846FDF7FB
:10460000A7F8E6E7A08AE3E7208B00EB4000DFE7AE
:10461000002241463846FDF79BF8012249463846BC
:10462000FDF796F8A58500BFA07A401CA072607ABD
:10463000401E6072607A00B9A572E08B4FF6FF7180
:10464000884201D2401CE083208C884201D2401C69
:104650002084764F4FF480513846FDF721F806004C
:1046600000D1658308213846FDF71AF830404FF035
:1046700001030FD0218C628A914202D1491C21840E
:10468000E371618A01EB4102218C8A4202D1491C0B
:10469000218423726178491E61707DD20521617089
:1046A000A178814222D1E17881421FD06049E07037
:1046B000A1F13C02D8B1E68BA6842584A68C678D37
:1046C00021F82760678C783921F81760A371638D12
:1046D0005B1C6385638D642B00D36585638C5B1CD9
:1046E0006384638C1E2B0ED2638C63B192E0238CA7
:1046F000E384E583E38C658D01EB85014B80618D5F
:1047000022F8113086E0638C1E2B00D3658425705F
:1047100000BF00255FF0000331F8137001EB430682
:10472000B6F802C0674506D931F81370B6F802C072
:1047300021F813C077805B1CDBB21D2BECD36D1C02
:10474000EDB21D2DE6D300255FF0000332F81370A3
:1047500002EB4306B6F802C0674506D932F813707B
:10476000B6F802C022F813C077805B1CDBB21D2BA9
:10477000ECD36D1CEDB21D2DE6D300BF01251D232A
:1047800031F8137031F8156006EB4606B74202D3D4
:1047900031F81360268200E03DE05B1EDBB20F2B98
:1047A000EED86D1CEDB20F2DE9D30F255FF001039C
:1047B00031F8137031F8156006EB4606B74202D89F
:1047C00031F81360E6815B1CDBB20F2BF0D36D1E5A
:1047D000EDB21D2DEAD300BF00231D4619464FF44C
:1047E000487600BF32F81170642F09D932F8117081
:1047F000B74205D232F811705B1C3D44ADB2DBB25A
:10480000491CC9B21E29EDD3B5FBF3F16182218A9F
:10481000618200BFA070BDE8F883000000000020A6
:1048200004ED00E000000240F00B00200004024014
:10483000600A0020804888B0816841F4805181601E
:10484000816841F400618160416841F00701416085
:10485000FDF734F8FEF72AFDFEF7E0FB7748002469
:10486000016841F400110160016801F40011009138
:10487000016841F4800101600068224600F4800074
:10488000009005211120FDF7AFF81120FDF77CF80D
:10489000002205213A20FDF7A7F83A20FDF774F829
:1048A000FEF734FCFEF70CFC664865490226C0E9B9
:1048B000001640F6FF718160FCF786FF20B140F2E0
:1048C000525161A0FEF7F0FF012291036248FCF70C
:1048D0003FFF6248FEF759FC5A4800210C30A0F512
:1048E000127528605C486860802028815A48E8601A
:1048F000402028822846FFF781FB2846FFF72CFD41
:10490000DFF85C810221C8F838002846FFF768FD0F
:1049100010210846FFF75AFD0C27CDE9004751A3A7
:104920002246002128460296FFF7E2FCCDE9004727
:10493000102250A3002128460296FFF7D9FC4FF021
:104940000E09CDE9009438224EA300212846029496
:10495000FFF7CEFC074607210520FFF737FDCDE91D
:1049600000944BA33C2207F1080128460294FFF76C
:10497000BFFC102148270846FFF728FD0F20CDE98E
:10498000000446A33A46002128460294FFF7B0FCF3
:104990002846FFF79FF92846FFF759FD4F20009062
:1049A000424F49F220496C22F02300212846FFF7AC
:1049B000EBFC4FF4FA734A46791C2868FDF7F8FDC2
:1049C0002846FFF7B3FA03220021012000F078FF08
:1049D000C8F8300000282ED01422354903A8FBF770
:1049E0008CFC002103A800F0A0F8C8F834000125D1
:1049F000CDE900540023C8222EA1314801F002F96C
:104A0000CDE900540023C8222EA1324801F0FAF863
:104A1000CDE90054002364222FA1334801F0F2F8BD
:104A2000CDE900640023642230A1344801F0EAF8A3
:104A300000F06CF8FEE7FEE7002004E030380240AA
:104A400000300040100C00202E2E2F5372632F6D6B
:104A500061696E2E63000000000402400806010830
:104A6000000000202044656B6F646572206B6F64EA
:104A700075202000204D6F72736527612056302EFF
:104A8000326120004D6179203235203230323000E1
:104A900031393A31333A32320000000073617340E9
:104AA000656C706F7274616C2E706C00C871000858
:104AB000985F0008476C6F776E795461736B0000E4
:104AC00085500008577973776965746C61637A540F
:104AD00061736B00295500084E61646177616E69EE
:104AE000655461736B000000455100084C656448D3
:104AF000616E646C65725461736B000091500008C4
:104B000001460020842900D0C81C704710B500F071
:104B1000A1FC002010BD10B501F0A0F8012803D0C1
:104B2000BDE8104000F0B6BE10BD3EB504460D46CF
:104B3000B0F90800FFF7E4FF02A9CDE90001208ADF
:104B40002B4682B2D4E9001001F05CF8012801D0B4
:104B500000203EBD02983EBD2DE9F041184C0F46A5
:104B60000546E6682068001D00F07AFA38B920682A
:104B700090F82C1001208840216981432161681C34
:104B800007D137B12168BDE8F0410E48091D00F09A
:104B9000CDBA20683544B5424560216805D2A06B86
:104BA000BDE8F041091D00F0A9BA606B091D00F0D5
:104BB000A5FAA06A854200D2A562BDE8F081000096
:104BC000C8000020543B01202DE9F041054600F0CB
:104BD0000DFB2E4CA068401CA06020682C4F10B12B
:104BE000606940B32DE02560A068012829D1002626
:104BF00006EB860007EB800000F072FA761C072EA9
:104C0000F6D323488C3000F06BFA2148A03000F036
:104C100067FA1F48B43000F063FA1D48C83000F04E
:104C20005FFA1B48DC3000F05BFA19488C30606397
:104C30001430A06305E02068E96AC06A884200D8A1
:104C40002560606A401C6062E96A01202269884030
:104C50001043206101EB810007EB8000291D00F06B
:104C600065FA00F0E3FA606900280CD02068E96A70
:104C7000C06A884207D207494FF080500860BFF3EE
:104C80004F8FBFF36F8FBDE8F0810000C800002098
:104C9000783A012004ED00E070B5114E114C17E098
:104CA00000F00CFC3068B8B101F084F800F09EFA16
:104CB000F068C568281D00F0D3F9A068401EA06008
:104CC0006068401E606000F0B1FA284600F01FF8EE
:104CD00060680028E4D170BD01F06CF8F8E70000CE
:104CE000403B0120C800002030B4026C0B46002A73
:104CF0000BD0C1681144C1604468A14201D301686E
:104D0000C16030BC1846FBF7F8BA30BC704710B52C
:104D10000446006B00F09EFA2046BDE8104000F00B
:104D200099BA000010484FF47051420706D0C01DD8
:104D30000D4920F00700411AC1F570510B4A0023BC
:104D40000144C2E900030839103A21F0070111605B
:104D50004B600B600B1AC0E9001393604FF00040EA
:104D60005360D06070470000683B012014010020B0
:104D7000074C4FF08056074DFFF78EFF2068012843
:104D8000FAD92E60BFF34F8FBFF36F8FF4E70000A7
:104D9000783A012004ED00E02DE9F0479A46DDE97C
:104DA000098481466FF00303206B03EB82021044F9
:104DB000089D20F00706700707D0502080F3118867
:104DC000BFF34F8FBFF36F8FFEE723180A5C83F8A2
:104DD00034200A5C12B1401C1028F6D3002784F856
:104DE0004370072D00D30625E562C4E91157201D45
:104DF00000F081F904F1180000F07DF92461C5F19B
:104E000007006462A061E76484F850705246494626
:104E1000304600F00FF92060B8F1000F01D0C8F85B
:104E20000040BDE8F087000030B5114900E01146B0
:104E30000A688242FBD34B685C18844203D1406805
:104E400018444860084643681C18944209D1084C2D
:104E5000103C2468A24209D052681A4442600A6891
:104E600012680260814200D0086030BD0460F9E73A
:104E70001401002010B5044600F0B8F9A06B28B169
:104E80005FF0000400F0D2F9204610BD0124F9E7DC
:104E90000648416B096829B1416BC968C96849680E
:104EA000816270474FF0FF31FAE70000C800002030
:104EB00008484068401C4FF0500080F3118804D02F
:104EC000BFF34F8FBFF36F8FFEE7BFF34F8FBFF37B
:104ED0006F8FFEE71C0100202DE9F041044600F031
:104EE00085F994F9455004F1240609E0606A48B157
:104EF000304600F025FF08B100F03AFA6D1E6DB2A1
:104F0000002DF3DC4FF0FF3684F8456000F08EF999
:104F100000F06CF994F9445004F1100709E020699D
:104F200048B1384600F00CFF08B100F021FA6D1EC0
:104F30006DB2002DF3DC84F84460BDE8F04100F070
:104F400075B900002DE9F0410546002700F0B6FADA
:104F5000314E306808B9FFF7E5FEF06805424BD1E5
:104F6000C5B3083568070ED005F00700C0F108008A
:104F70000544680707D0502080F31188BFF34F8F96
:104F8000BFF36F8FFEE72DB37068854234D8224897
:104F9000103001460C6801E020460C466168A942C9
:104FA00002D221680029F7D131688C4224D00768E9
:104FB0002168016060680837411B10290FD960190A
:104FC000420708D0502080F31188BFF34F8FBFF302
:104FD0006F8FFEE710E041606560FFF725FF6168B5
:104FE0007068401A7060B268904200D2B060F06899
:104FF00001430020C4E9000100F0DCFE780707D07F
:10500000502080F31188BFF34F8FBFF36F8FFEE7FF
:105010003846BDE8F081000004010020044908681A
:1050200018B10868826C521C8264086870470000DE
:10503000C800002010B5031F4FF080741C601B1FB8
:1050400021F001011960191F044B0B6014390A602B
:10505000091F6FF0020244380A6010BDB14E00080B
:10506000D0E9013201699A60D0E901235A604A68A7
:10507000824201D182684A60002202610868401EB3
:1050800008607047FBF7AEFD0A2000F04BF9F9E726
:10509000114C124D4FF47A764FF400474FF40058FC
:1050A000002332461946206B00F02EFC0128F7D170
:1050B00000BF207830B139462846FCF71DFB01229D
:1050C000414605E041462846FCF716FB01223946D9
:1050D0002846FCF73DFBE3E7000000200004024007
:1050E00000F108014FF0FF32C0E90112C160016117
:1050F00000210160704700210161704730B50B68E5
:105100005A1C02D000F1080202E0026904E02246C3
:10511000546825689D42FAD953684B6099608A604B
:10512000516008610168491C016030BD42684A60F5
:1051300093688B6093685960916008610168491CAD
:1051400001607047264C607A78BB94F904001228FD
:1051500030D2DFE800F0090E220E10181A261C1EAD
:105160002022282426282B2D812005E0FDF72AFD6A
:1051700028E07320FAE74020FDF724FD19A11A4822
:10518000FBF7DFF81EE06520F0E76C20EEE76F200C
:10519000ECE77220EAE77420E8E76120E6E72E20DA
:1051A000E4E77020E2E76C20E6E714E08820DDE722
:1051B0008620E1E7FF2020710B480AA148380988C2
:1051C000A0F848100848FBF7C8F8401C607200BF00
:1051D0002079401C20710A2000F0A4F8B3E70000F9
:1051E0000000002070000000F00B0020502080F331
:1051F0001188BFF34F8FBFF36F8F0A494868401C77
:10520000486001280CD10848006810F0FF0F07D053
:10521000502080F31188BFF34F8FBFF36F8FFEE7ED
:10522000704700001C01002004ED00E008494868B8
:1052300028B1401E486001D180F31188704750208A
:1052400080F31188BFF34F8FBFF36F8FFEE700002D
:105250001C01002070B5002827D0144DA0F10804CF
:105260006168E868014207D1502080F31188BFF3DC
:105270004F8FBFF36F8FFEE722683AB1502080F363
:105280001188BFF34F8FBFF36F8FFEE781436160DB
:1052900000F014F960686968084468602046FFF708
:1052A000C3FDBDE8704000F085BD70BD0401002065
:1052B00006484FF47A710068B0FBF1F14FF0E0203E
:1052C000491E41610721016170470000B8000020BC
:1052D00010B5FAF7C5FF114910280ED300F1E020F0
:1052E00090F8F0030A78904207D2502080F311889A
:1052F000BFF34F8FBFF36F8FFEE7094800688968DF
:1053000000F4E060884207D9502080F31188BFF391
:105310004F8FBFF36F8FFEE710BD00001C01002010
:105320000CED00E010B5020014D00F48006B38B14E
:10533000502080F31188BFF34F8FBFF36F8FFEE7CC
:1053400000F0BCF800211046FFF706FC00F032FD2B
:10535000002807D105494FF080500860BFF34F8FF8
:10536000BFF36F8F10BD0000C800002004ED00E007
:1053700001490120C8617047C800002010B50C46E3
:1053800050B1094909681831FFF7B8FE2046BDE859
:1053900010400121FFF7E0BB502080F31188BFF3DC
:1053A0004F8FBFF36F8FFEE7C800002070B5040079
:1053B00039D01D4DE06A2968C96A884233D2A06994
:1053C000002804DB2868C06AC0F10700A061E16A18
:1053D000164E01EB8101606906EB810188421FD105
:1053E000201DFFF73DFE012150B9E06A00EB80026D
:1053F00056F8222022B92A6901FA00F082432A6174
:105400002868C06AE0622A6981401143296100EB83
:10541000800006EB8000211DBDE87040FFF786BECE
:105420002868C06AE06270BDC8000020783A012098
:1054300028B107490A6A0260C96841607047502074
:1054400080F31188BFF34F8FBFF36F8FFEE700002B
:10545000C80000201CB515480024CDE900402346B3
:10546000802213A1144800F0CDFB012809D0401C74
:105470001AD1502080F31188BFF34F8FBFF36F8F85
:10548000FEE7502080F31188BFF34F8FBFF36F8F7B
:1054900006484FF0FF312C38816201214161C46020
:1054A000BDE81C4000F086B91CBD0000F4000020DF
:1054B00049444C4500000000714D00080248016B52
:1054C000491C016370470000C80000201448016BAC
:1054D00011B10121C16170470021C1610169B1FAB7
:1054E00081F1C1F11F0101EB81020E4951F8223017
:1054F0006BB101EB820101F108034A6852684A600E
:105500009A4201D152684A60D168016070475020C8
:1055100080F31188BFF34F8FBFF36F8FFEE700005A
:10552000C8000020783A01200EB5DFF804A2814DB2
:105530004FF0000B688B002879D102217E48FEF7DE
:10554000ADFB10210846FEF741FF02270C24CDE9F0
:105550000074002279A3114677480297FEF7C8FE2F
:10556000CDE9007479A31022002173480297FEF759
:10557000BFFE0720CDE9004078A32022002102973A
:105580006D48FEF7B5FE4FF0300807210520FEF705
:105590001DFF1820CDE9000B5C46A52342464B2198
:1055A0006548FEF7CBFC688C1E21CDE90001EB8C31
:1055B000AA8C6EA17548FEF791F90F26CDE900641B
:1055C000724B424650215C480294FEF791FE688A75
:1055D00000902B8AEA896EA16C48FEF77FF9CDE92D
:1055E00000646A4B3822502153480294FEF780FE33
:1055F0002A8D6EA16548FEF771F9CDE90064634B11
:10560000402250214C480294FEF772FE102148249B
:105610000846FEF7DBFE287850B10321CDF800B034
:10562000434BCDE90117143B2246002108E07BE003
:105630000D203F4BCDE90060143B2246002102972C
:105640003D48FEF755FE00274FF058093E463C46C0
:1056500064E000BF1AF804300020842B25D00CDC55
:10566000812B25D004DC092B15D0802B29D114E007
:10567000822B20D0832B24D108E0A3F185010529BA
:105680001FD2DFE801F00C0F051A1C00452300E0D3
:1056900052230B2016E0742314E0772312E05523E5
:1056A00004200FE0572307200CE072230A2009E0B2
:1056B0005323092006E0532304E0452302E043235B
:1056C00000E00E20CDE9000B09EB071231011A486A
:1056D000CDF808B0FEF72CFB761C0F21F6B20F2E8A
:1056E0001AD37F1C0026FFB20E2F15D300BF002057
:1056F00095F80C805246A8EB010307E001EB000C83
:1057000012F80CC002F800C0401C80B28342F5DCE5
:10571000A8EB0100287300BF641CA4B2287B84425C
:1057200098D30548FEF7D6FA3220FFF7FBFD01E7D4
:10573000C80C002000000020D40900202044656B24
:105740006F646572206B6F6475202000204D6F724E
:10575000736527612056302E3261200073617340DB
:10576000656C706F7274616C2E706C00746F6E3D3E
:105770002534646D732070727A3D2534646D732016
:105780005B2532642F25645D00000000EA050020DF
:10579000272E273D2533646D7320272D273D253384
:1057A000646D7320703D25336400000057504D3DFB
:1057B000253364001CB532480168324A914207D152
:1057C000502080F31188BFF34F8FBFF36F8FFEE738
:1057D00000682C49491E884207D1502080F3118867
:1057E000BFF34F8FBFF36F8FFEE727490878019013
:1057F000FF20087008788DF800009DF800009DF8E3
:10580000002000F0F000904207D0502080F3118873
:10581000BFF34F8FBFF36F8FFEE79DF800001B4A69
:1058200000F0500010700720906005E09DF80030F7
:105830005B008DF80030401E9DF800301B06F5D44B
:10584000000200F4E0609060019808700C4820307D
:10585000016841F470010160016841F0704101602C
:10586000FFF726FD00205060FAF7C0FC08480168E9
:1058700041F040410160FAF7A9FC00201CBD000086
:1058800000ED00E071C20F4100E400E01C010020C7
:1058900034EF00E010B5502080F31188BFF34F8F34
:1058A000BFF36F8F00F0E8F918B104494FF0805052
:1058B0000860002080F3118810BD000004ED00E0B6
:1058C00070B50E46050013D0D6B105FB06F0483082
:1058D000FFF738FB040009D004F1480120468EB1DF
:1058E0000160C0E90F56012100F0C4F8204670BDE8
:1058F000502080F31188BFF34F8FBFF36F8FFEE707
:105900000020E4E70060ECE72DE9FF4F002683B0BC
:105910009B468A46040003D0BAF1000F08D011E07C
:10592000502080F31188BFF34F8FBFF36F8FFEE7D6
:10593000206C38B1502080F31188BFF34F8FBFF334
:105940006F8FFEE700F08AF9DFF824814FF000093D
:105950004FF0805748B9059838B1502080F311882E
:10596000BFF34F8FBFF36F8FFEE7FFF73FFCA56BD1
:1059700045B351462046E668FFF7B6F9BBF1000F84
:1059800013D0E660606A50B104F1240000F0D8F949
:1059900028B1C8F80070BFF34F8FBFF36F8FFFF7C8
:1059A00045FC012007B0BDE8F08F6D1EA56320689F
:1059B00010B9FFF733FB606020690028EFD004F1D5
:1059C0001000E3E7059808B11EB106E0FFF72EFCD2
:1059D00027E06846FFF72CFD0126FFF727FCFFF7BD
:1059E0006DFDFFF703FC94F94400401C01D184F8DD
:1059F000449094F94500401C01D184F84590FFF78C
:105A000015FC05A9684600F0C7F8002820460AD012
:105A1000FFF762FA00F0CEF92046FFF72BFA0028D4
:105A2000A3D00020BEE7FFF725FAD8B1206830B92F
:105A3000FFF7DCFB6068FFF7B9FCFFF7F7FB04F149
:105A400024000599FFF79AFC2046FFF745FA00F07D
:105A5000B1F9002889D1C8F80070BFF34F8FBFF3A8
:105A60006F8F82E72046FFF737FA00F0A3F97CE753
:105A700004ED00E070B50D46040025D0FFF7B6FB3D
:105A8000D4E90F20216802FB001161600021A163AD
:105A90002168A1600A46D4E90F01401E00FB0121E4
:105AA000E16021464FF0FF3001F8440F487004F1E7
:105AB00010008DB1FFF714FB04F12400FFF710FB79
:105AC000FFF7B4FB012070BD502080F31188BFF3B5
:105AD0004F8FBFF36F8FFEE721690029F0D000F0F0
:105AE0002FF90028ECD004494FF080500860BFF334
:105AF0004F8FBFF36F8FE3E704ED00E070B50E4604
:105B0000040009D0206C78B1502080F31188BFF3D5
:105B10004F8FBFF36F8FFEE7502080F31188BFF3E4
:105B20004F8FBFF36F8FFEE7206848B9606838B1C8
:105B3000502080F31188BFF34F8FBFF36F8FFEE7C4
:105B4000FFF7C6FB5020EFF3118580F31188BFF3F8
:105B50004F8FBFF36F8FA16BE06B884218D994F918
:105B60004500491CA163411C04D0401C84F8450039
:105B700001200EE0606A0028FAD004F1240000F051
:105B8000DFF80028F4D0002EF2D001203060EFE7DB
:105B9000002085F3118870BD70B50D46040019D042
:105BA00005B3FFF723FB164AD1682868431C0FD0C2
:105BB0002368126A934202D062688A421AD96268E4
:105BC000891A814216D2401A28602046FFF730FC1D
:105BD000002410E0502080F31188BFF34F8FBFF3F3
:105BE0006F8FFEE7502080F31188BFF34F8FBFF314
:105BF0006F8FFEE70124FFF719FB204670BD000000
:105C0000C80000202DE9FF5F8346DDE90E87994635
:105C100016468A469000FFF795F905001AD05420E1
:105C2000FFF790F9040012D025630021CDE902416D
:105C3000CDE900874B46324651465846FFF7ACF84F
:105C40002046FEF7C1FF012004B0BDE8F09F2846C2
:105C5000FFF700FB4FF0FF30F6E700000548416911
:105C600019B1006B18B10020704701207047022065
:105C700070470000C80000202DE9F0412E4C00279D
:105C8000206B40B1A069401CA061E06900B1012710
:105C90003846BDE8F081E668761CE66013D1606B9B
:105CA000006838B1502080F31188BFF34F8FBFF3E5
:105CB0006F8FFEE7606BA16B6163A063206A401C7D
:105CC0002062FFF7E5F8A06ADFF87080864209D30A
:105CD000606B006880B1606BC068C56868688642A8
:105CE0000DD2A0622068C06A00EB800158F8210044
:105CF0000128CAD90127C8E74FF0FF30F1E7281D76
:105D0000FFF7AEF9A86A18B105F11800FFF7A8F976
:105D1000E86A0121226981401143216100EB800181
:105D200008EB8100291DFFF701FAE86A2168C96ABA
:105D30008842CDD30127CBE7C8000020783A012064
:105D40002DE9F041C068C468ACB104F11800074601
:105D5000FFF786F9154D286B0126A0B13946144886
:105D6000FFF7E4F9E06A2968C96A88421CD9012072
:105D7000EE61BDE8F081502080F31188BFF34F8FB2
:105D8000BFF36F8FFEE7201DFFF76AF9E16A2A690A
:105D900006FA01F01043286101EB81000449B4398F
:105DA00001EB8000211DDBE70020E2E7C8000020B6
:105DB0002C3B01202DE9F0472C4D00242746286B71
:105DC00038B1FFF713FA286B401E2863286B40B1E7
:105DD00046E0502080F31188BFF34F8FBFF36F8FE1
:105DE000FEE7A968224E0120D1B3A6F1B40980468E
:105DF0003068E8B1F068C46804F11800FFF730F9C2
:105E0000201DFFF72DF9E06A2A6908FA00F1114315
:105E1000296100EB800109EB8100211DFFF786F964
:105E2000E06A2968C96A8842E2D3C5F81C80DFE7C6
:105E30000CB1FFF72DF8AC6944B14646FFF71CFFE3
:105E400000B1EE61641EF9D10020A861E86938B1A3
:105E50000849012738070860BFF34F8FBFF36F8FE2
:105E6000FFF7E4F93846BDE8F0870000C8000020DD
:105E70002C3B012004ED00E0000000007B142E3ECE
:105E80007B14AE3E0000003F0AD7233FB81E453FBB
:105E900052B85E3FD7A3703F48E17A3F0000803F91
:105EA00048E17A3FD7A3703F52B85E3FB81E453FE6
:105EB0000AD7233F0000003F7B14AE3E7B142E3EEA
:105EC000000000007B142EBE7B14AEBE000000BF9D
:105ED0000AD723BFB81E45BF52B85EBFD7A370BF55
:105EE00048E17ABF000080BF48E17ABFD7A370BF06
:105EF00052B85EBFB81E45BF0AD723BF000000BF1F
:105F00007B14AEBE7B142EBE0000803F48E17A3F7A
:105F1000D7A3703F52B85E3FB81E453F0AD7233F14
:105F20000000003F7B14AE3E7B142E3E00000000BC
:105F30007B142EBE7B14AEBE000000BF0AD723BF69
:105F4000B81E45BF52B85EBFD7A370BF48E17ABF45
:105F5000000080BF48E17ABFD7A370BF52B85EBFD0
:105F6000B81E45BF0AD723BF000000BF7B14AEBEDA
:105F70007B142EBE000000007B142E3E7B14AE3E30
:105F80000000003F0AD7233FB81E453F52B85E3F8E
:105F9000D7A3703F48E17A3F7406010885320008B4
:105FA0000000000000000000800000000000000071
:105FB000000000000E1111111F111102020E141029
:105FC00010110E001F10101E10101F0210101418B8
:105FD00010101F000411191513111100020E1511D4
:105FE00011110E00040E100E01011E00041F0A0400
:105FF00008101F001F01020E08101F007E819DA1C6
:10600000A19D817E7E810000000000000000000054
:106010000000000000000000000000000000000080
:106020000000000000000000000000000000000070
:106030000000000000000E010F110F0202040E10FC
:1060400010110E0000000E111F100E0206020302B6
:1060500006020300020416191111110002040E11A8
:1060600011110E0002040E100E011E0006001F0288
:1060700004081F0000001F020E081F00000000009F
:106080000000000000000000000000000000000010
:106090000000000000000000000000000000000000
:1060A00000000000000000000000000000000000F0
:1060B00000000000010101010000010005050500CC
:1060C000000000000A0A1F0A1F0A0A00040F140E2B
:1060D000051E040018190204081303000C1214080A
:1060E00014120D000301020000000000010204046C
:1060F0000402010004020101010204000004150E63
:1061000015040000000004041F0404000000000047
:10611000000301020000001F00000000000000005A
:106120000003030000010204081000000E11131503
:1061300019110E0002060202020207000E110102EE
:1061400004081F001F02040201110E0002060A12B9
:106150001F0202001F101E0101110E000608101E72
:1061600011110E001F110102040404000E11110E82
:1061700011110E000E11110F01020C00000303009B
:1061800003030000000303000301020001020408EE
:106190000402010000001F001F00000008040201AB
:1061A000020408000E110102040004000E11010D8A
:1061B00015150E000E1111111F1111001E11111EC7
:1061C00011111E000E11101010110E001C121111D1
:1061D00011121C001F10101E10101F001F10101E87
:1061E000101010000E11101711110F001111111FB6
:1061F000111111000302020202020300070202024F
:1062000002120C00111214181412110010101010A8
:1062100010101F00111B1515111111001111191566
:10622000131111000E11111111110E001E11111E6A
:10623000101010000E11111115120D001E11111E5B
:10624000141211000F10100E01011E001F0404048F
:10625000040404001111111111110E00111111117A
:10626000110A04001111111515150A0011110A0463
:106270000A1111001111110A040404001F01020483
:1062800008101F000704040404040700110A1F0477
:106290001F0404000701010101010700040A1100A5
:1062A000000000000000000000001F0004020100C8
:1062B0000000000000000E010F110F001010161951
:1062C00011111E0000000E1010110E0001010D131F
:1062D00011110F0000000E111F100E000609081CFE
:1062E00008080800000F11110F010E0010101619F8
:1062F0001111110002000602020207000100030151
:1063000001090600101012141814120006020202ED
:106310000202070000001A151511110000001619DD
:106320001111110000000E1111110E0000001E11BC
:106330001E10100000000D130F01010000001619BF
:106340001010100000000E100E011E0008081C089E
:10635000080906000000111111130D0000001111B1
:10636000110A04000000111515150A000000110A99
:10637000040A1100000011110F010E0000001F029D
:1063800004081F00000505050505050505050808A5
:1063900005050708080505050305050505050000B1
:1063A00000000000020103050505050403030505BF
:1063B000020402050503050505050505050502029C
:1063C0000405040505050505050505050503050581
:1063D0000505050505050505050505050503050371
:1063E0000503050503050505050505050503040564
:1063F0000305050505010505050505050505050355
:10640000010305050505050606050505060606063C
:106410000606060606060600000000000000000052
:10642000000000000000000000000000000000006C
:10643000000000000000000000000007000F800FB7
:10644000800F800F800F800700070000000000070A
:106450000007000700000000000E380E380E380E4E
:1064600038063000000000000000000000000000BE
:106470000000000000000000000C300C300C307FE9
:10648000FE7FFE0C300C300C300C307FFE7FFE0C9B
:10649000300C300C3000000000024002400FF81FAA
:1064A000F81A401A401FF00FF8025802581FF81F40
:1064B000F00240024000000000000000000E100E3C
:1064C000300E7000E001C0038007000E700C7008F1
:1064D00070000000000000000000000F001980198B
:1064E0008019800F000F080F9819F818F018E0199C
:1064F000F00F9800000000000000000700070007F0
:10650000000E00000000000000000000000000007D
:10651000000000000000000000000000F001C003C7
:106520008007000E000E000E000E00070003800121
:10653000C000F000000000000000000F0003800118
:10654000C000E0007000700070007000E001C00347
:10655000800F000000000000000000018011880989
:106560009007E007E03FFC3FFC07E007E0099011DF
:106570008801800000000000000000000000000111
:1065800080018001800FF00FF00180018001800008
:1065900000000000000000000000000000000000FB
:1065A00000000000000000000000000000070007DD
:1065B0000007000E000000000000000000000000C6
:1065C00000000000001FF81FF8000000000000009D
:1065D00000000000000000000000000000000000BB
:1065E000000000000000000000000000000700079D
:1065F000000700000000000000000000020006008C
:106600000E001C0038007000E001C0038007000E7F
:10661000001C0000000000000000000FF01C381CEF
:10662000781CF81CF81DB81DB81F381F381E381C00
:10663000380FF0000000000000000001800180031E
:10664000801F801F800380038003800380038003FA
:10665000801FF000000000000000000FE01C701C14
:10666000380038007000E001C0038007000E381CBD
:10667000381FF800000000000000000FE01C701C34
:10668000380038007003C003C0007000381C381C8C
:10669000700FE0000000000000000000E001E003D7
:1066A000E006E00CE018E01FF81FF800E000E00052
:1066B000E003F800000000000000001FF81C001CB0
:1066C000001C001C001FE01FF0007800381C381C64
:1066D000700FE0000000000000000003E007000E63
:1066E000001C001C001FF01FF81C381C381C381C34
:1066F000380FF000000000000000001FFC1C1C1CF4
:106700001C1C1C001C0038007000E001C00380034A
:1067100080038000000000000000000FF01C381C07
:10672000381C381F3807E007E01CF81C381C381CE0
:10673000380FF000000000000000000FF01C381CB3
:10674000381C381C381FF80FF8003800380070006B
:10675000E007C0000000000000000000000000038F
:10676000800380038000000000038003800380001A
:106770000000000000000000000000000000000316
:1067800080038003800000000003800380038007F3
:10679000000000000000000000007000E001C003E5
:1067A0008007000E001C001C000E00070003800183
:1067B000C000E000700000000000000000000000C9
:1067C000003FFC3FFC000000003FFC3FFC000000DD
:1067D0000000000000000000001C000E0007000385
:1067E0008001C000E00070007000E001C00380077D
:1067F000000E001C000000000003C00FF01E7818FF
:10680000380038007000E001C001C0000000000145
:10681000C001C001C0000000000FF81C1C1C1C1CA3
:106820001C1C1C1CFC1CFC1CFC1CFC1C001C001C60
:10683000001FF007F800000000000003C007E00E92
:10684000701C381C381C381C381FF81C381C381CAD
:10685000381C3800000000000000001FF00E380E49
:10686000380E380E380FF00FF00E380E380E380E86
:10687000381FF0000000000000000007F00E381C78
:10688000381C001C001C001C001C001C001C380EC6
:106890003807F000000000000000001FE00E700E3E
:1068A000380E380E380E380E380E380E380E380EB8
:1068B000701FE000000000000000001FF80E180E1E
:1068C000080E000E300FF00FF00E300E000E080E06
:1068D000181FF800000000000000001FF80E180E3E
:1068E000080E000E300FF00FF00E300E000E000EEE
:1068F000001F00000000000000000007F00E381C20
:10690000381C381C001C001C001CF81C381C380EDD
:106910003807F800000000000000001C701C701C0C
:10692000701C701C701FF01FF01C701C701C701C01
:10693000701C7000000000000000000FE0038003E6
:10694000800380038003800380038003800380032F
:10695000800FE0000000000000000001FC0070005B
:1069600070007000700070007038703870387038C7
:10697000700FE000000000000000001E380E380E0E
:10698000700EE00FC00F800F800FC00EE00E700E73
:10699000381E3800000000000000001F000E000E2E
:1069A000000E000E000E000E000E000E080E180E57
:1069B000381FF800000000000000001C1C1E3C1FD7
:1069C0007C1FFC1FFC1DDC1C9C1C1C1C1C1C1C1CA0
:1069D0001C1C1C00000000000000001C1C1C1C1ED5
:1069E0001C1F1C1F9C1DDC1CFC1C7C1C3C1C1C1C40
:1069F0001C1C1C000000000000000003E007F00E5B
:106A0000381C1C1C1C1C1C1C1C1C1C1C1C0E3807B1
:106A1000F003E000000000000000001FF00E380E40
:106A2000380E380E380FF00FF00E000E000E000E6C
:106A3000001F00000000000000000003E00F780EBF
:106A4000381C1C1C1C1C1C1C1C1C7C1CFC0FF80F68
:106A5000F8003800FC0000000000001FF00E380EA7
:106A6000380E380E380FF00FF00E700E380E380E4C
:106A7000381E3800000000000000000FF01C381C19
:106A8000381C381C000FE007F000381C381C381C7C
:106A9000380FF000000000000000001FFC19CC11AE
:106AA000C401C001C001C001C001C001C001C001DA
:106AB000C007F000000000000000001C701C701CEB
:106AC000701C701C701C701C701C701C701C701C66
:106AD000700FE000000000000000001C701C701C23
:106AE000701C701C701C701C701C701C700EE007F9
:106AF000C0038000000000000000001C1C1C1C1CC7
:106B00001C1C1C1C1C1C9C1C9C1C9C0FF80FF807BC
:106B100070077000000000000000001C701C701C5A
:106B2000700EE007C00380038007C00EE01C701CDD
:106B3000701C7000000000000000001C701C701C25
:106B4000701C701C700EE007C0038003800380037C
:106B5000800FE000000000000000001FF81C381843
:106B600038107000E001C0038007000E081C181CDC
:106B7000381FF8000000000000000007F0070007C1
:106B800000070007000700070007000700070007CD
:106B90000007F00000000000000000100018001CBA
:106BA000000E000700038001C000E0007000380004
:106BB0001C0007000000000000000007F00070004B
:106BC0007000700070007000700070007000700045
:106BD0007007F0000000000000018003C007E00E15
:106BE000701C3800000000000000000000000000E1
:106BF0000000000000000000000000000000000095
:106C00000000000000000000000000000000000084
:106C10000000007FFF7FFF000000001C001C000739
:106C2000000700000000000000000000000000005D
:106C30000000000000000000000000000000000054
:106C40000000000FE0007000700FF01C701C701C42
:106C5000700FD800000000000000001E000E000EA3
:106C6000000E000FF00E380E380E380E380E380EAB
:106C7000381BF000000000000000000000000000D1
:106C80000000000FE01C701C701C001C001C701C1D
:106C9000700FE0000000000000000000F80070002D
:106CA0007000700FF01C701C701C701C701C701C2D
:106CB000700FD8000000000000000000000000007D
:106CC0000000000FE01C701C701FF01C001C701CEA
:106CD000700FE0000000000000000003E0077007F4
:106CE00070070007001FE01FE0070007000700070C
:106CF000001FC000000000000000000000000000B5
:106D00000000000FD81C701C701C701C700FF00766
:106D1000F000701C700FE0000000001E000E000E5E
:106D2000000E000EF00F380F380E380E380E380EE9
:106D3000381E38000000000000000001C001C00142
:106D4000C000000FC001C001C001C001C001C001EE
:106D5000C00FF8000000000000000000700070008C
:106D600070000003F0007000700070007000700090
:106D7000701C700CF007E0000000001E000E000EFA
:106D8000000E000E380E700EE00FC00EE00E700EFA
:106D9000381E3800000000000000000FC001C001D4
:106DA000C001C001C001C001C001C001C001C001DB
:106DB000C00FF8000000000000000000000000000C
:106DC0000000001FF81C9C1C9C1C9C1C9C1C9C1CF8
:106DD0009C1C9C000000000000000000000000005F
:106DE0000000001FE01C701C701C701C701C701CCC
:106DF000701C700000000000000000000000000097
:106E00000000000FE01C701C701C701C701C701CBB
:106E1000700FE00000000000000000000000000013
:106E20000000001BF00E380E380E380E380E380FEA
:106E3000F00E000E001F0000000000000000000027
:106E40000000001FB038E038E038E038E038E01FDC
:106E5000E000E000E001F0000000000000000000A1
:106E60000000001EF00FF80F380E000E000E000E8E
:106E7000001F0000000000000000000000000000F3
:106E80000000000FE01C301C300F8003E018701869
:106E9000700FE0000000000000000000000100038F
:106EA0000007001FF0070007000700070007700732
:106EB0007003E0000000000000000000000000007F
:106EC0000000001C701C701C701C701C701C701C5E
:106ED000700FD8000000000000000000000000005B
:106EE0000000001C701C701C701C701C700EE007F1
:106EF000C00380000000000000000000000000004F
:106F00000000001C1C1C1C1C1C1C9C1C9C0FF8075B
:106F1000700770000000000000000000000000008A
:106F20000000001CE01CE00FC0078007800FC01CA1
:106F3000E01CE00000000000000000000000000075
:106F40000000000E380E380E380E380E3807F003E9
:106F5000E000E001C01F8000000000000000000011
:106F60000000001FE018E011C0038007000E201C85
:106F7000601FE0000000000000000001F803800333
:106F800080038007001C001C0007000380038003AF
:106F90008001F800000000000001C001C001C00134
:106FA000C001C001C001C001C001C001C001C001D9
:106FB000C001C001C00000000000001F8001C0012E
:106FC000C001C000E00038003800E001C001C0018D
:106FD000C01F8000000000000000001F1C3B9C3907
:106FE000DC38F80000000000000000000000000095
:106FF00000000000000000000000FF071F001FF855
:1070000000041084E007008010000084108000F865
:1070100018C61004FFFFE0FF000006000C0013007C
:1070200019001F00800186018C01930199019F01C5
:10703000200326032C03330339033F03C004C60493
:10704000CC04D304D904DF04600666066C0673061C
:1070500079067F06E007E607EC07F307F907FF0765
:10706000003006300C30133019301F30803186313B
:107070008C31933199319F31203326332C33333384
:1070800039333F33C034C634CC34D334D934DF340D
:10709000603666366C36733679367F36E037E637DB
:1070A000EC37F337F937FF37006006600C60136088
:1070B00019601F60806186618C61936199619F6135
:1070C000206326632C63336339633F63C064C66403
:1070D000CC64D364D964DF64606666666C6673668C
:1070E00079667F66E067E667EC67F367F967FF67D5
:1070F000009806980C98139819981F98809986996B
:107100008C99939999999F99209B269B2C9B339BB3
:10711000399B3F9BC09CC69CCC9CD39CD99CDF9C3C
:10712000609E669E6C9E739E799E7F9EE09FE69F0A
:10713000EC9FF39FF99FFF9F00C806C80CC813C8B7
:1071400019C81FC880C986C98CC993C999C99FC964
:1071500020CB26CB2CCB33CB39CB3FCBC0CCC6CC32
:10716000CCCCD3CCD9CCDFCC60CE66CE6CCE73CEBB
:1071700079CE7FCEE0CFE6CFECCFF3CFF9CFFFCF04
:1071800000F806F80CF813F819F81FF880F986F9DA
:107190008CF993F999F99FF920FB26FB2CFB33FB23
:1071A00039FB3FFBC0FCC6FCCCFCD3FCD9FCDFFCAC
:1071B00060FE66FE6CFE73FE79FE7FFEE0FFE6FF7A
:1071C000ECFFF3FFF9FFFFFFFFFFFFFFFFFFFFFFF4
:1071D000FFFFFFFFFFFFFFFFFFFFFFFFAFBB63C02E
:1071E00062C063C062B808B25DEFFFFFFFFFFFFF40
:1071F000FFFFFFFFFFFFFFFFFFFFFFFFFFFFFFFF9F
:10720000FFFFFFFFFFFFFFFFFFFFFFFFFFFFFFFF8E
:10721000FFFFFFFFFFFFFFFFFFFFFFFFFFFFFFFF7E
:10722000FFFFFFFFFFFFFFFFFFFFFFFFFFFFFFFF6E
:10723000FFFFFFFFFFFFFFFFFFFFFFFFEFC362C086
:1072400062B862B862B862B86EC3FFFFFFFFFFFFAB
:10725000FFFFFFFFFFFFFFFFFFFFFFFFFFFFFFFF3E
:10726000FFFFFFFFFFFFFFFFFFFFFFFFFFFFFFFF2E
:10727000FFFFFFFFFFFFFFFFFFFFFFFFFFFFFFFF1E
:10728000FFFFFFFFFFFFDFF7DFF7DFF7DFF7DFF7D6
:10729000DEF7FFFFFFFFFFFFFFFFFFFFFFFFFFFF27
:1072A000FFFFFFFFFFFFFFFFFFFFFFFFFFFFFFFFEE
:1072B000FFFFFFFFFFFFFFFFFFFFFFFFFFFFFFFFDE
:1072C000FFFFFFFFFFFFFFFFFFFFFFFFFFFFFFFFCE
:1072D000FFFFFFFFFFFFFFFFFFFFFFFFFFFFFFFFBE
:1072E000FFFFFFFFFFFFFFFFFFFFFFFFFFFFFFFFAE
:1072F000FFFFFFFFFFFFFFFFFFFFFFFFFFFFFFFF9E
:10730000FFFFFFFFFFFFFFFFFFFFFFFFFFFFFFFF8D
:10731000FFFFFFFFFFFFFFFFFFFFFFFFFFFFFFFF7D
:10732000FFFFFFFFFFFFFFFFFFFFFFFFFFFFFFFF6D
:10733000FFFFFFFFFFFFFFFFFFFFFFFFFFFFFFFF5D
:10734000FFFFFFFFFFFFFFFFFFFFFFFFFFFFFFFF4D
:10735000FFFFFFFFFFFFFFFFFFFFFFFFFFFFFFFF3D
:10736000FFFFFFFFFFFFFFFFFFFFFFFFFFFFFFFF2D
:10737000FFFFFFFFFFFFFFFFFFFFFFFFFFFFFFFF1D
:10738000FFFFFFFFFFFFFFFFFFFFFFFFFFFFFFFF0D
:10739000FFFFFFFFFFFFFFFFFFFFFFFFFFFFFFFFFD
:1073A000FFFFFFFFFFFFFFFFFFFFFFFFFFFFFFFFED
:1073B000FFFFFFFFFFFFFFFFFFFFD3C462B863C003
:1073C00063C063C0EBB29EF7FFFFFFFFFFFFFFFF4D
:1073D000FFFFFFFFFFFFFFFFFFFFFFFFFFFFFFFFBD
:1073E000FFFFFFFFFFFFFFFFFFFFFFFFFFFFFFFFAD
:1073F000FFFFFFFFFFFFFFFFFFFFFFFFFFFFFFFF9D
:10740000FFFFFFFFFFFFFFFFFFFFFFFFFFFFFFFF8C
:10741000FFFFFFFFFFFFFFFFFFFFFFFFCFCB63C0BB
:1074200063C063C063C063C06EC3FFFFFFFFFFFFA5
:10743000FFFFFFFFFFFFFFFFFFFFFFFFFFFFFFFF5C
:10744000FFFFFFFFFFFFFFFFFFFFFFFFFFFFFFFF4C
:10745000FFFFFFFFFFFFFFFFFFFFFFFFFFFFFFFF3C
:10746000FFFFFFFFDFFF29B205B905B905B905B96F
:1074700005B918D6FFFFFFFFFFFFFFFFFFFFFFFF6C
:10748000FFFFFFFFFFFFFFFFFFFFFFFFFFFFFFFF0C
:10749000FFFFFFFFFFFFFFFFFFFFFFFFFFFFFFFFFC
:1074A000FFFFFFFFFFFFFFFFFFFFFFFFFFFFFFFFEC
:1074B000FFFFFFFFFFFFFFFFFFFFFFFFFFFFFFFFDC
:1074C000FFFFFFFFFFFFFFFFFFFFFFFFFFFFFFFFCC
:1074D000FFFFFFFFFFFFFFFFFFFFFFFFFFFFFFFFBC
:1074E000FFFFFFFFFFFFFFFFFFFFFFFFFFFFFFFFAC
:1074F000FFFFFFFFFFFFFFFFFFFFFFFFFFFFFFFF9C
:10750000FFFFFFFFFFFFFFFFFFFFFFFFFFFFFFFF8B
:10751000FFFFFFFFFFFFFFFFFFFFFFFFFFFFFFFF7B
:10752000FFFFFFFFFFFFFFFFFFFFFFFFFFFFFFFF6B
:10753000FFFFFFFFFFFFFFFFFFFFFFFFFFFFFFFF5B
:10754000FFFFFFFFFFFFFFFFFFFFFFFFFFFFFFFF4B
:10755000FFFFFFFFFFFFFFFFFFFFFFFFFFFFFFFF3B
:10756000FFFFFFFFFFFFFFFFFFFFFFFFFFFFFFFF2B
:10757000FFFFFFFFFFFFFFFFFFFFFFFFFFFFFFFF1B
:10758000FFFFFFFFFFFFFFFFFFFFFFFFFFFFFFFF0B
:10759000FFFFFFFFFFFFFFFFD7D583B863C063C0C6
:1075A00062C0AFBBDEF7FFFFFFFFFFFFFFFFFFFF84
:1075B000FFFFFFFFFFFFFFFFFFFFFFFFFFFFFFFFDB
:1075C000FFFFFFFFFFFFFFFFFFFFFFFFFFFFFFFFCB
:1075D000FFFFFFFFFFFFFFFFFFFFFFFFFFFFFFFFBB
:1075E000FFFFFFFFFFFFFFFFFFFFFFFFFFFFFFFFAB
:1075F000FFFFFFFFFFFFFFFFFFFFFFFFCFCB63C0DA
:1076000063C063C063C063C06EC3FFFFFFFFFFFFC3
:10761000FFFFFFFFFFFFFFFFFFFFFFFFFFFFFFFF7A
:10762000FFFFFFFFFFFFFFFFFFFFFFFFFFFFFFFF6A
:10763000FFFFFFFFFFFFFFFFFFFFFFFFFFFFFFFF5A
:10764000FFFFFFFFDFFF87B963C063C063C063C094
:1076500042C0F7D5FFFFFFFFFFFFFFFFFFFFFFFF68
:10766000FFFFFFFFFFFFFFFFFFFFFFFFFFFFFFFF2A
:10767000FFFFFFFFFFFFFFFFFFFFFFFFFFFFFFFF1A
:10768000FFFFFFFFFFFFFFFFFFFFFFFFFFFFFFFF0A
:10769000FFFFFFFFFFFFFFFFFFFFFFFFFFFFFFFFFA
:1076A000FFFFFFFFFFFFFFFFFFFFFFFFFFFFFFFFEA
:1076B000FFFFFFFFFFFFFFFFFFFFFFFFFFFFFFFFDA
:1076C000FFFFFFFFFFFFFFFFFFFFFFFFFFFFFFFFCA
:1076D000FFFFFFFFFFFFFFFFFFFFFFFFFFFFFFFFBA
:1076E000FFFFFFFFFFFFFFFFFFFFFFFFFFFFFFFFAA
:1076F000FFFFFFFFFFFFFFFFFFFFFFFFFFFFFFFF9A
:10770000FFFFFFFFFFFFFFFFFFFFFFFFFFFFFFFF89
:10771000FFFFFFFFFFFFFFFFFFFFFFFFFFFFFFFF79
:10772000FFFFFFFFFFFFFFFFFFFFFFFFFFFFFFFF69
:10773000FFFFFFFFFFFFFFFFFFFFFFFFFFFFFFFF59
:10774000FFFFFFFFFFFFFFFFFFFFFFFFFFFFFFFF49
:10775000FFFFFFFFFFFFFFFFFFFFFFFFFFFFFFFF39
:10776000FFFFFFFFFFFFFFFFFFFFFFFFFFFFFFFF29
:10777000FFFFFFFFFFFF7DEF6AAA09BA08BA08BA48
:10778000B3C4FFFFFFFFFFFFFFFFFFFFFFFFFFFF90
:10779000FFFFFFFFFFFFFFFFFFFFFFFFFFFFFFFFF9
:1077A000FFFFFFFFFFFFFFFFFFFFFFFFFFFFFFFFE9
:1077B000FFFFFFFFFFFFFFFFFFFFFFFFFFFFFFFFD9
:1077C000FFFFFFFFFFFFFFFFFFFFFFFFFFFFFFFFC9
:1077D000FFFFFFFFFFFFFFFFFFFFFFFF34CDECC206
:1077E000ECC2ECC2ECC2ECC2F3CCFFFFFFFFFFFF28
:1077F000FFFFFFFFFFFFFFFFFFFFFFFFFFFFFFFF99
:10780000FFFFFFFFFFFFFFFFFFFFFFFFFFFFFFFF88
:10781000FFFFFFFFFFFFFFFFFFFFFFFFFFFFFFFF78
:10782000FFFFFFFFFFFF87B963C063C063C063C092
:1078300042C0F8D5FFFFFFFFFFFFFFFFFFFFFFFF85
:10784000FFFFFFFFFFFFFFFFFFFFFFFFFFFFFFFF48
:10785000FFFFFFFFFFFFFFFFFFFFFFFFFFFFFFFF38
:10786000FFFFFFFFFFFFFFFFFFFFFFFFFFFFFFFF28
:10787000FFFFFFFFFFFFFFFFFFFFFFFFFFFFFFFF18
:10788000FFFFFFFFFFFFFFFFFFFFFFFFFFFFFFFF08
:10789000FFFFFFFFFFFFFFFFFFFFFFFFFFFFFFFFF8
:1078A000FFFFFFFFFFFFFFFFFFFFFFFFFFFFFFFFE8
:1078B000FFFFFFFFFFFFFFFFFFFFFFFFFFFFFFFFD8
:1078C000FFFFFFFFFFFFFFFFFFFFFFFFFFFFFFFFC8
:1078D000FFFFFFFFFFFFFFFFFFFFFFFFFFFFFFFFB8
:1078E000FFFFFFFFFFFFFFFFFFFFFFFFFFFFFFFFA8
:1078F000FFFFFFFFFFFFFFFFFFFFFFFFFFFFFFFF98
:10790000FFFFFFFFFFFFFFFFFFFFFFFFFFFFFFFF87
:10791000FFFFFFFFFFFFFFFFFFFFFFFFFFFFFFFF77
:10792000FFFFFFFFFFFFFFFFFFFFFFFFFFFFFFFF67
:10793000FFFFFFFFFFFFFFFFFFFFFFFFFFFFFFFF57
:10794000FFFFFFFFFFFFFFFFFFFFFFFFFFFFFFFF47
:10795000FFFFFFFF7DF7BADEB6D555D514CD35D57F
:10796000B6D579DE5DEFDFFFFFFFFFFFFFFFFFFF13
:10797000FFFFFFFFFFFFFFFFFFFFFFFFFFFFFFFF17
:10798000FFFFFFFFFFFFFFFFFFFFFFFFFFFFFFFF07
:10799000FFFFFFFFFFFFFFFFFFFFFFFFFFFFFFFFF7
:1079A000FFFFFFFFFFFFFFFFFFFFFFFFFFFFFFFFE7
:1079B000FFFFFFFFFFFFFFFFFFFFFFFFFFFFFFFFD7
:1079C000FFFFFFFFFFFFFFFFFFFFFFFFFFFFFFFFC7
:1079D000FFFFFFFFFFFFFFFFFFFFFFFFFFFF3CEF8A
:1079E00059DE96D534D534D555D5B6D559DE3CEFCC
:1079F000DFF7FFFFFFFFFFFFFFFFFFFFFFFFFFFFBF
:107A0000FFFFFFFFDFFF87B963C063C063C063C0D0
:107A100042C0F7D5FFFFFFFFFFFFFFFFFFFFFFFFA4
:107A2000FFFFFFFFFFFFFFFFFFFFFFFFFFFFFFFF66
:107A3000FFFFFFFFFFFFFFFFFFFFFFFFFFFFFFFF56
:107A4000FFFFFFFFFFFFFFFFFFFFFFFFFFFFFFFF46
:107A5000FFFFFFFFFFFFFFFFFFFFFFFFFFFFFFFF36
:107A6000FFFFFFFFFFFFFFFFFFFFFFFFFFFFFFFF26
:107A7000FFFFFFFFFFFFFFFFFFFFFFFFFFFFFFFF16
:107A8000FFFFFFFFFFFFFFFFFFFFFFFFFFFFFFFF06
:107A9000FFFFFFFFFFFFFFFFFFFFFFFFFFFFFFFFF6
:107AA000FFFFFFFFFFFFFFFFFFFFFFFFFFFFFFFFE6
:107AB000FFFFFFFFFFFFFFFFFFFFFFFFFFFFFFFFD6
:107AC000FFFFFFFFFFFFFFFFFFFFFFFFFFFFFFFFC6
:107AD000FFFFFFFFFFFFFFFFFFFFFFFFFFFFFFFFB6
:107AE000FFFFFFFFFFFFFFFFFFFFFFFFFFFFFFFFA6
:107AF000FFFFFFFFFFFFFFFFFFFFFFFFFFFFFFFF96
:107B0000FFFFFFFFFFFFFFFFFFFFFFFFFFFFFFFF85
:107B1000FFFFFFFFFFFFFFFFFFFFFFFFFFFFFFFF75
:107B2000FFFFFFFFFFFFFFFFFFFFFFFFFFFF9EF7CE
:107B3000F3CC29BAC4B063B843C063C062C063C0A9
:107B400063C063C0A3B8A7B110C4FBE6FFFFFFFF8B
:107B5000FFFFFFFFDFFF0CB3E8B9E8B9E8B9E8B908
:107B6000E8B975CDFFFFFFFFFFFFFFFFFFFF3CEF11
:107B7000E8B1E8B9E8B9E8B9E8B9E8B996D5FFFFDE
:107B8000FFFFFFFFFFFFFFFFBEF749B2E8B9E8B90B
:107B9000E8B9E8B949B29DF7FFFFFFFFB3CCE8B9F8
:107BA000E8B9E8B9E8B9E8B951C4FFFFFFFFFFFF42
:107BB000FFFFFFFFFFFFFFFFFBE6CFC387B183B8E7
:107BC00063C063C062C062C062C062C063C083B889
:107BD00046B12DBBF7D5DFFFFFFFFFFFFFFFFFFF24
:107BE000ECB2E8B9E8B9A4B863C063C063C063C0CD
:107BF00063C087B1E8B9E8B92DBBFFFFFFFFFFFF06
:107C0000FFFFFFFFFFFFFFFFFFFFFFFFFFFFFFFF84
:107C1000FFFFFFFFFFFFFFFFFFFFFFFFFFFFFFFF74
:107C2000FFFFFFFFFFFFFFFFFFFFFFFFFFFFFFFF64
:107C3000FFFFFFFFFFFFFFFFFFFFFFFFFFFFFFFF54
:107C4000FFFFFFFFFFFFFFFFFFFFFFFFFFFFFFFF44
:107C5000FFFFFFFFFFFFFFFFFFFFFFFFFFFFFFFF34
:107C6000FFFFFFFFFFFFFFFFFFFFFFFFFFFFFFFF24
:107C7000FFFFDFFFBEF79DF79DF79EF7BEF7DFFF23
:107C8000FFFFFFFFFFFFFFFFFFFFFFFFFFFFFFFF04
:107C9000FFFFFFFFFFFFFFFFFFFFFFFFFFFFFFFFF4
:107CA000FFFFFFFFFFFFFFFFFFFFFFFFFFFFFFFFE4
:107CB000FFFFFFFFFFFFFFFFFFFFFFFFFFFFFFFFD4
:107CC000FFFFFFFFFFFFFFFFFFFFFFFFFFFFFFFFC4
:107CD000FFFFFFFFFFFFFFFFFFFFFFFFFFFFFFFFB4
:107CE000FFFFFFFFFFFFFFFFFFFFFFFFFFFFFFFFA4
:107CF000FFFFFFFFFFFFFFFFFFFFFFFFFFFFFFFF94
:107D0000FFFFFFFFFFFFFFFFFFFFFFFF38D666B15A
:107D100063C063C063C063C063C063C063C063C04B
:107D200063C063C063C063C063C0A3B830C4DFFF77
:107D3000FFFFFFFFFFFF92C463C063C063C063C067
:107D400063C049BAFFFFFFFFFFFFFFFFFFFFD3CC78
:107D500063C063C063C063C063C063C0CBBAFFFFCE
:107D6000FFFFFFFFFFFFFFFFB6D563C063C063C027
:107D700063C063C00CBBFFFFFFFFFFFFCFC363C047
:107D800063C063C063C063C06EC3FFFFFFFFFFFF3C
:107D9000FFFFFFFFFFFF71C483B863C063C063C010
:107DA00063C063C063C063C063C063C063C063C0BB
:107DB00063C063C063B8AAB27DEFFFFFFFFFFFFFA0
:107DC000A7B163C063C063C063C063C063C063C066
:107DD00063C063C063C063C009BAFFFFFFFFFFFF5A
:107DE000FFFFFFFFFFFFFFFFFFFFFFFFFFFFFFFFA3
:107DF000FFFFFFFFFFFFFFFFFFFFFFFFFFFFFFFF93
:107E0000FFFF3BE773D693D693D693D693D693D6FC
:107E100093D693D693D693D693D693D693D693D61A
:107E200093D693D693D693D693D693D693D693D60A
:107E300093D693D693D693D693D6B7D6FFFFFFFFAC
:107E4000FFFFFFFFFFFFFFFFFFFFDFFFB9DE50CEA9
:107E50004ACE45D663D682DE82DE82DE43D646D661
:107E60004BCE51CEFADEDFFFFFFFFFFFFFFFFFFF2C
:107E7000FFFFFFFFFFFFFFFFFFFFFFFFFFFFFFFF12
:107E8000FFFFFFFFFFFFFFFFFFFFFFFFFFFFFFFF02
:107E9000FFFFFFFFFFFFFFFFFFFFFFFFFFFFFFFFF2
:107EA000FFFFFFFFFFFFFFFFFFFFFFFFFFFFFFFFE2
:107EB000FFFFFFFFFFFFFFFFFFFFFFFFFFFFFFFFD2
:107EC000FFFFFFFFFFFFFFFFFFFFFFFFFFFFFFFFC2
:107ED000FFFFFFFFFFFFFFFFFFFFFFFFFFFFFFFFB2
:107EE000FFFFFFFFFFFFFFFFFFFF99DEC4B863C086
:107EF00063C063C063C063C083B045B187B125B1BF
:107F000083B863C063C063C063C063C063C0CFBBDA
:107F1000FFFFFFFFFFFF7EF7C4B063C063C063C015
:107F200063C0A3B8FBE6FFFFFFFFFFFFFFFF8ABAB6
:107F300063C063C063C063C063C063C0C4B87DEF87
:107F4000FFFFFFFFFFFFFFFFECBA63C063C063C02A
:107F500063C063B859DEFFFFFFFFFFFFCFC363C0FD
:107F600063C063C063C063C06EC3FFFFFFFFFFFF5A
:107F7000FFFFFFFFB3C463C063C063C063C063C0DF
:107F800063C063B805B125B105B183B063C063C0F8
:107F900063C063C063C063C0ECB2FFFFFFFFFFFFBD
:107FA00087B142B842B863C063C063C063C063C0F6
:107FB00063C062B842B842B8E8B1FFFFFFFFFFFFFD
:107FC000FFFFFFFFFFFFFFFFFFFFFFFFFFFFFFFFC1
:107FD000FFFFFFFFFFFFFFFFFFFFFFFFFFFFFFFFB1
:107FE000FFFF94D680FF80FF80FF80FF80FF80FF2F
:107FF00080FF80FF80FF80FF80FF80FF80FF80FF89
:1080000080FF80FF80FF80FF80FF80FF80FF80FF78
:1080100080FF80FF80FF80FF80FF2BC6FFFFFFFFF8
:10802000FFFFFFFFFFFF7DEF50CE44D620F760FF3C
:1080300060FF60FF60FF60FF60FF60FF60FF60FF48
:1080400060FF80FF00EF25CE51CE7DEFFFFFFFFFE9
:10805000FFFFFFFFFFFFFFFFFFFFFFFFFFFFFFFF30
:10806000FFFFFFFFFFFFFFFFFFFFFFFFFFFFFFFF20
:10807000FFFFFFFFFFFFFFFFFFFFFFFFFFFFFFFF10
:10808000FFFFFFFFFFFFFFFFFFFFFFFFFFFFFFFF00
:10809000FFFFFFFFFFFFFFFFFFFFFFFFFFFFFFFFF0
:1080A000FFFFFFFFFFFFFFFFFFFFFFFFFFFFFFFFE0
:1080B000FFFFFFFFFFFFFFFFFFFFFFFFFFFFFFFFD0
:1080C000FFFFFFFFFFFFFFFFFFFFECBA63C063C0CE
:1080D00063C063C063C08EBB7DEFDFFFDFFFDFFFE8
:1080E0005DEF51C483B863C063C063C063C062B84E
:1080F000FBE6FFFFFFFFFFFF8EBB63C063C063C0F3
:1081000063C063C092C4FFFFFFFFFFFF7DEFC4B0F9
:1081100063C063C063C063C063C063C063C096D5FF
:10812000FFFFFFFFFFFF9DEFA3B063C063C063C00D
:1081300063C008B2DFFFFFFFFFFFFFFFEFC363C0B5
:1081400063C063C063C063C06EC3FFFFFFFFFFFF78
:10815000FFFFBEF746B163C063C063C063C083B8AE
:1081600051C43CEFDFFFDFFFDFFF5DEF51C463C0B1
:1081700063C063C063C063C0A3B0BEF7FFFFFFFF6F
:108180001CEFDBE6DBE666B163C063C063C063C0BF
:1081900042C034C5FBE6FBE61CEFFFFFFFFFFFFF1D
:1081A000FFFFFFFFFFFFFFFFFFFFFFFFFFFFFFFFDF
:1081B000FFFFFFFFFFFFFFFFFFFFFFFFFFFFFFFFCF
:1081C000FFFF94D660FF60FF60FF80FF80FF80FFAD
:1081D00080FF80FF80FF80FF80FF80FF80FF80FFA7
:1081E00080FF80FF80FF80FF80FF80FF80FF80FF97
:1081F00080FF80FF80FF60FF60FF2BC6FFFFFFFF57
:10820000FFFFFFFF75D663D660FF60FF60FF60FF72
:1082100040FF80F6C0ED61ED21ED81EDE0F5A0F6C7
:1082200040FF60FF60FF60FF60FF63D674CEDFFF3A
:10823000FFFFFFFFFFFFFFFFFFFFFFFFFFFFFFFF4E
:10824000FFFFFFFFFFFFFFFFFFFFFFFFFFFFFFFF3E
:10825000FFFFFFFFFFFFFFFFFFFFFFFFFFFFFFFF2E
:10826000FFFFFFFFFFFFFFFFFFFFFFFFFFFFFFFF1E
:10827000FFFFFFFFFFFFFFFFFFFFFFFFFFFFFFFF0E
:10828000FFFFFFFFFFFFFFFFFFFFFFFFFFFFFFFFFE
:10829000FFFFFFFFFFFFFFFFFFFFFFFFFFFFFFFFEE
:1082A000FFFFFFFFFFFFFFFFFFFF86B163C063C05B
:1082B00063C063C063C0F4C4DFFFFFFFFFFFFFFFC5
:1082C000FFFFFFFF8EBB46B146B166B166B146B156
:1082D00075CDFFFFFFFFFFFF9ADE83B863C063C069
:1082E00063C063C0E8B1FFFFFFFFFFFFB6D562C008
:1082F00063C063C083B8A3B063C063C063C02DBB59
:10830000FFFFFFFFFFFF14CD63C063C063C063C006
:1083100063C055CDFFFFFFFFFFFFFFFFEFC363C04B
:1083200063C063C063C063C06EC3FFFFFFFFFFFF96
:10833000FFFF3CEF05B1E4B0E4B8E4B8E4B0ABB2A1
:10834000FFFFFFFFFFFFFFFFFFFFFFFFBEF705B1CE
:1083500063C063C063C063C063B89DEFFFFFFFFFEE
:10836000FFFFFFFFFFFF87B963C063C063C063C047
:1083700042C0F7D5FFFFFFFFFFFFFFFFFFFFFFFF3B
:10838000FFFFFFFFFFFFFFFFFFFFFFFFFFFFFFFFFD
:10839000FFFFFFFFFFFFFFFFFFFFFFFFFFFFFFFFED
:1083A000FFFF94D660FF60FF21DC42D262D262D22E
:1083B00062D262D262D262D262D262D262D262D21D
:1083C00062D262D262D262D262D262D262D262D20D
:1083D00062D262D2C2D240FF60FF2BC6FFFFFFFF16
:1083E000DFFF0FC600EF60FF60FF20FFC1E482D215
:1083F00003C163C063C063C063C063C043C083C0C4
:1084000022C1A2D201E520FF60FF60FF20F7EDC589
:10841000DFFFFFFFFFFFFFFFFFFFFFFFFFFFFFFF8C
:10842000FFFFFFFFFFFFFFFFFFFFFFFFFFFFFFFF5C
:10843000FFFFFFFFFFFFFFFFFFFFFFFFFFFFFFFF4C
:10844000FFFFFFFFFFFFFFFFFFFFFFFFFFFFFFFF3C
:10845000FFFFFFFFFFFFFFFFFFFFFFFFFFFFFFFF2C
:10846000FFFFFFFFFFFFFFFFFFFFFFFFFFFFFFFF1C
:10847000FFFFFFFFFFFFFFFFFFFFFFFFFFFFFFFF0C
:10848000FFFFFFFFFFFFFFFFFFFF29BA63C063C0CD
:1084900063C063C063C063B8A7B10CBB71CC96D591
:1084A000BAE69EF7FFFFFFFFFFFFFFFFFFFFFFFFA3
:1084B000FFFFFFFFFFFFFFFFFFFF4AB263C063C084
:1084C00063C063C083B89ADEFFFFFFFF4DBB63C08C
:1084D00063C063C008B2CBBA63C063C063C0E4B01A
:1084E000DEF7FFFFFFFF6ABA63C063C063C063C00B
:1084F00025B1BEF7FFFFFFFFFFFFFFFFEFC363C024
:1085000063C063C063C063C06EC3FFFFFFFFFFFFB4
:10851000FFFFFFFFBEF7BEF7BEF7BEF7BEF7DEF701
:10852000FFFFDFFFBEF73CEF9AE6B6D56EBB63B840
:1085300063C063C063C063C063B89EF7FFFFFFFF03
:10854000FFFFFFFFDFFF87B963C063C063C063C085
:1085500042C0F7D5FFFFFFFFFFFFFFFFFFFFFFFF59
:10856000FFFFFFFFFFFFFFFFFFFFFFFFFFFFFFFF1B
:10857000FFFFFFFFFFFFFFFFFFFFFFFFFFFFFFFF0B
:10858000FFFF94D660FF60FFE2D263C063C063C0A8
:1085900063C063C063C063C063C063C063C063C0C3
:1085A00063C063C063C063C063C063C063C063C0B3
:1085B00063C063C003C140FF60FF2BC6FFFFFFFF26
:1085C00031CE40F760FF60FF81E403C163C063C048
:1085D00063C063C063C063C063C063C063C063C083
:1085E00063C063C063C003C161E460FF60FF40F724
:1085F0000EC6FFFFFFFFFFFFFFFFFFFFFFFFFFFFB5
:10860000FFFFFFFFFFFFFFFFFFFFFFFFFFFFFFFF7A
:10861000FFFFFFFFFFFFFFFFFFFFFFFFFFFFFFFF6A
:10862000FFFFFFFFFFFFFFFFFFFFFFFFFFFFFFFF5A
:10863000FFFFFFFFFFFFFFFFFFFFFFFFFFFFFFFF4A
:10864000FFFFFFFFFFFFFFFFFFFFFFFFFFFFFFFF3A
:10865000FFFFFFFFFFFFFFFFFFFFFFFFFFFFFFFF2A
:10866000FFFFFFFFFFFFFFFFFFFFD6D583B863C00B
:1086700063C063C063C063C063C063C063C063C0E2
:1086800042B883B086B1ECBAB2CCBADEDFFFFFFFEE
:10869000FFFFFFFFFFFFFFFFFFFF96D562C063C034
:1086A00063C063C063C010C4FFFFBEF746B163C0C0
:1086B00063C063C072C475CD63C063C063C042C091
:1086C000F7D5FFFF1CE7A3B863C063C063C063C0F6
:1086D00010C4FFFFFFFFFFFFFFFFFFFFEFC363C0FB
:1086E00063C063C063C063C06EC3FFFFFFFFFFFFD3
:1086F000FFFFFFFFFFFFFFFF7DEF96D5CFC3ABBAB4
:10870000A7B105B183B842B842B862C063C063C0C4
:1087100063C063C063C063C063B89EF7FFFFFFFF21
:10872000FFFFFFFFDFFF87B963C063C063C063C0A3
:1087300042C0F7D5FFFFFFFFFFFFFFFFFFFFFFFF77
:10874000FFFFFFFFFFFFFFFFFFFFFFFFFFFFFFFF39
:10875000FFFFFFFFFFFFFFFFFFFFFFFFFFFFFFFF29
:10876000FFFF94D660FF60FFE2D263C063C063C0C6
:1087700063C063C063C063C063C063C063C063C0E1
:1087800063C063C063C063C063C063C063C063C0D1
:1087900063C063C0E3C040FF60FF2BC6FFFFFADE8B
:1087A000C1E660FF40FFC2D263C063C063C063C064
:1087B00063C063C063C063C063C063C063C063C0A1
:1087C00063C063C063C063C063C042D200FF60FF88
:1087D00000EFB8D6FFFFFFFFFFFFFFFFFFFFFFFF28
:1087E000FFFFFFFFFFFFFFFFFFFFFFFFFFFFFFFF99
:1087F000FFFFFFFFFFFFFFFFFFFFFFFFFFFFFFFF89
:10880000FFFFFFFFFFFFFFFFFFFFFFFFFFFFFFFF78
:10881000FFFFFFFFFFFFFFFFFFFFFFFFFFFFFFFF68
:10882000FFFFFFFFFFFFFFFFFFFFFFFFFFFFFFFF58
:10883000FFFFFFFFFFFFFFFFFFFFFFFFFFFFFFFF48
:10884000FFFFFFFFFFFFFFFFFFFFFFFFF7D5C8B1EF
:1088500063B863C063C063C063C063C063C063C008
:1088600063C063C063C063C063C063B8C8B176D57A
:10887000FFFFFFFFFFFFFFFFFFFFBEF766B163C013
:1088800063C063C063C066B1FFFF59DE63B863C0F5
:1088900063C083B8DAE69EF7A4B063C063C063C068
:1088A0006EC3FFFFB2CC63C063C063C063C083B854
:1088B0003CE7FFFFFFFFFFFFFFFFFFFFEFC363C0CA
:1088C00063C063C063C063C06EC3FFFFFFFFFFFFF1
:1088D000FFFFFFFF1CE72DBBA3B063C063C063C0F5
:1088E00063C063C063C063C063C063C083B883B840
:1088F00063C063C063C063C063B89EF7FFFFFFFF40
:10890000FFFFFFFFDFFF87B963C063C063C063C0C1
:1089100042C0F7D5FFFFFFFFFFFFFFFFFFFFFFFF95
:10892000FFFFFFFFFFFFFFFFFFFFFFFFFFFFFFFF57
:10893000FFFFFFFFFFFFFFFFFFFFFFFFFFFFFFFF47
:10894000FFFF94D660FF60FFE2D263C063C063C0E4
:1089500063C063C063C063C063C063C063C063C0FF
:1089600063C063C063C063C063C063C063C063C0EF
:1089700063C063C0E3C040FF60FF2BC6FFFF2DCE86
:1089800060FF60FF81DB63C063C063C063C063C01E
:1089900063C063C063C063C063C063C063C063C0BF
:1089A00063C063C063C063C063C063C0C2D260FF02
:1089B00060FF2ACEFFFFFFFFFFFFFFFFFFFFFFFF6C
:1089C000FFFFFFFFFFFFFFFFFFFFFFFFFFFFFFFFB7
:1089D000FFFFFFFFFFFFFFFFFFFFFFFFFFFFFFFFA7
:1089E000FFFFFFFFFFFFFFFFFFFFFFFFFFFFFFFF97
:1089F000FFFFFFFFFFFFFFFFFFFFFFFFFFFFFFFF87
:108A0000FFFFFFFFFFFFFFFFFFFFFFFFFFFFFFFF76
:108A1000FFFFFFFFFFFFFFFFFFFFFFFFFFFFFFFF66
:108A2000FFFFFFFFFFFFFFFFFFFFFFFFFFFFDEF77F
:108A300038DECFC308B2C4B863B863C063C063C0D4
:108A400063C063C063C063C063C063C063C063B816
:108A500051C4FFFFFFFFFFFFFFFFFFFF72C463C0B2
:108A600063C063C063C062C038DE10C463C063C04B
:108A700063C0E8B1DFFFFFFFECBA63C063C063C04F
:108A800046B1BEF708B263C063C063C063C0ECBA4E
:108A9000FFFFFFFFFFFFFFFFFFFFFFFFEFC363C00D
:108AA00063C063C063C063C06EC3FFFFFFFFFFFF0F
:108AB000FFFFFBE645B163C063C063C063C063C032
:108AC00063B8C4B8A7B1ABBAF0C375D5DBE646B19D
:108AD00063C063C063C063C063B89EF7FFFFFFFF5E
:108AE000FFFFFFFFDFFF87B963C063C063C063C0E0
:108AF00042C0F7D5FFFFFFFFFFFFFFFFFFFFFFFFB4
:108B0000FFFFFFFFFFFFFFFFFFFFFFFFFFFFFFFF75
:108B1000FFFFFFFFFFFFFFFFFFFFFFFFFFFFFFFF65
:108B2000FFFF94D660FF60FFE2D263C063C063C002
:108B300063C063C063C063C063C063C063C063C01D
:108B400063C063C063C063C063C063C063C063C00D
:108B500063C063C0E3C040FF60FF2BC6BEF764D6AE
:108B600060FFA0F6A3C063C063C063C063C063C0FE
:108B700063C063C063C063C063C063C063C063C0DD
:108B800063C063C063C063C063C063C083C020F6BA
:108B900060FF62DE9DF7FFFFFFFFFFFFFFFFFFFFAC
:108BA000FFFFFFFFFFFFFFFFFFFFFFFFFFFFFFFFD5
:108BB000FFFFFFFFFFFFFFFFFFFFFFFFFFFFFFFFC5
:108BC000FFFFFFFFFFFFFFFFFFFFFFFFFFFFFFFFB5
:108BD000FFFFFFFFFFFFFFFFFFFFFFFFFFFFFFFFA5
:108BE000FFFFFFFFFFFFFFFFFFFFFFFFFFFFFFFF95
:108BF000FFFFFFFFFFFFFFFFFFFFFFFFFFFFFFFF85
:108C0000FFFFFFFFFFFFFFFFFFFFFFFFFFFFFFFF74
:108C1000FFFFFFFFFFFF7DF79AE655D530C42DC358
:108C2000E8B1C4B062C063C063C063C063C063C066
:108C3000A4B07DF7FFFFFFFFFFFFFFFF5DEFC4B0B4
:108C400063C063C063C063C08EBBC8B163C063C090
:108C500063C051C4FFFFFFFF96D563C063C063C00C
:108C600063B834C583B863C063C063C063B838DE1B
:108C7000FFFFFFFFFFFFFFFFFFFFFFFFEFC363C02B
:108C800063C063C063C063C06EC3FFFFFFFFFFFF2D
:108C9000FFFF0CBB63C063C063C063C063C029B285
:108CA000F8D57DEFFFFFFFFFFFFFFFFFDEF746B1C7
:108CB00063C063C063C063C063B89EF7FFFFFFFF7C
:108CC000FFFFFFFFDFFF87B963C063C063C063C0FE
:108CD00042C0F7D5FFFFFFFFFFFFFFFFFFFFFFFFD2
:108CE000FFFFFFFFFFFFFFFFFFFFFFFFFFFFFFFF94
:108CF000FFFFFFFFFFFFFFFFFFFFFFFFFFFFFFFF84
:108D0000FFFF94D660FF60FFE2D263C063C063C020
:108D100063C063C063C063C063C063C063C063C03B
:108D200063C063C063C063C063C063C063C063C02B
:108D300063C063C0E3C040FF60FF2BC67DEFA1E6C8
:108D400060FF21ED63C063C063C063C063C063C0E4
:108D500063C063C063C063C063C063C063C063C0FB
:108D600063C063C063C063C063C063C063C081E4A9
:108D700060FFC0EE3CE7FFFFFFFFFFFFFFFFFFFFCD
:108D8000FFFFFFFFFFFFFFFFFFFFFFFFFFFFFFFFF3
:108D9000FFFFFFFFFFFFFFFFFFFFFFFFFFFFFFFFE3
:108DA000FFFFFFFFFFFFFFFFFFFFFFFFFFFFFFFFD3
:108DB000FFFFFFFFFFFFFFFFFFFFFFFFFFFFFFFFC3
:108DC000FFFFFFFFFFFFFFFFFFFFFFFFFFFFFFFFB3
:108DD000FFFFFFFFFFFFFFFFFFFFFFFFFFFFFFFFA3
:108DE000FFFFFFFFFFFFFFFF35CDCBC2CBC2CBC2E2
:108DF000CBC2CBC251C4FFFFFFFFFFFFFFFFFFFF4E
:108E0000FFFFDEF714C563B863C063C063C063C00F
:108E100042B8DBE6FFFFFFFFFFFFFFFFFFFF4DBB99
:108E200063C063C063C063C0C4B083B863C063C0C1
:108E300063B8BAE6FFFFFFFF9EF7E4B063C063C00C
:108E400063C004A963C063C063C063C0E8B1FFFF2F
:108E5000FFFFFFFFFFFFFFFFFFFFFFFFEFC363C049
:108E600063C063C063C063C06EC3FFFFFFFFFFFF4B
:108E7000FFFF66B163C063C063C063C0A3B83CE7D3
:108E8000FFFFFFFFFFFFFFFFFFFFFFFF79DE83B85C
:108E900063C063C063C063C063B89EF7FFFFFFFF9A
:108EA000FFFFFFFFDFFF87B963C063C063C063C01C
:108EB00042C0F8D5FFFFFFFFFFFFFFFFFFFFFFFFEF
:108EC000FFFFFFFFFFFFFFFFFFFFFFFFFFFFFFFFB2
:108ED000FFFFFFFFFFFFFFFFFFFFFFFFFFFFFFFFA2
:108EE000FFFF94D660FF60FFE2D263C063C063C03F
:108EF00063C063C063C063C063C063C063C063C05A
:108F000063C063C063C063C063C063C063C063C049
:108F100063C063C0E3C040FF60FF2BC67CEFA1E6E7
:108F200060FF01E563C063C063C063C063C063C02A
:108F300063C063C063C063C063C063C063C063C019
:108F400063C063C063C063C063C063C063C061E4E7
:108F500060FFE0EE3BE7FFFFFFFFFFFFFFFFFFFFCC
:108F6000FFFFFFFFFFFFFFFFFFFFFFFFFFFFFFFF11
:108F7000FFFFFFFFFFFFFFFFFFFFFFFFFFFFFFFF01
:108F8000FFFFFFFFFFFFFFFFFFFFFFFFFFFFFFFFF1
:108F9000FFFFFFFFFFFFFFFFFFFFFFFFFFFFFFFFE1
:108FA000FFFFFFFFFFFFFFFFFFFFFFFFFFFFFFFFD1
:108FB000FFFFFFFFFFFFFFFFFFFFFFFFFFFFFFFFC1
:108FC000FFFFFFFFFFFFFFFF14CD63C063C063C05F
:108FD00063C063C0C4B818D6FFFFFFFFFFFFFFFFE9
:108FE000FFFFFFFF59D663B863C063C063C063C0AF
:108FF000A3B07DEFFFFFFFFFFFFFFFFFFFFF9ADE44
:1090000063B863C063C063C063C063C063C063C050
:10901000C7B1DFFFFFFFFFFFFFFF0CBB63C063C0F3
:1090200063C063C063C063C063C063C014CDFFFF8F
:10903000FFFFFFFFFFFFFFFFFFFFFFFFEFC363C067
:1090400063C063C063C063C06EC3FFFFFFFFFFFF69
:10905000FFFF86B163C063C063C063C083B838D606
:10906000FFFFFFFFFFFFFFFFFFFF79DE87B163C058
:1090700063C063C063C063C063B89EF7FFFFFFFFB8
:10908000FFFFFFFFFFFFA7B963C063C063C063C0FA
:1090900042C096CDFFFFFFFFFFFFFFFFFFFFFFFF77
:1090A000FFFFFFFFFFFFFFFFFFFFFFFFFFFFFFFFD0
:1090B000FFFFFFFFFFFFFFFFFFFFFFFFFFFFFFFFC0
:1090C000FFFF94D660FF60FFE2D263C063C063C05D
:1090D00063C063C063C063C063C063C063C063C078
:1090E00063C063C063C063C063C063C063C063C068
:1090F00063C063C0E3C040FF60FF2BCEBEF763D602
:1091000060FF61F683C063C063C063C063C063C0B7
:1091100063C063C063C063C063C063C063C063C037
:1091200063C063C063C063C063C063C063C0C0ED9D
:1091300060FF82DE7DEFFFFFFFFFFFFFFFFFFFFF0E
:10914000FFFFFFFFFFFFFFFFFFFFFFFFFFFFFFFF2F
:10915000FFFFFFFFFFFFFFFFFFFFFFFFFFFFFFFF1F
:10916000FFFFFFFFFFFFFFFFFFFFFFFFFFFFFFFF0F
:10917000FFFFFFFFFFFFFFFFFFFFFFFFFFFFFFFFFF
:10918000FFFFFFFFFFFFFFFFFFFFFFFFFFFFFFFFEF
:10919000FFFFFFFFFFFFFFFFFFFFFFFFFFFFFFFFDF
:1091A000FFFFFFFFFFFFFFFF7DEF25B163C063C03F
:1091B00063C063C063C083B829BACFC371CC92C403
:1091C00031C4CBBAC4B863C063C063C063C063C0FA
:1091D0000CB3FFFFFFFFFFFFFFFFFFFFFFFFFFFFDE
:1091E00049B263C063C063C063C063C063C063C08F
:1091F00010C4FFFFFFFFFFFFFFFFB6D562C063C0D3
:1092000063C063C063C063C063C025B19EF7FFFF46
:10921000FFFFFFFFFFFFFFFFFFFFFFFFEFC363C085
:1092200063C063C063C063C06EC3FFFFFFFFFFFF87
:10923000FFFF0CBB63C063C063C063C063C0C4B83E
:109240008EC3B3CCD3CC10C44ABA83B863C063C056
:1092500063C063C063C063C063B87EF7FFFFFFFFF6
:10926000FFFFFFFFFFFF6ABA63C063C063C063C054
:1092700063C0E5B849BA6ABA8EBBFFFFFFFFFFFFC4
:10928000FFFFFFFFFFFFFFFFFFFFFFFFFFFFFFFFEE
:10929000FFFFFFFFFFFFFFFFFFFFFFFFFFFFFFFFDE
:1092A000FFFF94D660FF60FFE2D263C063C063C07B
:1092B00063C063C063C063C063C063C063C063C096
:1092C00063C063C063C063C063C063C063C063C086
:1092D00063C063C0E3C040FF60FF2BC6FFFF2BCE1F
:1092E00060FF60FFC2D263C063C063C063C063C07D
:1092F00063C063C063C063C063C063C063C063C056
:1093000063C063C063C063C063C063C0E2C940FFA1
:1093100060FF28CEDFFFFFFFFFFFFFFFFFFFFFFF24
:10932000FFFFFFFFFFFFFFFFFFFFFFFFFFFFFFFF4D
:10933000FFFFFFFFFFFFFFFFFFFFFFFFFFFFFFFF3D
:10934000FFFFFFFFFFFFFFFFFFFFFFFFFFFFFFFF2D
:10935000FFFFFFFFFFFFFFFFFFFFFFFFFFFFFFFF1D
:10936000FFFFFFFFFFFFFFFFFFFFFFFFFFFFFFFF0D
:10937000FFFFFFFFFFFFFFFFFFFFFFFFFFFFFFFFFD
:10938000FFFFFFFFFFFFFFFFFFFF59DE05B163C0D7
:1093900063C063C063C063C063C063C063C063C0B5
:1093A00063C063C063C063C063C063C063C029B2ED
:1093B0007DEFFFFFFFFFFFFFFFFFFFFFFFFFFFFF4F
:1093C00075CD63C063C063C063C063C063C042B88F
:1093D0009ADEFFFFFFFFFFFFFFFF9EF705B163C0AF
:1093E00063C063C063C063C063C0EFC3FFFFFFFF20
:1093F000FFFFFFFFFFFFFFFFFFFFFFFFEFC363C0A4
:1094000063C063C063C063C06EC3FFFFFFFFFFFFA5
:10941000FFFF99DEA3B863C063C063C063C063C0CD
:1094200063C063C063C063C063C063C0C4B825B118
:1094300063C063C063C063C062B859DEFFFFFFFF53
:10944000FFFFFFFFFFFF92C463C063C063C063C040
:1094500063C063C063C063C009BAFFFFFFFFFFFFC3
:10946000FFFFFFFFFFFFFFFFFFFFFFFFFFFFFFFF0C
:10947000FFFFFFFFFFFFFFFFFFFFFFFFFFFFFFFFFC
:10948000FFFF94D660FF60FF21EDA3C063C063C0FF
:1094900063C063C063C063C063C063C063C063C0B4
:1094A00063C063C063C063C063C063C063C063C0A4
:1094B00063C063C0E3C040FF60FF2BC6FFFFB9D6A7
:1094C000E0EE60FF00FFE2C963C063C063C063C039
:1094D00063C063C063C063C063C063C063C063C074
:1094E00063C063C063C063C063C043C980F660FFEC
:1094F00040F754CEFFFFFFFFFFFFFFFFFFFFFFFF1F
:10950000FFFFFFFFFFFFFFFFFFFFFFFFFFFFFFFF6B
:10951000FFFFFFFFFFFFFFFFFFFFFFFFFFFFFFFF5B
:10952000FFFFFFFFFFFFFFFFFFFFFFFFFFFFFFFF4B
:10953000FFFFFFFFFFFFFFFFFFFFFFFFFFFFFFFF3B
:10954000FFFFFFFFFFFFFFFFFFFFFFFFFFFFFFFF2B
:10955000FFFFFFFFFFFFFFFFFFFFFFFFFFFFFFFF1B
:10956000FFFFFFFFFFFFFFFFFFFFFFFF5DEFCFC329
:1095700005B142C063C063C063C063C063C063C061
:1095800063C063C063C063C062B8C7B1F3CCDFFF20
:10959000FFFFFFFFFFFFFFFFFFFFFFFFFFFFFFFFDB
:1095A000BEF745B142C042C042C042C062C066B1CF
:1095B000FFFFFFFFFFFFFFFFFFFFFFFF2DBB42C0CD
:1095C00042C042C042C042C083B01BE7FFFFFFFF62
:1095D000FFFFFFFFFFFFFFFFFFFFFFFFCFC342C003
:1095E00042C042C042C042C06EC3FFFFFFFFFFFF48
:1095F000FFFFFFFFF7D546B162C063C063C063C021
:1096000063C063C063C063C063B86ABA9ADE30C423
:1096100042C042C042C042C042C025B19AE6FFFFEC
:10962000FFFFFFFFFFFFDFFF6DBB83B042C063C0E2
:1096300063C063C063C063C009BAFFFFFFFFFFFFE1
:10964000FFFFFFFFFFFFFFFFFFFFFFFFFFFFFFFF2A
:10965000FFFFFFFFFFFFFFFFFFFFFFFFFFFFFFFF1A
:10966000FFFF75CE20EF60FF60FFE1E463C063C0E1
:1096700063C063C063C063C063C063C063C063C0D2
:1096800063C063C063C063C063C063C063C063C0C2
:1096900063C063C0E3C040FF60FF2BC6FFFFFFFF56
:1096A0000EC660FF60FF40FFA2DBA3C063C063C0C3
:1096B00063C063C063C063C063C063C063C063C092
:1096C00063C063C063C083C002D3E0F660FF60FF85
:1096D000E9C5FFFFFFFFFFFFFFFFFFFFFFFFFFFFEA
:1096E000FFFFFFFFFFFFFFFFFFFFFFFFFFFFFFFF8A
:1096F000FFFFFFFFFFFFFFFFFFFFFFFFFFFFFFFF7A
:10970000FFFFFFFFFFFFFFFFFFFFFFFFFFFFFFFF69
:10971000FFFFFFFFFFFFFFFFFFFFFFFFFFFFFFFF59
:10972000FFFFFFFFFFFFFFFFFFFFFFFFFFFFFFFF49
:10973000FFFFFFFFFFFFFFFFFFFFFFFFFFFFFFFF39
:10974000FFFFFFFFFFFFFFFFFFFFFFFFFFFFFFFF29
:109750009EF718DE72CC2DC38ABA29BA09BA09BAA3
:109760006ABAECBAEFC334CDDBE6DFFFFFFFFFFFE1
:10977000FFFFFFFFFFFFFFFFFFFFFFFFFFFFFFFFF9
:10978000FFFFBAE618DE18DE18DE18DE18DEBAE6CD
:10979000FFFFFFFFFFFFFFFFFFFFFFFF3CEF18DEB4
:1097A00018DE18DE18DE18DE59DEFFFFFFFFFFFFB0
:1097B000FFFFFFFFFFFFFFFFFFFFFFFFFBEE18DED6
:1097C00018DE18DE18DE18DEDBE6FFFFFFFFFFFF06
:1097D000FFFFFFFFFFFF9EF755CD4DC329BAC8B964
:1097E000C7B909BAECBA72CCBAE6DFFFFFFF9EF741
:1097F00018DE18DE18DE18DE18DE18DE5DEFFFFF5B
:10980000FFFFFFFFFFFFFFFFFFFF5CEFD7D5F3CCAC
:1098100072CC72CC92CCB3CC75D5FFFFFFFFFFFFAB
:10982000FFFFFFFFFFFFFFFFFFFFFFFFFFFFFFFF48
:10983000FFFFFFFFFFFFFFFFFFFFFFFFFFFFFFFF38
:10984000FFFFDFFF75CE83DE60FF60FF42D263C0A3
:1098500063C063C063C063C063C063C063C063C0F0
:1098600063C063C063C063C063C063C063C063C0E0
:1098700063C063C0E3C040FF60FF2BC6FFFFFFFF74
:10988000BEF7EBBD40F760FF60FFC0F621E4E2C920
:10989000C3C063C063C063C063C063C063C063C050
:1098A000C3C0E2C901DC80F660FF60FF60FF08C64C
:1098B0009DF7FFFFFFFFFFFFFFFFFFFFFFFFFFFF22
:1098C000FFFFFFFFFFFFFFFFFFFFFFFFFFFFFFFFA8
:1098D000FFFFFFFFFFFFFFFFFFFFFFFFFFFFFFFF98
:1098E000FFFFFFFFFFFFFFFFFFFFFFFFFFFFFFFF88
:1098F000FFFFFFFFFFFFFFFFFFFFFFFFFFFFFFFF78
:10990000FFFFFFFFFFFFFFFFFFFFFFFFFFFFFFFF67
:10991000FFFFFFFFFFFFFFFFFFFFFFFFFFFFFFFF57
:10992000FFFFFFFFFFFFFFFFFFFFFFFFFFFFFFFF47
:10993000FFFFFFFFFFFFFFFFFFFFFFFFFFFFFFFF37
:10994000FFFFFFFFFFFFFFFFFFFFFFFFFFFFFFFF27
:10995000FFFFFFFFFFFFFFFFFFFFFFFFFFFFFFFF17
:10996000FFFFFFFFFFFFFFFFFFFFFFFFFFFFFFFF07
:10997000FFFFFFFFFFFFFFFFFFFFFFFFFFFFFFFFF7
:10998000FFFFFFFFFFFFFFFFFFFFFFFFFFFFFFFFE7
:10999000FFFFFFFFFFFFFFFFFFFFFFFFFFFFFFFFD7
:1099A000FFFFFFFFFFFFFFFFFFFFFFFFFFFFFFFFC7
:1099B000FFFFFFFFFFFFFFFFFFFFFFFFFFFFFFFFB7
:1099C000FFFFFFFFFFFFFFFFFFFFFFFFFFFFFFFFA7
:1099D000FFFFFFFFFFFFFFFFFFFFFFFFFFFFFFFF97
:1099E000FFFFFFFFFFFFFFFFFFFFFFFFFFFFFFFF87
:1099F000FFFFFFFFFFFFFFFFFFFFFFFFFFFFFFFF77
:109A0000FFFFFFFFFFFFFFFFFFFFFFFFFFFFFFFF66
:109A1000FFFFFFFFFFFFFFFFFFFFFFFFFFFFFFFF56
:109A2000FFFFFFFFFFFF76D620F760FFC1E463C0B2
:109A300063C063C063C063C063C063C063C063C00E
:109A400063C063C063C063C063C063C063C063C0FE
:109A500063C063C0E3C040FF60FF2BC6FFFFFFFF92
:109A6000FFFFDFFF31CEA2E660FF60FF60FF60FF17
:109A700000FF20F681ED01EDE1E421ED81ED40F6FE
:109A800000FF60FF60FF60FF60FFE1E60EC69EF72B
:109A9000FFFFFFFFFFFFFFFFFFFFFFFFFFFFFFFFD6
:109AA000FFFFFFFFFFFFFFFFFFFFFFFFFFFFFFFFC6
:109AB000FFFFFFFFFFFFFFFFFFFFFFFFFFFFFFFFB6
:109AC000FFFFFFFFFFFFFFFFFFFFFFFFFFFFFFFFA6
:109AD000FFFFFFFFFFFFFFFFFFFFFFFFFFFFFFFF96
:109AE000FFFFFFFFFFFFFFFFFFFFFFFFFFFFFFFF86
:109AF000FFFFFFFFFFFFFFFFFFFFFFFFFFFFFFFF76
:109B0000FFFFFFFFFFFFFFFFFFFFFFFFFFFFFFFF65
:109B1000FFFFFFFFFFFFFFFFFFFFFFFFFFFFFFFF55
:109B2000FFFFFFFFFFFFFFFFFFFFFFFFFFFFFFFF45
:109B3000FFFFFFFFFFFFFFFFFFFFFFFFFFFFFFFF35
:109B4000FFFFFFFFFFFFFFFFFFFFFFFFFFFFFFFF25
:109B5000FFFFFFFFFFFFFFFFFFFFFFFFFFFFFFFF15
:109B6000FFFFFFFFFFFFFFFFFFFFFFFFFFFFFFFF05
:109B7000FFFFFFFFFFFFFFFFFFFFFFFFFFFFFFFFF5
:109B8000FFFFFFFFFFFFFFFFFFFFFFFFFFFFFFFFE5
:109B9000FFFFFFFFFFFFFFFFFFFFFFFFFFFFFFFFD5
:109BA000FFFFFFFFFFFFFFFFFFFFFFFFFFFFFFFFC5
:109BB000FFFFFFFFFFFFFFFFFFFFFFFFFFFFFFFFB5
:109BC000FFFFFFFFFFFFFFFFFFFFFFFFFFFFFFFFA5
:109BD000FFFFFFFFFFFFFFFFFFFFFFFFFFFFFFFF95
:109BE000FFFFFFFFFFFFFFFFFFFFFFFFFFFFFFFF85
:109BF000FFFFFFFFFFFFFFFFFFFFFFFFFFFFFFFF75
:109C0000FFFFFFFFFFFFDEF743D660FF01F643C013
:109C100063C063C063C063C063C063C063C063C02C
:109C200063C063C063C063C063C063C063C063C01C
:109C300063C063C0E3C040FF60FF2BC6FFFFFFFFB0
:109C4000FFFFFFFFFFFF1BE72DCE62D660FF60FF27
:109C500060FF60FF60FF60FF60FF60FF60FF60FF0C
:109C600060FF60FF60FF62DE2CCEFADEFFFFFFFFC9
:109C7000FFFFFFFFFFFFFFFFFFFFFFFFFFFFFFFFF4
:109C8000FFFFFFFFFFFFFFFFFFFFFFFFFFFFFFFFE4
:109C9000FFFFFFFFFFFFFFFFFFFFFFFFFFFFFFFFD4
:109CA000FFFFFFFFFFFFFFFFFFFFFFFFFFFFFFFFC4
:109CB000FFFFFFFFFFFFFFFFFFFFFFFFFFFFFFFFB4
:109CC000FFFFFFFFFFFFFFFFFFFFFFFFFFFFFFFFA4
:109CD000FFFFFFFFFFFFFFFFFFFFFFFFFFFFFFFF94
:109CE000FFFFFFFFFFFFFFFFFFFFFFFFFFFFFFFF84
:109CF000FFFFFFFFFFFFFFFFFFFFFFFFFFFFFFFF74
:109D0000FFFFFFFFFFFFFFFFFFFFFFFFFFFFFFFF63
:109D1000FFFFFFFFFFFFFFFFFFFFFFFFFFFFFFFF53
:109D2000FFFFFFFFFFFF5DEF75D64FCE4BCE6AD62C
:109D30004AD66BD64CCE70CEF9DEFFFFFFFFFFFF99
:109D4000FFFFFFFFFFFFFFFFFFFFFFFFFFFFFFFF23
:109D5000FFFFFFFFFFFFFFFFFFFFFFFFDFF73CE716
:109D6000D9DE96D693D671CE6ECE4DCE4CCE4BCE9E
:109D70008BDE4AD68BDE4BCE4BCE4DCE4FCE71D640
:109D800074D697D61BE79EF7FFFFFFFFFFFFFFFF8D
:109D9000FFFFFFFFFFFFFFFFFFFFFFFFFFFFFFFFD3
:109DA000FFFFFFFFFFFFFFFFFFFFFFFFFFFFFFFFC3
:109DB000FFFFFFFFFFFFFFFFFFFFFFFFFFFFFFFFB3
:109DC000FFFF5CEFB7D673D64FCE4CCE4BCE8BD6C3
:109DD0006AD64BD64CCE6FCE74D6D8DE7DEFFFFF61
:109DE000FFFFFFFFFFFFDFFF45D660FF40F643C0E8
:109DF00063C063C063C063C063C063C063C063C04B
:109E000063C063C063C063C063C063C063C063C03A
:109E100063C063C0E3C040FF60FF2BCEFFFFFFFFC6
:109E2000FFFFFFFFFFFFFFFFFFFF9EF776CE4ECE47
:109E300068D665D682DEA1E6E1EEA2E683DE65D6CF
:109E400049D64ECE76CE9EF7FFFFFFFFFFFFFFFF06
:109E5000FFFFFFFFFFFFFFFFFFFFFFFFFFFFFFFF12
:109E6000FFFFFFFFFFFFFFFFFFFFFFFFFFFFFFFF02
:109E7000FFFFFFFFFFFFFFFF7EEF1BE797D674D6C4
:109E800092D66FCE4DCE4CCE4BCE6BD68BDE6AD6F5
:109E90006BD64BCE4CCE4CCE4DCE6FCE92D674D62A
:109EA00097D6FADE5DEFDFFFFFFFFFFFFFFFFFFF4B
:109EB000FFFFFFFFFFFFFFFFFFFFFFFFFFFFFFFFB2
:109EC000FFFFFFFFFFFFFFFF98D607C627C627C685
:109ED00027C627C627C627C627C627C627C627C61A
:109EE00027C627C627C627C627C627C627C627C60A
:109EF00027C627C627C627C627C627C627CE6AB5C0
:109F0000FFFFD9DE2BCEA1DE60FF60FF60FF60FFA8
:109F100060FF60FF60FF80FF32CEFFFFFFFFFFFFAB
:109F2000FFFFFFFFFFFFFFFFFFFFFFFFFFFFFFFF41
:109F3000FFFF9DF7D9DE72CE4DCE27CE63D6C1E6A8
:109F400020F760F760FF60FF60FF60FF60FF60FF69
:109F500060FF60FF60FF60FF60FF60FF60FF60FF09
:109F600060FF40F7E0EE82DE27CE4DCE74D63BE7B1
:109F7000FFFFFFFFFFFFFFFFFFFFFFFFFFFFFFFFF1
:109F8000FFFFFFFFFFFFFFFFFFFFFFFFFFFFFFFFE1
:109F9000FFFFFFFFFFFFFFFFFFFFDFFFD8DE4ECE1B
:109FA00045CEC1E640F760FF60FF60FF60FF60FFE5
:109FB00060FF60FF60FF60FF60FF20F782DE27CE5A
:109FC00050CED9DEDFFFFFFF25CE60FF40F643C055
:109FD00063C063C063C063C063C063C063C063C069
:109FE00063C063C063C063C063C063C063C063C059
:109FF00063C063C0E3C040FF60FFEABDA8BD27C6E1
:10A0000027C627C627C627C627C627C627C627CEE0
:10A0100027CE28CEE7C5A5BDC5BDC6BDE7C528CEA0
:10A0200027CE27C627C627C627C627C627C627C6C0
:10A0300027C607CED8DEFFFFFFFFFFFFFFFFFFFFB2
:10A04000FFFFFFFFFFFFFFFFFFFFFFFFFFFF9EF789
:10A05000B8DE51CE4ACE25CE81DEE0EE40F760FF7D
:10A0600060FF60FF60FF60FF60FF60FF60FF60FFF8
:10A0700060FF60FF60FF60FF60FF60FF60FF60FFE8
:10A0800040FF00F7A1E664D648CE4ECE95D63BE71A
:10A09000DFFFFFFFFFFFFFFFFFFFFFFFFFFFFFFFF0
:10A0A000FFFFFFFFFFFFFFFF76CE40F760FF60FF7F
:10A0B00060FF60FF60FF60FF60FF60FF60FF60FFA8
:10A0C00060FF60FF60FF60FF60FF60FF60FF60FF98
:10A0D00060FF60FF60FF60FF60FF60FF60FF03C61E
:10A0E00030C6C1E660FF60FF60FF60FF40FF40FFD9
:10A0F00040FF40FF60FF80FF31CEFFFFFFFFFFFF0B
:10A10000FFFFFFFFFFFFFFFFFFFFDEFFFADE51CE85
:10A1100028CE83DE00EF60FF60FF60FF60FF60FF1E
:10A1200060FF60FF60FF60FF60FF60FF40FF40FF77
:10A1300040FF40FF40FF40FF40FF60FF60FF60FFC7
:10A1400060FF60FF60FF60FF60FF60FF40FFC1E6EF
:10A1500047CE52CE5CEFFFFFFFFFFFFFFFFFFFFF89
:10A16000FFFFFFFFFFFFFFFFFFFFFFFFFFFFFFFFFF
:10A17000FFFFFFFFFFFFDFFF75D626CE00EF60FF7A
:10A1800060FF60FF60FF60FF60FF40FF40FF40FF37
:10A1900040FF40FF40FF60FF60FF60FF60FF60FF27
:10A1A00060FF00EF46CE52CE04C660FF40F643C0CB
:10A1B00063C063C063C063C063C063C063C063C087
:10A1C00063C063C063C063C063C063C063C063C077
:10A1D00063C063C0E3C040FF60FFA9BDA2DE60FFB3
:10A1E00060FF60FF60FF60FF60FF60FF60FF60FF77
:10A1F00060FF60FF60FF60FF60FF60FF60FF60FF67
:10A2000060FF60FF60FF60FF60FF60FF60FF60FF56
:10A2100060FF60FFB6DEFFFFFFFFFFFFFFFFFFFFF6
:10A22000FFFFFFFFFFFFFFFFBEF775D62BCE63DEFC
:10A2300020F760FF60FF60FF60FF60FF60FF60FF6E
:10A2400060FF60FF60FF40FF40FF40FF40FF40FFB6
:10A2500040FF40FF40FF40FF60FF60FF60FF60FF86
:10A2600060FF60FF60FF60FF60FF60FF40FFC1E6CE
:10A2700046CE51CE3BE7FFFFFFFFFFFFFFFFFFFF93
:10A28000FFFFFFFFFFFFFFFF76CE60F760FF40FF9D
:10A2900020FF20FF20FF20FF20FF20FF20FF20FFC6
:10A2A00020FF20FF20FF20FF20FF20FF20FF20FFB6
:10A2B00020FF20FF20FF20FF20FF60FF60FFE0EE77
:10A2C00060F760FF60FF60F6A1DBC2C9E2C0C3C0F7
:10A2D000C3C062CA60FF80FF31CEFFFFFFFFFFFFF8
:10A2E000FFFFFFFFFFFFFADE2FCE45D600EF80FF16
:10A2F00060FF60FF60FF60FF80FF00FF20F601E568
:10A3000021DC22DBA2D202CA62C923C9E3C0C3C0D6
:10A31000C3C0C3C0C3C0C3C0E3C023C983C922CA6A
:10A32000C2D2A1DBA1E4E1F500FF80FF60FF60FF86
:10A3300060FF60FF82DE2DCE3CE7FFFFFFFFFFFFE7
:10A34000FFFFFFFFFFFFFFFFFFFFFFFFFFFFFFFF1D
:10A35000FFFFFFFF1BE728C640F760FF60FF60FFBD
:10A3600000FF61EDC1DBA2D2A2C922C1E3C0C3C01C
:10A37000C3C0C3C022C1C2C9C2D201E4C0ED40FF04
:10A3800060FF60FF60FF60FF20F760FF40F643C0A2
:10A3900063C063C063C063C063C063C063C063C0A5
:10A3A00063C063C063C063C063C063C063C063C095
:10A3B00063C063C0E3C040FF60FFC9BDA2E660FFA9
:10A3C00040FF20FF20FF20FF20FF20FF20FF20FF75
:10A3D00020FF20FF20FF20FF20FF20FF20FF20FF85
:10A3E00020FF20FF20FF20FF20FF20FF20FF20FF75
:10A3F00060FF60FFB6DEFFFFFFFFFFFFFFFFFFFF15
:10A40000FFFFFFFF9EF731CE64D640F760FF60FF8D
:10A4100060FF60FF60FFC0F681ED61E482DBE2D2A5
:10A4200022D2A2C943C903C1E3C0C3C0C3C0C3C0D1
:10A43000C3C0E3C0E3C003C942C9A2C922D2C2D289
:10A4400041DB41E421ED40F640FF80FF60FF60FF0B
:10A4500060FF60FFC1E62BCEFADEFFFFFFFFFFFFCC
:10A46000FFFFFFFFFFFFFFFF76CE60F760FF02DB1D
:10A4700063C063C063C063C063C063C063C063C0C4
:10A4800063C063C063C063C063C063C063C063C0B4
:10A4900063C063C063C063C043C000F660FF60FF79
:10A4A00060FF00FF42DB63C063C063C063C063C082
:10A4B00063C002CA60FF80FF31CEFFFFFFFFFFFFD6
:10A4C000BEF775D627CEE0EE60FF60FF60FF60FF4D
:10A4D00040FF00F661E4C2D243C963C043C063C019
:10A4E00063C063C063C063C063C063C063C063C054
:10A4F00063C063C063C063C063C063C063C063C044
:10A5000063C063C063C043C063C082C981DBA1ED87
:10A5100040FF60FF60FF60FFA1DE30CEBEF7FFFFAF
:10A52000FFFFFFFFFFFFFFFFFFFFFFFFFFFFFFFF3B
:10A53000FFFF97D682DE60FF60FF60FF41ED62D2D1
:10A5400083C063C063C063C063C063C063C063C0D3
:10A5500063C063C063C063C063C063C043C0A3C0C3
:10A56000A2D241ED40FF60FF60FF60FF40F643C0B4
:10A5700063C063C063C063C063C063C063C063C0C3
:10A5800063C063C063C063C063C063C063C063C0B3
:10A5900063C063C0E3C040FF60FFC9BDA2E660FFC7
:10A5A00021ED63C063C063C063C063C063C063C0A8
:10A5B00063C063C063C063C063C063C063C063C083
:10A5C00063C063C063C063C063C063C063C0E2D2E2
:10A5D00060FF60FFB6DEFFFFFFFFFFFFFFFFFFFF33
:10A5E000FFFF75D644D660FF60FF60FF60FF60F636
:10A5F00061E462D202C143C063C063C063C063C090
:10A6000063C063C063C063C063C063C063C063C032
:10A6100063C063C063C063C063C063C063C063C022
:10A6200063C063C063C043C083C0A2C982DB61ED65
:10A6300020FF60FF60FF60FFC0E60FC6BEF7FFFFB0
:10A64000FFFFFFFFFFFFFFFF76CE60F760FF02DB3B
:10A6500063C063C063C063C063C063C063C063C0E2
:10A6600063C063C063C063C063C063C063C063C0D2
:10A6700063C063C063C063C043C020F660FF60FF77
:10A68000E0F6C2C963C063C063C063C063C063C097
:10A6900063C002CA80FF80FF31CEFFFFBEF773CEDA
:10A6A00044D640F760FF60FF60FF00FF01EDC2D2BB
:10A6B000E3C063C063C063C063C063C063C063C002
:10A6C00063C063C063C063C063C063C063C063C072
:10A6D00063C063C063C063C063C063C063C063C062
:10A6E00063C063C063C063C063C063C063C063C052
:10A6F00002C1C2DBA0F660FF60FF40FF27CE3BE750
:10A70000FFFFFFFFFFFFFFFFFFFFFFFFFFFFFFFF59
:10A7100097D6C1E660FF60FF01EEC2C963C063C0A7
:10A7200063C063C063C063C063C063C063C063C011
:10A7300063C063C063C063C063C063C063C063C001
:10A7400063C063C023C941E420FF60FF40F643C0FB
:10A7500063C063C063C063C063C063C063C063C0E1
:10A7600063C063C063C063C063C063C063C063C0D1
:10A7700063C063C0E3C040FF60FFC9BDA2E660FFE5
:10A7800021ED63C063C063C063C063C063C063C0C6
:10A7900063C063C063C063C063C063C063C063C0A1
:10A7A00063C063C063C063C063C063C063C0E2DAF8
:10A7B00060FF60FFB6DEFFFFFFFFFFFFFFFFBEF79A
:10A7C000EDC520EF60FF60FF20FFA1E4C2C963C0B8
:10A7D00063C063C063C063C063C063C063C063C061
:10A7E00063C063C063C063C063C063C063C063C051
:10A7F00063C063C063C063C063C063C063C063C041
:10A8000063C063C063C063C063C063C063C063C030
:10A81000E3C042DB40F660FF60FF60FF07C63CE735
:10A82000FFFFFFFFFFFFFFFF76CE60F760FF02DB59
:10A8300063C063C063C063C063C063C063C063C000
:10A8400063C063C063C063C063C063C063C063C0F0
:10A8500063C063C063C063C043C001ED40FF20FF1D
:10A86000E2C963C063C063C063C063C063C063C048
:10A8700063C002CA80FF80FF32CE96D626D640F74C
:10A8800060FF60FF60FFA1EDE2D2C3C063C063C0A0
:10A8900063C063C063C063C063C063C063C063C0A0
:10A8A00063C063C063C063C063C063C063C063C090
:10A8B00063C063C063C063C063C063C063C063C080
:10A8C00063C063C063C063C063C063C063C063C070
:10A8D00063C063C0A3C0A1DB00FF60FF60FF64D65C
:10A8E000FADEFFFFFFFFFFFFFFFFFFFFFFFF1AE79B
:10A8F00082DE60FF60FFA1E483C063C063C063C009
:10A9000063C063C063C063C063C063C063C063C02F
:10A9100063C063C063C063C063C063C063C063C01F
:10A9200063C063C063C063C043C901ED20F643C088
:10A9300063C063C063C063C063C063C063C063C0FF
:10A9400063C063C063C063C063C063C063C063C0EF
:10A9500063C063C0E3C040FF60FFC9BDA2E660FF03
:10A9600021ED63C063C063C063C063C063C063C0E4
:10A9700063C063C063C063C063C063C063C063C0BF
:10A9800063C063C063C063C063C063C063C0E2DA16
:10A9900060FF60FFB6DEFFFFFFFFFFFFBEF70AC6E6
:10A9A00040FF60FF60FFC1E422C163C063C063C0B9
:10A9B00063C063C063C063C063C063C063C063C07F
:10A9C00063C063C063C063C063C063C063C063C06F
:10A9D00063C063C063C063C063C063C063C063C05F
:10A9E00063C063C063C063C063C063C063C063C04F
:10A9F00063C063C0A3C042DBE0FE60FF60FF45CEE2
:10AA00005CEFFFFFFFFFFFFF76CE60F760FF02DB2A
:10AA100063C063C063C063C063C063C063C063C01E
:10AA200063C063C063C063C063C063C063C063C00E
:10AA300063C063C063C063C063C063C022C1E2C9B6
:10AA400063C063C063C063C063C063C063C063C0EE
:10AA500063C002CA60FF80FF31CE25CE60FF60FF79
:10AA600060FFE1E4A2C943C063C063C063C063C0C8
:10AA700063C063C063C063C063C063C063C063C0BE
:10AA800063C063C063C063C063C063C063C063C0AE
:10AA900063C063C063C063C063C063C063C063C09E
:10AAA00063C063C063C063C063C063C063C063C08E
:10AAB00063C063C063C063C063C921F660FF60FF09
:10AAC00044CE5CEFFFFFFFFFFFFFFFFFDFFF08C685
:10AAD00060FF60FFA1E463C063C063C063C063C084
:10AAE00063C063C063C063C063C063C063C063C04E
:10AAF00063C063C063C063C063C063C063C063C03E
:10AB000063C063C063C063C063C063C082C963C005
:10AB100063C063C063C063C063C063C063C063C01D
:10AB200063C063C063C063C063C063C063C063C00D
:10AB300063C063C0E3C040FF60FFC9BDA2E660FF21
:10AB400021ED63C063C063C063C063C063C063C002
:10AB500063C063C063C063C063C063C063C063C0DD
:10AB600063C063C063C063C063C063C063C0E2DA34
:10AB700060FF60FFB6DEFFFFFFFFFFFFEDC560FF78
:10AB800060FF00FF82D263C063C063C063C063C064
:10AB900063C063C063C063C063C063C063C063C09D
:10ABA00063C063C063C063C063C063C063C063C08D
:10ABB00063C063C063C063C063C063C063C063C07D
:10ABC00063C063C063C063C063C063C063C063C06D
:10ABD00063C063C063C063C043C941F660FF60FFE8
:10ABE00007C6DEF7FFFFFFFF76CE60F760FF02DBF0
:10ABF00063C063C063C063C063C063C063C063C03D
:10AC000063C063C063C063C063C063C063C063C02C
:10AC100063C063C063C063C063C063C063C063C01C
:10AC200063C063C063C063C063C063C063C063C00C
:10AC300063C002CA60FF80FF31CE25CE60FFE0F620
:10AC400063C963C063C063C063C063C063C063C0E3
:10AC500063C063C063C063C063C063C063C063C0DC
:10AC600063C063C063C063C063C063C063C063C0CC
:10AC700063C063C063C063C063C063C063C063C0BC
:10AC800063C063C063C063C063C063C063C063C0AC
:10AC900063C063C063C063C063C0A3C081ED60FFD5
:10ACA00060FF09C6DFFFFFFFFFFFFFFF75D640F71C
:10ACB00060FF01EE83C063C063C063C063C063C054
:10ACC00063C063C063C063C063C063C063C063C06C
:10ACD00063C063C063C063C063C063C063C063C05C
:10ACE00063C063C063C063C063C063C063C063C04C
:10ACF00063C063C063C063C063C063C063C063C03C
:10AD000063C063C063C063C063C063C063C063C02B
:10AD100063C063C0E3C040FF60FFC9BDA2E660FF3F
:10AD200021ED63C063C063C063C063C063C063C020
:10AD300063C063C063C063C063C063C063C063C0FB
:10AD400063C063C063C063C063C063C063C0E2DA52
:10AD500060FF60FFB6DEFFFFFFFF54CE20F760FF0D
:10AD6000E0F6A2C963C063C063C063C063C063C0D0
:10AD700063C063C063C063C063C063C063C063C0BB
:10AD800063C063C063C063C063C063C063C063C0AB
:10AD900063C063C063C063C063C063C063C063C09B
:10ADA00063C063C063C063C063C063C063C063C08B
:10ADB00063C063C063C063C063C0E3C041F660FFAB
:10ADC00060FF30C6FFFFFFFF76CE60F760FF02DB5B
:10ADD00063C063C063C063C063C063C063C063C05B
:10ADE00063C063C063C063C063C063C063C063C04B
:10ADF00063C063C063C063C063C063C063C063C03B
:10AE000063C063C063C063C063C063C063C063C02A
:10AE100063C002CA60FF80FF31CE24CE60FF80F69F
:10AE200043C063C063C063C063C063C063C063C02A
:10AE300063C063C063C063C063C063C063C063C0FA
:10AE400063C063C063C063C063C063C063C063C0EA
:10AE500063C063C063C063C063C063C063C063C0DA
:10AE600063C063C063C063C063C063C063C063C0CA
:10AE700063C063C063C063C063C063C0C3C041F646
:10AE800060FF40F754CEFFFFFFFFDFFF27CE60FFDC
:10AE900060FFE2C963C063C063C063C063C063C0D6
:10AEA00063C063C063C063C063C063C063C063C08A
:10AEB00063C063C063C063C063C063C063C063C07A
:10AEC00063C063C063C063C063C063C063C063C06A
:10AED00063C063C063C063C063C063C063C063C05A
:10AEE00063C063C063C063C063C063C063C063C04A
:10AEF00063C063C0E3C040FF60FFC9BDA2E660FF5E
:10AF000021ED63C063C063C063C063C063C063C03E
:10AF100063C063C063C063C063C063C063C063C019
:10AF200063C063C063C063C063C063C063C0E2DA70
:10AF300060FF60FFB6DEFFFF9EF744CE60FF40FF7C
:10AF400062D263C063C063C063C063C063C063C0D8
:10AF500063C063C063C063C063C063C063C063C0D9
:10AF600063C063C063C063C063C063C063C063C0C9
:10AF700063C063C063C063C063C063C063C063C0B9
:10AF800063C063C063C063C063C063C063C063C0A9
:10AF900063C063C063C063C063C063C063C900FFB4
:10AFA00060FF82DE3CEFFFFF76CE60F760FF02DBE2
:10AFB00063C063C063C063C063C063C063C063C079
:10AFC00063C063C063C063C063C063C063C063C069
:10AFD00063C063C063C063C063C063C063C063C059
:10AFE00063C063C063C063C063C063C063C063C049
:10AFF00063C002CA60FF80FF31CE24CE60FFA0F69E
:10B0000043C063C063C063C063C063C063C063C048
:10B0100063C063C063C063C063C063C063C063C018
:10B0200063C063C063C063C063C063C063C063C008
:10B0300063C063C063C063C063C063C063C063C0F8
:10B0400063C063C063C063C063C063C063C063C0E8
:10B0500063C063C063C063C063C063C063C0C2C970
:10B0600060FF60FF45CEBEF7FFFFFADEE1EE60FF56
:10B0700081ED63C063C063C063C063C063C063C06D
:10B0800063C063C063C063C063C063C063C063C0A8
:10B0900063C063C063C063C063C063C063C063C098
:10B0A00063C063C063C063C063C063C063C063C088
:10B0B00063C063C063C063C063C063C063C063C078
:10B0C00063C063C063C063C063C063C063C063C068
:10B0D00063C063C0E3C040FF60FFC9BDA2E660FF7C
:10B0E00021ED63C063C063C063C063C063C063C05D
:10B0F00063C063C063C063C063C063C063C063C038
:10B1000063C063C063C063C063C063C063C0E2DA8E
:10B1100060FF60FFB6DEFFFF53CE60FF60FFC1E45B
:10B1200063C063C063C063C063C063C063C063C007
:10B1300063C063C063C063C063C063C063C063C0F7
:10B1400063C063C063C063C063C063C063C063C0E7
:10B1500063C063C063C063C063C063C063C063C0D7
:10B1600063C063C063C063C063C063C063C063C0C7
:10B1700063C063C063C063C063C063C063C0C2DB3D
:10B1800060FF60FF30CEFFFF76CE60F760FF02D336
:10B1900063C063C063C063C063C063C063C063C097
:10B1A00063C063C063C063C063C063C063C063C087
:10B1B00063C063C063C063C063C063C063C063C077
:10B1C00063C063C063C063C063C063C063C063C067
:10B1D00063C002CA60FF80FF31CE24CE60FF80F6DC
:10B1E00043C063C063C063C063C063C063C063C067
:10B1F00063C063C063C063C063C063C063C063C037
:10B2000063C063C063C063C063C063C0C3C082C99E
:10B21000A2C902C163C063C063C063C063C063C02E
:10B2200063C063C063C063C063C063C063C063C006
:10B2300063C063C063C063C063C063C063C063C0F6
:10B24000E1E460FF40F796D6FFFF51CE60FF60FF5C
:10B25000E2D263C063C063C063C063C063C063C045
:10B2600063C063C063C063C063C063C063C063C0C6
:10B2700063C063C063C063C063C063C063C063C0B6
:10B2800063C063C063C063C063C063C063C063C0A6
:10B2900063C063C063C063C063C063C063C063C096
:10B2A00063C063C063C063C063C063C063C063C086
:10B2B00063C063C0E3C040FF60FFC9BDA2E660FF9A
:10B2C00021ED63C063C063C063C063C063C063C07B
:10B2D00063C063C063C063C063C063C063C063C056
:10B2E00063C063C063C063C063C063C063C0E2DAAD
:10B2F00060FF60FFB6DEFFFF27CE60FF40FF62C940
:10B3000063C063C063C063C063C063C063C063C025
:10B3100063C063C063C063C063C063C063C063C015
:10B3200063C063C063C063C063C063C063C0A3C0C5
:10B3300063C043C063C063C063C063C063C063C015
:10B3400063C063C063C063C063C063C063C063C0E5
:10B3500063C063C063C063C063C063C063C0E2C056
:10B3600000FF60FF45CEDFFF76CE60F760FF02D3BF
:10B3700063C063C063C063C063C063C063C063C0B5
:10B3800063C063C063C063C063C063C063C063C0A5
:10B3900063C063C063C063C063C063C063C063C095
:10B3A00063C063C063C063C063C063C063C063C085
:10B3B00063C002CA60FF80FF31CE24CE60FF80F6FA
:10B3C00043C063C063C063C063C063C063C063C085
:10B3D00063C063C063C063C063C063C063C063C055
:10B3E00063C063C063C063C0A2C981ED60FF80FF1A
:10B3F00080FF60FFA1EDA2C963C063C063C063C0EA
:10B4000063C063C063C063C063C063C063C063C024
:10B4100063C063C063C063C063C063C063C063C014
:10B42000E2C960FF60FF2CCEFFFF29CE60FF60FF06
:10B43000E2C063C063C063C063C063C063C063C075
:10B4400063C063C063C063C063C063C063C063C0E4
:10B4500063C063C063C063C063C063C063C063C0D4
:10B4600063C063C063C063C063C063C063C063C0C4
:10B4700063C063C063C063C063C063C063C063C0B4
:10B4800063C063C063C063C063C063C063C063C0A4
:10B4900063C063C0E3C040FF60FFC9BDA2E660FFB8
:10B4A00041ED63C063C063C063C063C063C063C079
:10B4B00063C063C063C063C063C063C063C063C074
:10B4C00063C063C063C063C063C063C063C0E2DACB
:10B4D00060FF60FFB5DE3CEFC0E660FF81ED63C05A
:10B4E00063C063C063C063C063C063C063C063C044
:10B4F00063C063C063C063C063C063C063C063C034
:10B5000063C063C063C063C002CA61ED20FF60FF17
:10B5100020FFE1EDE2D263C063C063C063C063C0DB
:10B5200063C063C063C063C063C063C063C063C003
:10B5300063C063C063C063C063C063C063C063C0F3
:10B54000E1E460FF00EFFADE76CE40F760FF00F640
:10B5500022C163C063C063C063C063C063C063C013
:10B5600063C063C063C063C063C063C063C063C0C3
:10B5700063C063C063C063C063C063C063C063C0B3
:10B5800063C063C063C063C063C063C063C063C0A3
:10B5900063C002CA60FF80FF31CE24CE60FF80F618
:10B5A00043C063C063C063C063C063C063C063C0A3
:10B5B00063C063C063C063C063C063C063C063C073
:10B5C00063C063C063C0C2C920FF60FF60FF60FF4B
:10B5D00060FF60FF60FF00FF63C963C063C063C0BA
:10B5E00063C063C063C063C063C063C063C063C043
:10B5F00063C063C063C063C063C063C063C063C033
:10B6000063C0A0F660FF44CEDFFF44D660FF80F643
:10B6100043C063C063C063C063C063C063C063C032
:10B6200063C063C063C063C063C063C063C063C002
:10B6300063C063C063C063C063C063C063C063C0F2
:10B6400083C083C083C063C063C063C063C063C082
:10B6500063C063C063C063C063C063C063C063C0D2
:10B6600063C063C063C063C063C063C063C063C0C2
:10B6700063C063C0E3C040FF60FFC9BDA2DE60FFDE
:10B6800040FFE1DB83C063C063C063C063C063C0CD
:10B6900063C063C063C063C063C063C063C063C092
:10B6A00063C063C063C063C063C063C063C0E2DAE9
:10B6B00060FF60FFB6DE75D660FF60FF62DB63C0CF
:10B6C00063C063C063C063C063C063C063C063C062
:10B6D00063C063C063C063C063C063C063C063C052
:10B6E00063C063C063C022DB60FF60FF60FF60FF78
:10B6F00060FF60FF60FFA1E463C063C063C063C01C
:10B7000063C063C063C063C063C063C063C063C021
:10B7100063C063C063C063C063C063C063C063C011
:10B72000E2D260FF60FF73CEB8D6C1DE60FF60FF7B
:10B7300061F6E3C063C063C063C063C063C063C03D
:10B7400063C063C063C063C063C063C063C063C0E1
:10B7500063C063C063C063C063C063C063C063C0D1
:10B7600063C063C063C063C063C063C063C063C0C1
:10B7700063C002CA60FF80FF31CE24CE60FF80F636
:10B7800043C063C063C063C063C063C063C063C0C1
:10B7900063C063C063C063C063C063C063C063C091
:10B7A00063C063C083C000F660FF40F727CE4FCE72
:10B7B00070CE27CE40FF60FF41ED63C063C063C021
:10B7C00063C063C063C063C063C063C063C063C061
:10B7D00063C063C063C063C063C063C063C063C051
:10B7E00043C001ED60FFC1E6BBD681DE60FF41EDE5
:10B7F00043C063C063C063C063C063C063C063C051
:10B8000063C063C063C063C063C063C063C063C020
:10B8100063C063C063C063C063C0A3C042DBC1ED4B
:10B82000C0F6E0FEA0F6E1ED21E4C2C963C063C04A
:10B8300063C063C063C063C063C063C063C063C0F0
:10B8400063C063C063C063C063C063C063C063C0E0
:10B8500063C063C0E3C040FF60FFEABDE6C540F7D8
:10B8600060FF60FF82DB63C063C063C063C063C00E
:10B8700063C063C063C063C063C063C063C063C0B0
:10B8800063C063C063C063C063C063C063C0E2DA07
:10B8900060FF60FFB6DE50D660FF80FFE2C963C084
:10B8A00063C063C063C063C063C063C063C063C080
:10B8B00063C063C063C063C063C063C063C063C070
:10B8C00063C063C062C920FF60FF20F726CE6BD63D
:10B8D00027CEE1EE60FF60FFC2D263C063C063C0E9
:10B8E00063C063C063C063C063C063C063C063C040
:10B8F00063C063C063C063C063C063C063C063C030
:10B9000042C980FF60FF4DCEFFFFFADE07CE60FF29
:10B9100060FF81E463C063C063C063C063C063C091
:10B9200063C063C063C063C063C063C063C063C0FF
:10B9300063C063C063C063C063C063C063C063C0EF
:10B9400063C063C063C063C063C063C063C063C0DF
:10B9500063C002CA60FF80FF31CE24CE60FF80F654
:10B9600043C063C063C063C063C063C063C063C0DF
:10B9700063C063C063C063C063C063C063C063C0AF
:10B9800063C063C082C960FF60FF29CEBFFFFFFFB5
:10B99000FFFF9EF726CE60FF40FFE3C063C063C099
:10B9A00063C063C063C063C063C063C063C063C07F
:10B9B00063C063C063C063C063C063C063C063C06F
:10B9C00063C001DC60FF20F716C6E1EE60FF81E492
:10B9D00063C063C063C063C063C063C063C063C04F
:10B9E00063C063C063C063C063C063C063C063C03F
:10B9F00063C063C063C063C083C0A1ED60FF60FF2C
:10BA000060FF60FF60FF60FF60FF60FFC1E463C034
:10BA100063C063C063C063C063C063C063C063C00E
:10BA200063C063C063C063C063C063C063C063C0FE
:10BA300063C063C0E3C040FF60FF2BCEBEF753CEB0
:10BA4000C1E660FF00FFC3C063C063C063C063C0E2
:10BA500063C063C063C063C063C063C063C063C0CE
:10BA600063C063C063C063C063C063C063C0E2DA25
:10BA700060FF60FFB6DE4BCE60FF40FFE3C063C0F7
:10BA800063C063C063C063C063C063C063C063C09E
:10BA900063C063C063C063C063C063C063C063C08E
:10BAA00063C063C041E460FF60FF10C6DFFFFFFFBB
:10BAB000FFFF77D6E1EE60FFC1ED63C063C063C0F6
:10BAC00063C063C063C063C063C063C063C063C05E
:10BAD00063C063C063C063C063C063C063C063C04E
:10BAE00083C040FF60FF28CEFFFFFFFFD9DEA2E644
:10BAF00060FF80F683C063C063C063C063C063C07F
:10BB000063C063C063C063C063C063C063C063C01D
:10BB100063C063C063C063C063C063C063C063C00D
:10BB200063C063C063C063C063C063C063C063C0FD
:10BB300063C002CA60FF80FF31CE24CE60FF80F672
:10BB400043C063C063C063C063C063C063C063C0FD
:10BB500063C063C063C063C063C063C063C063C0CD
:10BB600063C063C0A2D260FF80FF52CEFFFFFFFF21
:10BB7000FFFFFFFF4ECE60FF80FFC2C963C063C0FE
:10BB800063C063C063C063C063C063C063C063C09D
:10BB900063C063C063C063C063C063C063C063C08D
:10BBA00063C081DB60FF40FFF3BD20F760FF21E44D
:10BBB00063C063C063C063C063C063C063C063C06D
:10BBC00063C063C063C063C063C063C063C063C05D
:10BBD00063C063C063C063C002DB60FF60FF40F707
:10BBE00081DE41D681DE20F760FF60FF40F643C072
:10BBF00063C063C063C063C063C063C063C063C02D
:10BC000063C063C063C063C063C063C063C063C01C
:10BC100063C063C0E3C040FF60FF2BCEFFFFFFFFA8
:10BC20000BC660FF60FF22D263C063C063C063C005
:10BC300063C063C063C063C063C063C063C063C0EC
:10BC400063C063C063C063C063C063C063C0E2DA43
:10BC500060FF60FFB6DE29CE60FF00FFA3C063C0B7
:10BC600063C063C063C063C063C063C063C063C0BC
:10BC700063C063C063C063C063C063C063C063C0AC
:10BC800063C063C0A1ED60FF81DE5DEFFFFFFFFFDA
:10BC9000FFFFDFFF26CE60FF00FF63C063C063C00D
:10BCA00063C063C063C063C063C063C063C063C07C
:10BCB00063C063C063C063C063C063C063C063C06C
:10BCC00043C0E0F660FFE6C5FFFFFFFFFFFF4BCE7E
:10BCD00060FF60FF62C963C063C063C063C063C0CC
:10BCE00063C063C063C063C063C063C063C063C03C
:10BCF00063C063C063C063C063C063C063C063C02C
:10BD000063C063C063C063C063C083C003C9C2C9EA
:10BD100042D2C2DB60FF80FF31CE24CE60FF80F6CE
:10BD200043C063C063C063C063C063C063C063C01B
:10BD300063C063C063C063C063C063C063C063C0EB
:10BD400063C063C081DB60FF40FFD8DEFFFFFFFF01
:10BD5000FFFFFFFF74D680FF60FFC2D263C063C0E5
:10BD600063C063C063C063C063C063C063C063C0BB
:10BD700063C063C063C063C063C063C063C063C0AB
:10BD800063C062DB60FF60FF91B520F760FF02E4F3
:10BD900063C063C063C063C063C063C063C063C08B
:10BDA00063C063C063C063C063C063C063C063C07B
:10BDB00063C063C063C063C060F660FFE1E654CE59
:10BDC0007DEFDEFF7DEFB8D643CE60FF40F643C087
:10BDD00063C063C063C063C063C063C063C063C04B
:10BDE00063C063C063C063C063C063C063C063C03B
:10BDF00063C063C0E3C040FF60FF2BC6FFFFFFFFCF
:10BE000096D660FF60FF82DB63C063C063C063C01F
:10BE100063C063C063C063C063C063C063C063C00A
:10BE200063C063C063C063C063C063C063C0E2DA61
:10BE300060FF60FFB6DE68D660FFE0FEA3C063C0AF
:10BE400063C063C063C063C063C063C063C063C0DA
:10BE500063C063C063C063C063C063C063C063C0CA
:10BE600063C063C080F660FF25CEFFFFFFFFFFFFCA
:10BE7000FFFFFFFF4BCE60FF60FFC3C063C063C026
:10BE800063C063C063C063C063C063C063C063C09A
:10BE900063C063C063C063C063C063C063C063C08A
:10BEA00043C080F660FF04CEFFFFFFFFFFFF71D6A7
:10BEB00080FF80FF02CA63C063C063C063C063C009
:10BEC00063C063C063C063C063C063C063C063C05A
:10BED00063C063C063C063C063C063C063C063C04A
:10BEE00063C063C083C082D201E5A0F640FF60FF5B
:10BEF00080FF60FF60FF80FF31CE24CE60FFA0F6A0
:10BF0000E3C003C903C903C903C903C903C903C9FA
:10BF100003C903C903C903C903C903C903C903C9C1
:10BF200003C103C101DC60FF20F7D9DEFFFFFFFF83
:10BF3000FFFF9DF7F1C560FF60FF22DB63C063C0B8
:10BF400063C063C063C063C063C063C063C063C0D9
:10BF500063C063C063C063C063C063C063C063C0C9
:10BF600063C062DB60FF60FF70AD20F760FFC1DB84
:10BF700063C063C063C063C063C063C063C063C0A9
:10BF800063C063C063C063C063C063C063C063C099
:10BF900063C063C063C022C160FF60FF2ACEFFFFA1
:10BFA000FFFFFFFFFFFFFFFF25CE60FF40F643C00E
:10BFB00063C063C063C063C063C063C063C063C069
:10BFC00063C063C063C063C063C063C063C063C059
:10BFD00063C063C0E3C040FF60FF2BC6FFFFFFFFED
:10BFE000FADE20F760FF21E463C063C063C063C072
:10BFF00063C063C063C063C063C063C063C063C029
:10C0000063C063C063C063C063C063C063C0E2DA7F
:10C0100060FF60FFB6DE47CE60FFE0FE83C063C016
:10C0200063C063C063C063C063C063C063C063C0F8
:10C0300063C063C063C063C063C063C063C063C0E8
:10C0400063C063C0A0F660FF46D6FFFFFFFFFFFF9F
:10C05000FFFFFFFF4CCE60FF80FFE3C063C063C003
:10C0600063C063C063C063C063C063C063C063C0B8
:10C0700063C063C063C063C063C063C063C063C0A8
:10C0800043C060F660FFE3C5FFFFFFFFFFFF32CE56
:10C0900080FF80FF22D263C063C063C063C063C0FF
:10C0A00063C063C063C063C063C063C063C063C078
:10C0B00063C063C063C063C063C063C063C063C068
:10C0C00063C0E2C921F660FF60FF60FF60FF60FFB0
:10C0D00060FF60FF80FF80FF52CE25CE60FF60FFD3
:10C0E00060FF60FF60FF60FF60FF60FF60FF60FF58
:10C0F00060FF60FF60FF60FF60FF60FF60FF60FF48
:10C1000060FF60FF60FF60FF20F777CEB8DE50CEA3
:10C1100048CE82DE20F760FF60FF42DB63C063C071
:10C1200063C063C063C063C063C063C063C063C0F7
:10C1300063C063C063C063C063C063C063C063C0E7
:10C1400063C062DB60FF60FF70AD20F760FFC1DBA2
:10C1500063C063C063C063C063C063C063C063C0C7
:10C1600063C063C063C063C063C063C063C063C0B7
:10C1700063C063C063C002CA80FF80FF51CEFFFF6F
:10C18000FFFFFFFFFFFFFFFF25CE60FF40F643C02C
:10C1900063C063C063C063C063C063C063C063C087
:10C1A00063C063C063C063C063C063C063C063C077
:10C1B00063C063C0E3C040FF60FF2BC6FFFFFFFF0B
:10C1C0001BE700EF60FF41DC63C063C063C063C076
:10C1D00063C063C063C063C063C063C063C063C047
:10C1E00063C063C063C063C063C063C063C0E2DA9E
:10C1F00060FF60FFB6DE47CE60FFE0FE83C063C035
:10C2000063C063C063C063C063C063C063C063C016
:10C2100063C063C063C063C063C063C063C063C006
:10C2200063C063C0A0F660FF46D6FFFFFFFFFFFFBD
:10C23000FFFFFFFF4CCE60FF80FF03C163C063C000
:10C2400063C063C063C063C063C063C063C063C0D6
:10C2500063C063C063C063C063C063C063C063C0C6
:10C2600043C040F660FFE3C5FFFFFFFFFFFF32CE94
:10C2700080FF80FF22D263C063C063C063C063C01D
:10C2800063C063C063C063C063C063C063C063C096
:10C2900063C063C063C063C063C063C063C063C086
:10C2A00062D240FF60FF60FF00EF44D64BCE70D6F5
:10C2B00072CE74CE95D635CEFADE25CE60FF60FF05
:10C2C00060FF60FF60FF60FF60FF60FF60FF60FF76
:10C2D00060FF60FF60FF60FF60FF60FF60FF60FF66
:10C2E00060FF60FF60FF60FF60FF61D640F760FFA6
:10C2F00060FF60FF60FF80FF40FFE2D263C063C069
:10C3000063C063C063C063C063C063C063C063C015
:10C3100063C063C063C063C063C063C063C063C005
:10C3200063C062DB60FF60FF70AD20F760FFC1DBC0
:10C3300063C063C063C063C063C063C063C063C0E5
:10C3400063C063C063C063C063C063C063C063C0D5
:10C3500063C063C063C082D280FF60FF93D6FFFFDB
:10C36000FFFFFFFFFFFFFFFF25CE60FF40F643C04A
:10C3700063C063C063C063C063C063C063C063C0A5
:10C3800063C063C063C063C063C063C063C063C095
:10C3900063C063C0E3C040FF60FF2BC6FFFFFFFF29
:10C3A0001BE700EF60FF41DC63C063C063C063C094
:10C3B00063C063C063C063C063C063C063C063C065
:10C3C00063C063C063C063C063C063C063C0E2DABC
:10C3D00060FF60FFB6DE47CE60FFE0FE83C063C053
:10C3E00063C063C063C063C063C063C063C063C035
:10C3F00063C063C063C063C063C063C063C063C025
:10C4000063C063C0A0F660FF46D6FFFFFFFFFFFFDB
:10C41000FFFFFFFF4CCE60FF80FF03C163C063C01E
:10C4200063C063C063C063C063C063C063C063C0F4
:10C4300063C063C063C063C063C063C063C063C0E4
:10C4400043C040F660FFE3C5FFFFFFFFFFFF32CEB2
:10C4500080FF80FF22D263C063C063C063C063C03B
:10C4600063C063C063C063C063C063C063C063C0B4
:10C4700063C063C063C063C063C063C063C043C9BB
:10C4800020FF60FF40F709C6D9DEDFFFFFFFFFFF97
:10C49000FFFFFFFFFFFFFFFFFFFF10C68DD68DD60A
:10C4A0008DD68DD68DD68DD68DD68DD68DD68DD674
:10C4B0008DD68DD68DD68DD68DD66DD6EAC542ADAC
:10C4C000A0E660FF60FF60FF60FF60FF60FF80FF2D
:10C4D00020FFE1F521E462D2C2C063C063C063C043
:10C4E00063C063C063C063C063C063C063C063C034
:10C4F00063C063C063C063C063C063C063C063C024
:10C5000063C062DB60FF60FF70AD20F760FFC1DBDE
:10C5100063C063C063C063C063C063C063C063C003
:10C5200063C063C063C063C063C063C063C063C0F3
:10C5300063C063C063C082D280FF80FF94D6FFFFD8
:10C54000FFFFFFFFFFFFFFFF25CE60FF40F643C068
:10C5500063C063C063C063C063C063C063C063C0C3
:10C5600063C063C063C063C063C063C063C063C0B3
:10C5700063C063C0E3C040FF60FF2BC6FFFFFFFF47
:10C580001BE700EF60FF41DC63C063C063C063C0B2
:10C5900063C063C063C063C063C063C063C063C083
:10C5A00063C063C063C063C063C063C063C0E2DADA
:10C5B00060FF60FFB6DE47CE60FFE0FE83C063C071
:10C5C00063C063C063C063C063C063C063C063C053
:10C5D00063C063C063C063C063C063C063C063C043
:10C5E00063C063C0A0F660FF46D6FFFFFFFFFFFFFA
:10C5F000FFFFFFFF4CCE60FF80FF03C163C063C03D
:10C6000063C063C063C063C063C063C063C063C012
:10C6100063C063C063C063C063C063C063C063C002
:10C6200043C040F660FFE3C5FFFFFFFFFFFF32CED0
:10C6300080FF80FF22D263C063C063C063C063C059
:10C6400063C063C063C063C063C063C063C063C0D2
:10C6500063C063C063C063C063C063C063C0E1E420
:10C6600060FF40FF0EC6DFFFFFFFFFFFFFFFFFFF82
:10C67000FFFFFFFFFFFFFFFFFFFFFFFFFFFFFFFFCA
:10C68000FFFFFFFFFFFFFFFFFFFFFFFFFFFFFFFFBA
:10C69000FFFFFFFF9DF7B7D64ECE46CEE1E660FF27
:10C6A00060FF60FF60FF60FF40FF00F641E462D280
:10C6B000E3C063C063C063C063C063C063C063C0E2
:10C6C00063C063C063C063C063C063C063C063C052
:10C6D00063C063C063C063C063C063C063C063C042
:10C6E00063C062DB60FF60FF70AD20F760FFC1DBFD
:10C6F00063C063C063C063C063C063C063C063C022
:10C7000063C063C063C063C063C063C063C063C011
:10C7100063C063C063C082D280FF60FF94D6FFFF16
:10C72000FFFFFFFFFFFFFFFF25CE60FF40F643C086
:10C7300063C063C063C063C063C063C063C063C0E1
:10C7400063C063C063C063C063C063C063C063C0D1
:10C7500063C063C0E3C040FF60FF2BC6FFFFFFFF65
:10C760001BE700EF60FF41DC63C063C063C063C0D0
:10C7700063C063C063C063C063C063C063C063C0A1
:10C7800063C063C063C063C063C063C063C0E2DAF8
:10C7900060FF60FFB6DE47CE60FFE0FE83C063C08F
:10C7A00063C063C063C063C063C063C063C063C071
:10C7B00063C063C063C063C063C063C063C063C061
:10C7C00063C063C0A0F660FF46D6FFFFFFFFFFFF18
:10C7D000FFFFFFFF4CCE60FF80FF03C163C063C05B
:10C7E00063C063C063C063C063C063C063C063C031
:10C7F00063C063C063C063C063C063C063C063C021
:10C8000043C040F660FFE3C5FFFFFFFFFFFF32CEEE
:10C8100080FF80FF22D263C063C063C063C063C077
:10C8200063C063C063C063C063C063C063C063C0F0
:10C8300063C063C063C063C063C063C0E3C020FF64
:10C8400060FF45D69EF7FFFFFFFFFFFFFFFFFFFFE3
:10C85000FFFFFFFFFFFFFFFFFFFFFFFFFFFFFFFFE8
:10C86000FFFFFFFFFFFFFFFFFFFFFFFFFFFF3CE7B3
:10C8700053CE49CE82DE20F760FF60FF60FF60FF8D
:10C8800060FF80F6A1E4A2D203C143C063C063C0CD
:10C8900063C063C063C063C063C063C063C063C080
:10C8A00063C063C063C063C063C063C063C063C070
:10C8B00063C063C063C063C063C063C063C063C060
:10C8C00063C062DB60FF60FF70AD20F760FFC1DB1B
:10C8D00063C063C063C063C063C063C063C063C040
:10C8E00063C063C063C063C063C063C063C063C030
:10C8F00063C063C063C082D280FF60FF94D6FFFF35
:10C90000FFFFFFFFFFFFFFFF25CE60FF40F643C0A4
:10C9100063C063C063C063C063C063C063C063C0FF
:10C9200063C063C063C063C063C063C063C063C0EF
:10C9300063C063C0E3C040FF60FF2BC6FFFFFFFF83
:10C940001BE700EF60FF41DC63C063C063C063C0EE
:10C9500063C063C063C063C063C063C063C063C0BF
:10C9600063C063C063C063C063C063C063C0E2DA16
:10C9700060FF60FFB6DE47CE60FFE0FE83C063C0AD
:10C9800063C063C063C063C063C063C063C063C08F
:10C9900063C063C063C063C063C063C063C063C07F
:10C9A00063C063C0A0F660FF46D6FFFFFFFFFFFF36
:10C9B000FFFFFFFF4CCE60FF80FF03C163C063C079
:10C9C00063C063C063C063C063C063C063C063C04F
:10C9D00063C063C063C063C063C063C063C063C03F
:10C9E00043C040F660FFE3C5FFFFFFFFFFFF32CE0D
:10C9F00080FF80FF22D263C063C063C063C063C096
:10CA000063C063C063C063C063C063C063C063C00E
:10CA100063C063C063C063C063C063C062D280FF91
:10CA200060FF50CEFFFFFFFFFFFFFFFFFFFFFFFF95
:10CA3000FFFFFFFFFFFFFFFFFFFFFFFFFFFFFFFF06
:10CA4000FFFFFFFFFFFFFFFF9EF774CE29CEA1E699
:10CA500080FF60FF60FF60FF80FF00FF41ED42DB71
:10CA600062C963C063C063C063C063C063C063C0A6
:10CA700063C063C063C063C063C063C063C063C09E
:10CA800063C063C063C063C063C063C063C063C08E
:10CA900063C063C063C063C063C063C063C063C07E
:10CAA00063C062DB60FF60FF70AD20F760FFC1DB39
:10CAB00063C063C063C063C063C063C063C063C05E
:10CAC00063C063C063C063C063C063C063C063C04E
:10CAD00063C063C063C082D280FF60FF94D6FFFF53
:10CAE000FFFFFFFFFFFFFFFF25CE60FF40F643C0C3
:10CAF00063C063C063C063C063C063C063C063C01E
:10CB000063C063C063C063C063C063C063C063C00D
:10CB100063C063C0E3C040FF60FF2BC6FFFFFFFFA1
:10CB20001BE700EF60FF41DC63C063C063C063C00C
:10CB300063C063C063C063C063C063C063C063C0DD
:10CB400063C063C063C063C063C063C063C0E2DA34
:10CB500060FF60FFB6DE47CE60FFE0FE83C063C0CB
:10CB600063C063C063C063C063C063C063C063C0AD
:10CB700063C063C063C063C063C063C063C063C09D
:10CB800063C063C0A0F660FF46D6FFFFFFFFFFFF54
:10CB9000FFFFFFFF4CCE60FF80FF03C163C063C097
:10CBA00063C063C063C063C063C063C063C063C06D
:10CBB00063C063C063C063C063C063C063C063C05D
:10CBC00043C040F660FFE3C5FFFFFFFFFFFF32CE2B
:10CBD00080FF80FF22D263C063C063C063C063C0B4
:10CBE00063C063C063C063C063C063C063C063C02D
:10CBF00063C063C063C063C063C063C0C1DB60FF68
:10CC000040F7B7D6FFFFFFFFFFFFFFFFFFFFFFFF6C
:10CC1000FFFFFFFFFFFFFFFFFFFFFFFFFFFFFFFF24
:10CC2000FFFFFFFF9DF751CE43D640FF60FF60FF3F
:10CC300060FF40FF20F621E402CAA3C063C063C0C6
:10CC400063C063C063C063C063C063C063C063C0CC
:10CC500063C063C063C063C063C063C063C063C0BC
:10CC600063C063C063C063C063C063C063C063C0AC
:10CC700063C063C063C063C063C063C063C063C09C
:10CC800063C062DB60FF60FF70AD20F760FFC1DB57
:10CC900063C063C063C063C063C063C063C063C07C
:10CCA00063C063C063C063C063C063C063C063C06C
:10CCB00063C063C063C082D280FF60FF94D6FFFF71
:10CCC000FFFFFFFFFFFFFFFF25CE60FF40F643C0E1
:10CCD00063C063C063C063C063C063C063C063C03C
:10CCE00063C063C063C063C063C063C063C063C02C
:10CCF00063C063C0E3C040FF60FF2BC6FFFFFFFFC0
:10CD00001BE700EF60FF41DC63C063C063C063C02A
:10CD100063C063C063C063C063C063C063C063C0FB
:10CD200063C063C063C063C063C063C063C0E2DA52
:10CD300060FF60FFB6DE47CE60FFE0FE83C063C0E9
:10CD400063C063C063C063C063C063C063C063C0CB
:10CD500063C063C063C063C063C063C063C063C0BB
:10CD600063C063C0A0F660FF46D6FFFFFFFFFFFF72
:10CD7000FFFFFFFF4CCE60FF80FF03C163C063C0B5
:10CD800063C063C063C063C063C063C063C063C08B
:10CD900063C063C063C063C063C063C063C063C07B
:10CDA00043C040F660FFE3C5FFFFFFFFFFFF32CE49
:10CDB00080FF80FF22D263C063C063C063C063C0D2
:10CDC00063C063C063C063C063C063C063C063C04B
:10CDD00063C063C063C063C063C063C081E460FFBD
:10CDE000E0E61BE7FFFFFFFFFFFFFFFFFFFFFFFF87
:10CDF000FFFFFFFFFFFFFFFFFFFFFFFFFFFFFFFF43
:10CE0000DFFF74CE64D660FF60FF60FF60FFE0ED7F
:10CE100062DB43C963C063C063C063C063C063C0F7
:10CE200063C063C063C063C063C063C063C063C0EA
:10CE300063C063C063C063C063C063C063C063C0DA
:10CE400063C063C063C063C063C063C063C063C0CA
:10CE500063C063C063C063C063C063C063C063C0BA
:10CE600063C062DB60FF60FF70AD20F760FFC1DB75
:10CE700063C063C063C063C063C063C063C063C09A
:10CE800063C063C063C063C063C063C063C063C08A
:10CE900063C063C063C082D280FF60FF94D6FFFF8F
:10CEA000FFFFFFFFFFFFFFFF25CE60FF40F643C0FF
:10CEB00063C063C063C063C063C063C063C063C05A
:10CEC00063C063C063C063C063C063C063C063C04A
:10CED00063C063C0E3C040FF60FF2BC6FFFFFFFFDE
:10CEE0001BE700EF60FF41DC63C063C063C063C049
:10CEF00063C063C063C063C063C063C063C063C01A
:10CF000063C063C063C063C063C063C063C0E2DA70
:10CF100060FF60FFB6DE47CE60FFE0FE83C063C007
:10CF200063C063C063C063C063C063C063C063C0E9
:10CF300063C063C063C063C063C063C063C063C0D9
:10CF400063C063C0A0F660FF46D6FFFFFFFFFFFF90
:10CF5000FFFFFFFF4CCE60FF80FF03C163C063C0D3
:10CF600063C063C063C063C063C063C063C063C0A9
:10CF700063C063C063C063C063C063C063C063C099
:10CF800043C040F660FFE3C5FFFFFFFFFFFF32CE67
:10CF900080FF80FF22D263C063C063C063C063C0F0
:10CFA00063C063C063C063C063C063C063C063C069
:10CFB00063C063C063C063C063C063C0C1E460FF9B
:10CFC000A0E65DEFFFFFFFFFFFFFFFFFFFFFFFFF9B
:10CFD000FFFFFFFFFFFFFFFFFFFFFFFFFFFF7DEFF3
:10CFE000EAC520F760FF60FF40FF81E4A2C963C08B
:10CFF00063C063C063C063C063C063C063C063C019
:10D0000063C063C063C063C063C063C063C063C008
:10D0100063C063C063C063C063C063C063C063C0F8
:10D0200063C063C063C063C063C063C063C063C0E8
:10D0300063C063C063C063C063C063C063C063C0D8
:10D0400063C062DB60FF60FF70AD20F760FFC1DB93
:10D0500063C063C063C063C063C063C063C063C0B8
:10D0600063C063C063C063C063C063C063C063C0A8
:10D0700063C063C063C082D280FF60FF94D6FFFFAD
:10D08000FFFFFFFFFFFFFFFF25CE60FF40F643C01D
:10D0900063C063C063C063C063C063C063C063C078
:10D0A00063C063C063C063C063C063C063C063C068
:10D0B00063C063C0E3C040FF60FF2BC6FFFFFFFFFC
:10D0C0001BE700EF60FF41DC63C063C063C063C067
:10D0D00063C063C063C063C063C063C063C063C038
:10D0E00063C063C063C063C063C063C063C0E2DA8F
:10D0F00060FF60FFB6DE47CE60FFE0FE83C063C026
:10D1000063C063C063C063C063C063C063C063C007
:10D1100063C063C063C063C063C063C063C063C0F7
:10D1200063C063C0A0F660FF46D6FFFFFFFFFFFFAE
:10D13000FFFFFFFF4CCE60FF80FF03C163C063C0F1
:10D1400063C063C063C063C063C063C063C063C0C7
:10D1500063C063C063C063C063C063C063C063C0B7
:10D1600043C040F660FFE3C5FFFFFFFFFFFF32CE85
:10D1700080FF80FF22D263C063C063C063C063C00E
:10D1800063C063C063C063C063C063C063C063C087
:10D1900063C063C063C063C063C063C0C1E460FFB9
:10D1A000A0E65DEFFFFFFFFFFFFFFFFFFFFFFFFFB9
:10D1B000FFFFFFFFFFFFFFFFFFFFFFFF1BE725CE86
:10D1C00060FF60FF40FFA1E403C163C063C063C0B0
:10D1D00063C063C063C063C063C063C063C063C037
:10D1E00063C063C063C063C063C063C063C063C027
:10D1F00063C063C063C063C063C063C063C063C017
:10D2000063C063C063C063C063C063C063C063C006
:10D2100063C063C063C063C063C063C063C063C0F6
:10D2200063C062DB60FF60FF70AD20F760FFC1DBB1
:10D2300063C063C063C063C063C063C063C063C0D6
:10D2400063C063C063C063C063C063C063C063C0C6
:10D2500063C063C063C082D280FF60FF94D6FFFFCB
:10D26000FFFFFFFFFFFFFFFF25CE60FF40F643C03B
:10D2700063C063C063C063C063C063C063C063C096
:10D2800063C063C063C063C063C063C063C063C086
:10D2900063C063C0E3C040FF60FF2BC6FFFFFFFF1A
:10D2A0001BE700EF60FF41DC63C063C063C063C085
:10D2B00063C063C063C063C063C063C063C063C056
:10D2C00063C063C063C063C063C063C063C0E2DAAD
:10D2D00060FF60FFB6DE47CE60FFE0FE83C063C044
:10D2E00063C063C063C063C063C063C063C063C026
:10D2F00063C063C063C063C063C063C063C063C016
:10D3000063C063C0A0F660FF46D6FFFFFFFFFFFFCC
:10D31000FFFFFFFF4CCE60FF80FF03C163C063C00F
:10D3200063C063C063C063C063C063C063C063C0E5
:10D3300063C063C063C063C063C063C063C063C0D5
:10D3400043C040F660FFE3C5FFFFFFFFFFFF32CEA3
:10D3500080FF80FF22D263C063C063C063C063C02C
:10D3600063C063C063C063C063C063C063C063C0A5
:10D3700063C063C063C063C063C063C0C1E460FFD7
:10D38000A0E65DEFFFFFFFFFFFFFFFFFFFFFFFFFD7
:10D39000FFFFFFFFFFFFFFFFFFFF3BE744D660FFFC
:10D3A00060FF61F602CA63C063C063C063C063C04C
:10D3B00063C063C063C063C063C063C063C063C055
:10D3C00063C063C063C063C063C063C063C063C045
:10D3D00063C063C063C083C002D2C2C963C063C0FC
:10D3E00063C063C063C063C063C063C063C063C025
:10D3F00063C063C063C063C063C063C063C063C015
:10D4000063C062DB60FF60FF70AD20F760FFC1DBCF
:10D4100063C063C063C063C063C063C063C063C0F4
:10D4200063C063C063C063C063C063C063C063C0E4
:10D4300063C063C063C082D280FF60FF94D6FFFFE9
:10D44000FFFFFFFFFFFFFFFF25CE60FF40F643C059
:10D4500063C063C063C063C063C063C063C063C0B4
:10D4600063C063C063C063C063C063C063C063C0A4
:10D4700063C063C0E3C040FF60FF2BC6FFFFFFFF38
:10D480001BE700EF60FF41DC63C063C063C063C0A3
:10D4900063C063C063C063C063C063C063C063C074
:10D4A00063C063C063C063C063C063C063C0E2DACB
:10D4B00060FF60FFB6DE47CE60FFE0FE83C063C062
:10D4C00063C063C063C063C063C063C063C063C044
:10D4D00063C063C063C063C063C063C063C063C034
:10D4E00063C063C0A0F660FF46D6FFFFFFFFFFFFEB
:10D4F000FFFFFFFF4CCE60FF80FF03C163C063C02E
:10D5000063C063C063C063C063C063C063C063C003
:10D5100063C063C063C063C063C063C063C063C0F3
:10D5200043C040F660FFE3C5FFFFFFFFFFFF32CEC1
:10D5300080FF80FF22D263C063C063C063C063C04A
:10D5400063C063C063C063C063C063C063C063C0C3
:10D5500063C063C063C063C063C063C0C1E460FFF5
:10D56000A0E65DEFFFFFFFFFFFFFFFFFFFFFFFFFF5
:10D57000FFFFFFFFFFFFFFFFBEF708C660FF60FF72
:10D58000C1EDE3C063C063C063C063C063C063C078
:10D5900063C063C063C063C063C063C063C063C073
:10D5A00063C063C063C063C063C063C063C063C063
:10D5B00003C1C2D2A1E4A0F680FF42DB63C063C016
:10D5C00063C063C063C063C063C063C063C063C043
:10D5D00063C063C063C063C063C063C063C063C033
:10D5E00063C062DB60FF60FF70AD20F760FFC1DBEE
:10D5F00063C063C063C063C063C063C063C063C013
:10D6000063C063C063C063C063C063C063C063C002
:10D6100063C063C063C082D280FF60FF94D6FFFF07
:10D62000FFFFFFFFFFFFFFFF25CE60FF40F643C077
:10D6300063C063C063C063C063C063C063C063C0D2
:10D6400063C063C063C063C063C063C063C063C0C2
:10D6500063C063C0E3C040FF60FF2BC6FFFFFFFF56
:10D660001BE700EF60FF41DC63C063C063C063C0C1
:10D6700063C063C063C063C063C063C063C063C092
:10D6800063C063C063C063C063C063C063C0E2DAE9
:10D6900060FF60FFB6DE47CE60FFE0FE83C063C080
:10D6A00063C063C063C063C063C063C063C063C062
:10D6B00063C063C063C063C063C063C063C063C052
:10D6C00063C063C0A0F660FF46D6FFFFFFFFFFFF09
:10D6D000FFFFFFFF4CCE60FF80FF03C163C063C04C
:10D6E00063C063C063C063C063C063C063C063C022
:10D6F00063C063C063C063C063C063C063C063C012
:10D7000043C040F660FFE3C5FFFFFFFFFFFF32CEDF
:10D7100080FF80FF22D263C063C063C063C063C068
:10D7200063C063C063C063C063C063C063C063C0E1
:10D7300063C063C063C063C063C063C0C1E460FF13
:10D74000A0E65DEFFFFFFFFFFFFFFFFFFFFFFFFF13
:10D75000FFFFFFFFFFFFFFFF31CE40FF60FF40F6FE
:10D76000C3C063C063C063C063C063C063C063C041
:10D7700063C063C063C063C063C063C063C063C091
:10D7800063C063C063C063C063C0E3C082DBE1ED1C
:10D7900040FF60FF60FF60FF60FF42DB63C063C06B
:10D7A00063C063C063C063C063C063C063C063C061
:10D7B00063C063C063C063C063C063C063C063C051
:10D7C00063C062DB60FF60FF70AD20F760FFC1DB0C
:10D7D00063C063C063C063C063C063C063C063C031
:10D7E00063C063C063C063C063C063C063C063C021
:10D7F00063C063C063C082D280FF60FF94D6FFFF26
:10D80000FFFFFFFFFFFFFFFF25CE60FF40F643C095
:10D8100063C063C063C063C063C063C063C063C0F0
:10D8200063C063C063C063C063C063C063C063C0E0
:10D8300063C063C0E3C040FF60FF2BC6FFFFFFFF74
:10D840001BE700EF60FF41DC63C063C063C063C0DF
:10D8500063C063C063C063C063C063C063C063C0B0
:10D8600063C063C063C063C063C063C063C0E2DA07
:10D8700060FF60FFB6DE47CE60FFE0FE83C063C09E
:10D8800063C063C063C063C063C063C063C063C080
:10D8900063C063C063C063C063C063C063C063C070
:10D8A00063C063C0A0F660FF46D6FFFFFFFFFFFF27
:10D8B000FFFFFFFF4CCE60FF80FF03C163C063C06A
:10D8C00063C063C063C063C063C063C063C063C040
:10D8D00063C063C063C063C063C063C063C063C030
:10D8E00043C040F660FFE3C5FFFFFFFFFFFF32CEFE
:10D8F00080FF80FF22D263C063C063C063C063C087
:10D9000063C063C063C063C063C063C063C063C0FF
:10D9100063C063C063C063C063C063C0C1E460FF31
:10D92000A0E65DEFFFFFFFFFFFFFFFFFFFFFFFFF31
:10D93000FFFFFFFFFFFF9DEF62D660FF20FF62C980
:10D9400063C063C063C063C063C063C063C063C0BF
:10D9500063C063C063C063C063C063C063C063C0AF
:10D9600063C063C063C0C3C061E440FF60FF60FF89
:10D9700060FF60FF20F760FF60FF42DB63C063C0B1
:10D9800063C063C063C063C063C063C063C063C07F
:10D9900063C063C063C063C063C063C063C063C06F
:10D9A00063C062DB60FF60FF70AD20F760FFC1DB2A
:10D9B00063C063C063C063C063C063C063C063C04F
:10D9C00063C063C063C063C063C063C063C063C03F
:10D9D00063C063C063C082D280FF60FF94D6FFFF44
:10D9E000FFFFFFFFFFFFFFFF25CE60FF40F643C0B4
:10D9F00063C063C063C063C063C063C063C063C00F
:10DA000063C063C063C063C063C063C063C063C0FE
:10DA100063C063C003C140FF60FF2BC6FFFFFFFF71
:10DA20001BE700EF60FF41DC63C063C063C063C0FD
:10DA300063C063C063C063C063C063C063C063C0CE
:10DA400063C063C063C063C063C063C063C0E2DA25
:10DA500060FF60FFB6DE47CE60FFE0FE83C063C0BC
:10DA600063C063C063C063C063C063C063C063C09E
:10DA700063C063C063C063C063C063C063C063C08E
:10DA800063C063C0A0F660FF46D6FFFFFFFFFFFF45
:10DA9000FFFFFFFF4CCE60FF80FF03C163C063C088
:10DAA00063C063C063C063C063C063C063C063C05E
:10DAB00063C063C063C063C063C063C063C063C04E
:10DAC00043C040F660FFE3C5FFFFFFFFFFFF32CE1C
:10DAD00080FF80FF22D263C063C063C063C063C0A5
:10DAE00063C063C063C063C063C063C063C063C01E
:10DAF00063C063C063C063C063C063C0C1E460FF50
:10DB0000A0E65DEFFFFFFFFFFFFFFFFFFFFFFFFF4F
:10DB1000FFFFFFFFFFFF53CE60FF60FF21E463C004
:10DB200063C063C063C063C063C063C063C063C0DD
:10DB300063C063C063C063C063C063C063C063C0CD
:10DB400063C063C042C980F660FF60FF60FFA1E66A
:10DB500048CE51CE12C660FF60FF42DB63C063C097
:10DB600063C063C063C063C063C063C063C063C09D
:10DB700063C063C063C063C063C063C063C063C08D
:10DB800063C062DB60FF60FF70AD20F760FFC1DB48
:10DB900063C063C063C063C063C063C063C063C06D
:10DBA00063C063C063C063C063C063C063C063C05D
:10DBB00063C063C063C082D280FF60FF94D6FFFF62
:10DBC000FFFFFFFFFFFFFFFF25CE60FF40F643C0D2
:10DBD00063C063C063C063C063C063C063C063C02D
:10DBE00063C063C063C063C063C063C063C063C01D
:10DBF00063C063C003C160FF60FF6CCEFFFFFFFF27
:10DC00001BE700EF60FF41DC63C063C063C063C01B
:10DC100063C063C063C063C063C063C063C063C0EC
:10DC200063C063C063C063C063C063C063C0E2DA43
:10DC300060FF60FFB6DE47CE60FFE0FE83C063C0DA
:10DC400063C063C063C063C063C063C063C063C0BC
:10DC500063C063C063C063C063C063C063C063C0AC
:10DC600063C063C0A0F660FF46D6FFFFFFFFFFFF63
:10DC7000FFFFFFFF4CCE60FF80FF03C163C063C0A6
:10DC800063C063C063C063C063C063C063C063C07C
:10DC900063C063C063C063C063C063C063C063C06C
:10DCA00043C040F660FFE3C5FFFFFFFFFFFF32CE3A
:10DCB00080FF80FF22D263C063C063C063C063C0C3
:10DCC00063C063C063C063C063C063C063C063C03C
:10DCD00063C063C063C063C063C063C0C1E460FF6E
:10DCE000A0E65DEFFFFFFFFFFFFFFFFFFFFFFFFF6E
:10DCF000FFFFFFFFFFFF49CE60FF40FF42C963C047
:10DD000063C063C063C063C063C063C063C063C0FB
:10DD100063C063C063C063C063C063C063C063C0EB
:10DD200063C083C021EE60FF60FF63D651CE5CE725
:10DD3000FFFFFFFFD7DE40FF60FF42DB63C063C031
:10DD400063C063C063C063C063C063C063C063C0BB
:10DD500063C063C063C063C063C063C063C063C0AB
:10DD600063C062DB60FF60FF70AD20F760FFC2DB65
:10DD700063C063C063C063C063C063C063C063C08B
:10DD800063C063C063C063C063C063C063C063C07B
:10DD900063C063C063C042D280FF80FF52CEFFFFEA
:10DDA000FFFFFFFFFFFFFFFF25CE60FF40F643C0F0
:10DDB00063C063C063C063C063C063C063C063C04B
:10DDC00063C063C063C063C063C063C063C063C03B
:10DDD00063C063C063C960FF60FF6ED6FFFFFFFFD3
:10DDE0001BE700EF60FF41E463C063C063C063C032
:10DDF00063C063C063C063C063C063C063C063C00B
:10DE000063C063C063C063C063C063C063C0E2DA61
:10DE100060FF60FFB6DE47CE60FFE0FE83C063C0F8
:10DE200063C063C063C063C063C063C063C063C0DA
:10DE300063C063C063C063C063C063C063C063C0CA
:10DE400063C063C0A0F660FF46D6FFFFFFFFFFFF81
:10DE5000FFFFFFFF4CCE60FF80FF03C163C063C0C4
:10DE600063C063C063C063C063C063C063C063C09A
:10DE700063C063C063C063C063C063C063C063C08A
:10DE800043C040F660FFE3C5FFFFFFFFFFFF32CE58
:10DE900080FF80FF22D263C063C063C063C063C0E1
:10DEA00063C063C063C063C063C063C063C063C05A
:10DEB00063C063C063C063C063C063C0C1E460FF8C
:10DEC000A0E65DEFFFFFFFFFFFFFFFFFFFFFFFFF8C
:10DED000FFFFFFFFBEF762D660FF00F663C063C0BE
:10DEE00063C063C063C063C063C063C063C063C01A
:10DEF00063C063C063C063C063C063C063C063C00A
:10DF000063C062D260FF60FF28CE5CEFFFFFFFFFBF
:10DF1000FFFFFFFFD7DE40FF60FF42DB63C063C04F
:10DF200063C063C063C063C063C063C063C063C0D9
:10DF300063C063C063C063C063C063C063C063C0C9
:10DF400063C061DB60FF60FF70AD20F760FFE1DB65
:10DF500063C063C063C063C063C063C063C063C0A9
:10DF600063C063C063C063C063C063C063C063C099
:10DF700063C063C063C082C980FF60FF4ECEFFFFF5
:10DF8000FFFFFFFFFFFFFFFF25CE60FF40F643C00E
:10DF900063C063C063C063C063C063C063C063C069
:10DFA00063C063C063C063C063C063C063C063C059
:10DFB00063C063C0E2C980FF80FF71D6FFFFFFFF2F
:10DFC0001BE700F760FF41E463C063C063C063C048
:10DFD00063C063C063C063C063C063C063C063C029
:10DFE00063C063C063C063C063C063C063C0E2DA80
:10DFF00060FF60FFB6DE47CE60FFE0FE83C063C017
:10E0000063C063C063C063C063C063C063C063C0F8
:10E0100063C063C063C063C063C063C063C063C0E8
:10E0200063C063C0A0F660FF46D6FFFFFFFFFFFF9F
:10E03000FFFFFFFF4CCE60FF80FF03C163C063C0E2
:10E0400063C063C063C063C063C063C063C063C0B8
:10E0500063C063C063C063C063C063C063C063C0A8
:10E0600043C040F660FFE3C5FFFFFFFFFFFF72D62E
:10E0700080FF80FF22D263C063C063C063C063C0FF
:10E0800063C063C063C063C063C063C063C063C078
:10E0900063C063C063C063C063C063C061E460FF0A
:10E0A000E0EE1BE7FFFFFFFFFFFFFFFFFFFFFFFFAC
:10E0B000FFFFFFFFFBDEE0EE60FF81E463C063C0B3
:10E0C00063C063C063C063C063C063C063C063C038
:10E0D00063C063C063C063C063C063C063C063C028
:10E0E00063C0E1DB60FF40FF77D6FFFFFFFFFFFF6C
:10E0F000FFFFFFFFD7DE40FF60FF42DB63C063C06E
:10E1000063C063C063C063C063C063C063C063C0F7
:10E1100063C063C063C063C063C063C063C063C0E7
:10E1200063C042DB60FF60FF91B520F760FF21E430
:10E1300063C063C063C063C063C063C063C063C0C7
:10E1400063C063C063C063C063C063C063C063C0B7
:10E1500063C063C063C0A3C020FF60FF25CEBEF7CD
:10E16000FFFFFFFFFFFFFFFF25CE60FF40F643C02C
:10E1700063C063C063C063C063C063C063C063C087
:10E1800063C063C063C063C063C063C063C063C077
:10E1900063C063C062C980FF60FF4ED6FFFFFFFF10
:10E1A000FADE20F760FF21DC63C063C063C063C098
:10E1B00063C063C063C063C063C063C063C063C047
:10E1C00063C063C063C063C063C063C063C0E2D2A6
:10E1D00060FF60FFB6DE68D660FFE0FE83C063C00C
:10E1E00063C063C063C063C063C063C063C063C017
:10E1F00063C063C063C063C063C063C063C063C007
:10E2000063C063C0A0F660FF26CEFFFFFFFFFFFFE5
:10E21000FFFFFFFF4CCE60FF80FFE3C063C063C021
:10E2200063C063C063C063C063C063C063C063C0D6
:10E2300063C063C063C063C063C063C063C063C0C6
:10E2400043C061F660FFE3C5FFFFFFFFFFFF6ECE37
:10E2500060FF80FFA2C963C063C063C063C063C0C6
:10E2600063C063C063C063C063C063C063C063C096
:10E2700063C063C063C063C063C063C0A2DB60FFF0
:10E2800040F7B7D6FFFFFFFFFFFFFFFFFFFFFFFFD6
:10E29000FFFFFFFFD8DE40F760FFA2DB63C063C073
:10E2A00063C063C063C063C063C063C063C063C056
:10E2B00063C063C063C063C063C063C063C063C046
:10E2C00063C0E2E360FF60FF34CEFFFFFFFFFFFFAC
:10E2D0005CEF73CE46CE60FF60FF42DB63C063C07D
:10E2E00063C063C063C063C063C063C063C063C016
:10E2F00063C063C063C063C063C063C063C063C006
:10E3000063C082D260FF60FF8DB500EF60FF21E443
:10E3100063C063C063C063C063C063C063C063C0E5
:10E3200063C063C063C063C063C063C063C063C0D5
:10E3300063C063C063C063C001E560FF60FF0CC6DB
:10E340001BE77DEF1AE774D662D660FF40F643C044
:10E3500063C063C063C063C063C063C063C063C0A5
:10E3600063C063C063C063C063C063C063C063C095
:10E3700063C063C0C3C000FF60FF47CEDFFFFFFF85
:10E3800097D640FF60FFA1DB63C063C063C063C07A
:10E3900063C063C063C063C063C063C063C063C065
:10E3A00063C063C063C063C063C063C063C082D224
:10E3B00080FF80FF52CE29CE60FF00FFA3C063C064
:10E3C00063C063C063C063C063C063C063C063C035
:10E3D00063C063C063C063C063C063C063C063C025
:10E3E00063C063C040F660FF24CEFFFFFFFFFFFF66
:10E3F000FFFFFFFF4ACE60FF60FFA3C063C063C0A2
:10E4000063C063C063C063C063C063C063C063C0F4
:10E4100063C063C063C063C063C063C063C063C0E4
:10E4200043C0A0F660FF05CEFFFFFFFF3CEF63D6C1
:10E4300060FFE0FEA3C063C063C063C063C063C08D
:10E4400063C063C063C063C063C063C063C063C0B4
:10E4500063C063C063C063C063C063C042D280FF57
:10E4600060FF2DCEFFFFFFFFFFFFFFFFFFFFFFFF5E
:10E47000FFFFFFFF96D640FF60FF22DB63C063C053
:10E4800063C063C063C063C063C063C063C063C074
:10E4900063C063C063C063C063C063C063C063C064
:10E4A00063C0A2C940FF60FFC2E64DCE6DD647CE25
:10E4B000A1DE40FF60FF60FF40FF82D263C063C007
:10E4C00063C063C063C063C063C063C063C063C034
:10E4D00063C063C063C063C063C063C063C063C024
:10E4E00063C042C940FF60FFA5BDE0E660FFA1E454
:10E4F00063C063C063C063C063C063C063C063C004
:10E5000063C063C063C063C063C063C063C063C0F3
:10E5100063C063C063C063C063C920FF60FF60FF66
:10E52000C1E682DEE0EE60FF60FF60FF40F643C0C0
:10E5300063C063C063C063C063C063C063C063C0C3
:10E5400063C063C063C063C063C063C063C063C0B3
:10E5500063C063C063C0C1ED60FFE1E6B8D6DFFF12
:10E560000CC660FF60FF62D263C063C063C063C05B
:10E5700063C063C063C063C063C063C063C063C083
:10E5800063C063C063C063C063C063C063C043C98A
:10E5900080FF60FF28CE2BCE60FF40FFE3C063C04A
:10E5A00063C063C063C063C063C063C063C063C053
:10E5B00063C063C063C063C063C063C063C063C043
:10E5C00063C043C061ED60FFA1DE5DEFFFFFFFFFB1
:10E5D000FFFFDFFF44D660FFA0FE63C063C063C0DF
:10E5E00063C063C063C063C063C063C063C063C013
:10E5F00063C063C063C063C063C063C063C063C003
:10E6000063C000FF60FF07C6DFFF76D664D660FFF9
:10E6100060FF81E463C063C063C063C063C063C064
:10E6200063C063C063C063C063C063C063C063C0D2
:10E6300063C063C063C063C063C063C0A3C0C0F6EF
:10E6400060FFE1EE2ECE1BE7FFFFFFFFFFFFFFFFA6
:10E65000FFFFFFFFB7D640FF60FF42DB63C063C030
:10E6600063C063C063C063C063C063C063C063C092
:10E6700063C063C063C063C063C063C063C063C082
:10E6800063C063C061E460FF60FF60FF60FF60FF24
:10E6900060FF60FF60FF61EDA2C963C063C063C03B
:10E6A00063C063C063C063C063C063C063C063C052
:10E6B00063C063C063C063C063C063C063C063C042
:10E6C00063C063C081ED60FF40FF40FF60FF41ED2C
:10E6D00043C063C063C063C063C063C063C063C042
:10E6E00063C063C063C063C063C063C063C063C012
:10E6F00063C063C063C063C063C042D2E0F660FF22
:10E7000060FF60FF60FF60FF80FFC0FE21E443C048
:10E7100063C063C063C063C063C063C063C063C0E1
:10E7200063C063C063C063C063C063C063C063C0D1
:10E7300063C063C063C0C2D260FF60FF84D60BC6F3
:10E7400020F760FFA0F6A3C063C063C063C063C0CE
:10E7500063C063C063C063C063C063C063C063C0A1
:10E7600063C063C063C063C063C063C063C063C091
:10E77000C1ED60FF40F7E3C560FF80FFA2C963C041
:10E7800063C063C063C063C063C063C063C063C071
:10E7900063C063C063C063C063C063C063C063C061
:10E7A00063C063C0A1DB60FF60FFEEC5BEF7FFFF83
:10E7B000DFFF33CE20F760FF01ED63C063C063C0AD
:10E7C00063C063C063C063C063C063C063C063C031
:10E7D00063C063C063C063C063C063C063C063C021
:10E7E000E3C080FF60FF4BCE76CE20EF60FF60FF7E
:10E7F00021F6C3C063C063C063C063C063C063C0AD
:10E8000063C063C063C063C063C063C063C063C0F0
:10E8100063C063C063C063C063C063C063C022D30E
:10E8200060FF60FF60FFC1E6FADEFFFFFFFFFFFF52
:10E83000FFFFFFFFD9DE20F760FFC1DB63C063C0CD
:10E8400063C063C063C063C063C063C063C063C0B0
:10E8500063C063C063C063C063C063C063C063C0A0
:10E8600063C063C083C001DC20FF80FF80FF00FF26
:10E87000C1EDA1DB42C963C063C063C063C063C0B4
:10E8800063C063C063C063C063C063C063C063C070
:10E8900063C063C063C063C063C063C063C063C060
:10E8A00063C063C063C900F760FF60FF60FF40F6AC
:10E8B00043C063C063C063C063C063C063C063C060
:10E8C00063C063C063C063C063C063C063C063C030
:10E8D00063C063C063C063C063C063C0C3C042DBC6
:10E8E000E1E461ED81E422DB63C963C063C063C01E
:10E8F00063C063C063C063C063C063C063C063C000
:10E9000063C063C063C063C063C063C063C063C0EF
:10E9100063C063C063C063C061ED60FF60FF60FF00
:10E9200060FF40FF82D263C063C063C063C063C046
:10E9300063C063C063C063C063C063C063C063C0BF
:10E9400063C063C063C063C063C063C063C063C0AF
:10E95000C2C920FF60FF60FF60FF60FF02D363C099
:10E9600063C063C063C063C063C063C063C063C08F
:10E9700063C063C063C063C063C063C063C063C07F
:10E9800063C063C022C100FF60FF40F742D625CEBE
:10E9900024D620EF60FF60FF02CA63C063C063C07B
:10E9A00063C063C063C063C063C063C063C063C04F
:10E9B00063C063C063C063C063C063C063C063C03F
:10E9C00022D280FF60FF50CE76CE60F760FF61ED0F
:10E9D000C3C063C063C063C063C063C063C063C0BF
:10E9E00063C063C063C063C063C063C063C063C00F
:10E9F00063C063C063C063C063C063C063C063C0FF
:10EA000042DBE0F660FF60FFD9DEFFFFFFFFFFFFA4
:10EA1000FFFFFFFF3CE7C0E660FFC1EC63C063C0DF
:10EA200063C063C063C063C063C063C063C063C0CE
:10EA300063C063C063C063C063C063C063C063C0BE
:10EA400063C063C063C063C0A3C062C942C9A3C03E
:10EA500063C063C063C063C063C063C063C063C09E
:10EA600063C063C063C063C063C063C063C063C08E
:10EA700063C063C063C063C063C063C063C063C07E
:10EA800063C063C063C0C2C9C0F660FF60FF20FFFF
:10EA900083C063C063C063C063C063C063C063C03E
:10EAA00063C063C063C063C063C063C063C063C04E
:10EAB00063C063C063C063C063C063C063C063C03E
:10EAC00063C063C063C063C063C063C063C063C02E
:10EAD00063C063C063C063C063C063C063C063C01E
:10EAE00063C063C063C063C063C063C063C063C00E
:10EAF00063C063C063C063C0A3C041E560FF60FF43
:10EB0000E0FE62D263C063C063C063C063C063C021
:10EB100063C063C063C063C063C063C063C063C0DD
:10EB200063C063C063C063C063C063C063C063C0CD
:10EB300063C042CAC0F660FF60FF60FFC1E463C00B
:10EB400063C063C063C063C063C063C063C063C0AD
:10EB500063C063C063C063C063C063C063C063C09D
:10EB600063C063C063C0E2D240FF60FF60FF60FF2C
:10EB700060FF60FF60FFE1DB63C063C063C063C030
:10EB800063C063C063C063C063C063C063C063C06D
:10EB900063C063C063C063C063C063C063C063C05D
:10EBA00001DC60FF40F7B7D676CE60F760FF02DB8E
:10EBB00063C063C063C063C063C063C063C063C03D
:10EBC00063C063C063C063C063C063C063C063C02D
:10EBD00063C063C063C063C063C063C063C063C01D
:10EBE00063C0A2DB60FF60FFD9DEFFFFFFFFFFFF16
:10EBF000FFFFFFFFBEF763D660FF40F663C063C050
:10EC000063C063C063C063C063C063C063C063C0EC
:10EC100063C063C063C063C063C063C063C063C0DC
:10EC200063C063C063C063C063C063C063C063C0CC
:10EC300063C063C063C063C063C063C063C063C0BC
:10EC400063C063C063C063C063C063C063C063C0AC
:10EC500063C063C063C063C063C063C063C063C09C
:10EC600063C063C063C063C0E1E460FF60FF80FF16
:10EC7000A2C963C063C063C063C063C063C063C034
:10EC800063C063C063C063C063C063C063C063C06C
:10EC900063C063C063C063C063C063C063C063C05C
:10ECA00063C063C063C063C063C063C063C063C04C
:10ECB00063C063C063C063C063C063C063C063C03C
:10ECC00063C063C063C063C063C063C063C063C02C
:10ECD00063C063C063C063C063C062CA60FF60FF9B
:10ECE00021ED63C063C063C063C063C063C063C021
:10ECF00063C063C063C063C063C063C063C063C0FC
:10ED000063C063C063C063C063C063C063C063C0EB
:10ED100063C063C061E460FF60FF60FFC0F6A3C032
:10ED200063C063C063C063C063C063C063C063C0CB
:10ED300063C063C063C063C063C063C063C063C0BB
:10ED400063C063C063C063C082C981E401F660F63A
:10ED500020F621E542D263C063C063C063C063C0D4
:10ED600063C063C063C063C063C063C063C063C08B
:10ED700063C063C063C063C063C063C063C063C07B
:10ED800020F660FF82DE7DEF76CE60F760FF02D373
:10ED900063C063C063C063C063C063C063C063C05B
:10EDA00063C063C063C063C063C063C063C063C04B
:10EDB00063C063C063C063C063C063C063C063C03B
:10EDC00063C0A1DB60FF60FFD9DEFFFFFFFFFFFF35
:10EDD000FFFFFFFFFFFF4ACE60FF40FF62C963C035
:10EDE00063C063C063C063C063C063C063C063C00B
:10EDF00063C063C063C063C063C063C063C063C0FB
:10EE000063C063C063C063C063C063C063C063C0EA
:10EE100063C063C063C063C063C063C063C063C0DA
:10EE200063C063C063C063C063C063C063C063C0CA
:10EE300063C063C063C063C063C063C063C063C0BA
:10EE400063C063C063C063C0E1E460FF60FF60FF54
:10EE500082DB63C063C063C063C063C063C063C060
:10EE600063C063C063C063C063C063C063C063C08A
:10EE700063C063C063C063C063C063C063C063C07A
:10EE800063C063C063C063C063C063C063C063C06A
:10EE900063C063C063C063C063C063C063C063C05A
:10EEA00063C063C063C063C063C063C063C063C04A
:10EEB00063C063C063C063C063C062D260FF60FFB1
:10EEC00021ED63C063C063C063C063C063C063C03F
:10EED00063C063C063C063C063C063C063C063C01A
:10EEE00063C063C063C063C063C063C063C063C00A
:10EEF00063C063C061E460FF60FF60FF60FFC2D277
:10EF000063C063C063C063C063C063C063C063C0E9
:10EF100063C063C063C063C063C063C063C063C0D9
:10EF200063C063C063C063C063C063C043C043C009
:10EF300043C063C063C063C063C063C063C063C0D9
:10EF400063C063C063C063C063C063C063C063C0A9
:10EF500063C063C063C063C063C063C063C022CAD0
:10EF600060FF60FF2BCEFFFF76CE60F760FF02DB15
:10EF700063C063C063C063C063C063C063C063C079
:10EF800063C063C063C063C063C063C063C063C069
:10EF900063C063C063C063C063C063C063C063C059
:10EFA00063C0A1DB60FF60FFD9DEFFFFFFFFFFFF53
:10EFB000FFFFFFFFFFFF74CE60FF60FF61E463C0EF
:10EFC00063C063C063C063C063C063C063C063C029
:10EFD00063C063C063C063C063C063C063C063C019
:10EFE00063C063C063C063C063C063C063C063C009
:10EFF00063C063C063C063C063C063C063C063C0F9
:10F0000063C063C063C063C063C063C063C063C0E8
:10F0100063C063C063C063C063C063C063C063C0D8
:10F0200063C063C063C063C0E1E460FF60FF60FF72
:10F0300001F663C063C063C063C063C063C063C0E4
:10F0400063C063C063C063C063C063C063C063C0A8
:10F0500063C063C063C063C063C063C063C063C098
:10F0600063C063C063C063C063C063C063C063C088
:10F0700063C063C063C063C063C063C063C063C078
:10F0800063C063C063C063C063C063C063C063C068
:10F0900063C063C063C063C063C062D260FF60FFCF
:10F0A00021ED63C063C063C063C063C063C063C05D
:10F0B00063C063C063C063C063C063C063C063C038
:10F0C00063C063C063C063C063C063C063C063C028
:10F0D00063C063C061E460FF00EFE0EE60FF60F6D4
:10F0E00083C063C063C063C063C063C063C063C0E8
:10F0F00063C063C063C063C063C063C063C063C0F8
:10F1000063C063C063C063C063C063C063C063C0E7
:10F1100063C063C063C063C063C063C063C063C0D7
:10F1200063C063C063C063C063C063C063C063C0C7
:10F1300063C063C063C063C063C063C083C001F6C3
:10F1400060FF20EFB8D6FFFF76CE60F760FF02DBEE
:10F1500063C063C063C063C063C063C063C063C097
:10F1600063C063C063C063C063C063C063C063C087
:10F1700063C063C063C063C063C063C063C063C077
:10F1800063C0A1DB60FF60FFD9DEFFFFFFFFFFFF71
:10F19000FFFFFFFFFFFF9EF743D660FF20FF62C91E
:10F1A00063C063C063C063C063C063C063C063C047
:10F1B00063C063C063C063C063C063C063C063C037
:10F1C00063C063C063C063C063C063C063C063C027
:10F1D00063C063C063C063C063C063C063C063C017
:10F1E00063C063C063C063C063C063C063C063C007
:10F1F00063C063C063C063C063C063C063C063C0F7
:10F2000063C063C063C063C0E1E460FF60FF60FF90
:10F2100060FFE2C963C063C063C063C063C063C012
:10F2200063C063C063C063C063C063C063C063C0C6
:10F2300063C063C063C063C063C063C063C063C0B6
:10F2400063C063C063C063C063C063C063C063C0A6
:10F2500063C063C063C063C063C063C063C063C096
:10F2600063C063C063C063C063C063C063C063C086
:10F2700063C063C063C063C063C062D260FF60FFED
:10F2800021ED63C063C063C063C063C063C063C07B
:10F2900063C063C063C063C063C063C063C063C056
:10F2A00063C063C063C063C063C063C063C063C046
:10F2B00063C063C061E460FFE0E668B560FF60FFC3
:10F2C00042E463C063C063C063C063C063C063C023
:10F2D00063C063C063C063C063C063C063C063C016
:10F2E00063C063C063C063C063C063C063C063C006
:10F2F00063C063C063C063C063C063C063C063C0F6
:10F3000063C063C063C063C063C063C063C063C0E5
:10F3100063C063C063C063C063C063C0C2DB60FF1F
:10F3200060FF08C6DFFFFFFF76CE60F760FF02DBFD
:10F3300063C063C063C063C063C063C063C063C0B5
:10F3400063C063C063C063C063C063C063C063C0A5
:10F3500063C063C063C063C063C063C063C063C095
:10F3600063C0A1DB60FF60FFD9DEFFFFFFFFFFFF8F
:10F37000FFFFFFFFFFFFFFFF31CE60F760FFC1ED32
:10F3800083C063C063C063C063C063C063C063C045
:10F3900063C063C063C063C063C063C063C063C055
:10F3A00063C063C063C063C063C063C063C063C045
:10F3B00063C063C063C063C063C062D202CA63C07B
:10F3C00063C063C063C063C063C063C063C063C025
:10F3D00063C063C063C063C063C063C063C063C015
:10F3E00063C063C063C063C0E1E460FF20F720F73F
:10F3F00060FFC1ED83C063C063C063C063C063C00E
:10F4000063C063C063C063C063C063C063C063C0E4
:10F4100063C063C063C063C063C063C063C063C0D4
:10F4200063C063C063C063C063C063C063C083C0A4
:10F4300063C063C063C063C063C063C063C063C0B4
:10F4400063C063C063C063C063C063C063C063C0A4
:10F4500063C063C063C063C063C062D260FF60FF0B
:10F4600021ED63C063C063C063C063C063C063C099
:10F4700063C063C063C063C063C063C063C063C074
:10F4800063C063C063C063C063C063C063C063C064
:10F4900063C063C061E460FFC0E658CE82DE60FFF7
:10F4A00060FF62DB63C063C063C063C063C063C0EE
:10F4B00063C063C063C063C063C063C063C063C034
:10F4C00063C063C063C063C063C063C063C063C024
:10F4D00063C063C063C063C063C063C063C063C014
:10F4E00063C063C063C063C063C063C063C063C004
:10F4F00063C063C063C063C063C0E2D240FF60FF0B
:10F50000A1DEFADEFFFFFFFF76CE60F760FF02DBD1
:10F5100063C063C063C063C063C063C063C063C0D3
:10F5200063C063C063C063C063C063C063C063C0C3
:10F5300063C063C063C063C063C063C063C063C0B3
:10F5400063C0A1DB60FF60FFD9DEFFFFFFFFFFFFAD
:10F55000FFFFFFFFFFFFFFFFBEF706C660FF60FF74
:10F56000E1E483C063C063C063C063C063C063C0C1
:10F5700063C063C063C063C063C063C063C063C073
:10F5800063C063C063C063C063C063C063C063C063
:10F5900063C063C063C022C121ED80FFA2D263C0FB
:10F5A00063C063C063C063C063C063C063C063C043
:10F5B00063C063C063C063C063C063C063C063C033
:10F5C00063C063C063C063C0E1E460FFC1E6A6BD81
:10F5D00060FF60FFA2DB63C063C063C063C063C041
:10F5E00063C063C063C063C063C063C063C063C003
:10F5F00063C063C063C063C063C063C063C063C0F3
:10F6000063C063C063C063C063C0A3C021DC42D2D7
:10F6100063C063C063C063C063C063C063C063C0D2
:10F6200063C063C063C063C063C063C063C063C0C2
:10F6300063C063C063C063C063C062D260FF60FF29
:10F6400021ED63C063C063C063C063C063C063C0B7
:10F6500063C063C063C063C063C063C063C063C092
:10F6600063C063C063C063C063C063C063C063C082
:10F6700063C063C061E460FFC0E61BE775D6E1EEDE
:10F6800060FF60FF41E483C063C063C063C063C0C8
:10F6900063C063C063C063C063C063C063C063C052
:10F6A00063C063C063C063C063C063C063C063C042
:10F6B00063C063C063C063C063C063C063C063C032
:10F6C00063C063C063C063C063C063C063C063C022
:10F6D00063C063C063C063C0A1DB60FF60FF20EF55
:10F6E00053CEFFFFFFFFFFFF76CE60F760FF02DB28
:10F6F00063C063C063C063C063C063C063C063C0F2
:10F7000063C063C063C063C063C063C063C063C0E1
:10F7100063C063C063C063C063C063C063C063C0D1
:10F7200063C0A1DB60FF60FFD9DEFFFFFFFFFFFFCB
:10F73000FFFFFFFFFFFFFFFFFFFF1AE783DE60FF12
:10F7400060FF81ED02C163C063C063C063C063C07A
:10F7500063C063C063C063C063C063C063C063C091
:10F7600063C063C063C063C063C063C063C063C081
:10F7700063C0C3C0E1DB20FF60FF80FFA2D263C093
:10F7800063C063C063C063C063C063C063C063C061
:10F7900063C063C063C063C063C063C063C063C051
:10F7A00063C063C063C063C0E1E460FFC1E657CEDD
:10F7B000C1E660FF60FF42D363C063C063C063C043
:10F7C00063C063C063C063C063C063C063C063C021
:10F7D00063C063C063C063C063C063C063C063C011
:10F7E00063C063C063C063C062D260F660FF82D250
:10F7F00063C063C063C063C063C063C063C063C0F1
:10F8000063C063C063C063C063C063C063C063C0E0
:10F8100063C063C063C063C063C062D260FF60FF47
:10F8200021ED63C063C063C063C063C063C063C0D5
:10F8300063C063C063C063C063C063C063C063C0B0
:10F8400063C063C063C063C063C063C063C063C0A0
:10F8500063C063C061E460FFC0E61BE7FFFF53CEF7
:10F8600001EF60FF60FF40F662D263C063C063C017
:10F8700063C063C063C063C063C063C063C063C070
:10F8800063C063C063C063C063C063C063C063C060
:10F8900063C063C063C063C063C063C063C063C050
:10F8A00063C063C063C063C063C063C063C063C040
:10F8B00063C063C0A2C9A1ED60FF60FF20EF31CE3D
:10F8C000FFFFFFFFFFFFFFFF76CE60F760FF02DB69
:10F8D00063C063C063C063C063C063C063C063C010
:10F8E00063C063C063C063C063C063C063C063C000
:10F8F00063C063C063C063C063C063C063C063C0F0
:10F9000063C0A2DB60FF60FFD9DEFFFFFFFFFFFFE8
:10F91000FFFFFFFFFFFFFFFFFFFFFFFFD8DE83DEDC
:10F9200060FF60FFC0F602D383C063C063C063C0E2
:10F9300063C063C063C063C063C063C063C063C0AF
:10F9400063C063C063C063C063C063C063C0E3C01F
:10F95000A2DBC0F660FF60FF60FF60FFA2D263C061
:10F9600063C063C063C063C063C063C063C063C07F
:10F9700063C063C063C063C063C063C063C063C06F
:10F9800063C063C063C063C0E1E460FFE1E65CEFB5
:10F9900053CE00EF60FF60FFA1E4E3C063C063C02B
:10F9A00063C063C063C063C063C063C063C063C03F
:10F9B00063C063C063C063C063C063C063C063C02F
:10F9C00063C083C042D2A1ED60FF60FF60FF82D2BE
:10F9D00063C063C063C063C063C063C063C063C00F
:10F9E00063C063C063C063C063C063C063C063C0FF
:10F9F00063C063C063C063C063C062D260FF60FF66
:10FA000021ED63C063C063C063C063C063C063C0F3
:10FA100063C063C063C063C063C063C063C063C0CE
:10FA200063C063C063C063C063C063C063C063C0BE
:10FA300063C063C061E460FFC0E61CE7FFFFFFFF37
:10FA400075D682DE60FF60FF60FF01F622D303C13E
:10FA500063C063C063C063C063C063C063C063C08E
:10FA600063C063C063C063C063C063C063C063C07E
:10FA700063C063C063C063C063C063C063C063C06E
:10FA800063C063C063C063C063C063C063C083C03E
:10FA900002CA01ED40FF60FF60FFC1E653CEFFFFE9
:10FAA000FFFFFFFFFFFFFFFF76CE60F760FF82DB07
:10FAB00023C923C923C923C923C923C923C923C9E6
:10FAC00023C923C923C923C923C923C923C923C9D6
:10FAD00023C923C923C923C923C923C923C923C9C6
:10FAE00043C901DC60FF60FFD9DEFFFFFFFFFFFFBE
:10FAF000FFFFFFFFFFFFFFFFFFFFFFFFFFFFF9DE3D
:10FB000045D660FF60FF60FF60F681DB43C963C0DC
:10FB100063C063C063C063C063C063C063C063C0CD
:10FB200063C063C063C063C0A3C042D2C1E400FF2E
:10FB300060FF60FF60FFA1E660FF60FF42DB23C95A
:10FB400023C923C923C923C923C923C923C923C955
:10FB500023C923C923C923C923C923C923C923C945
:10FB600023C923C943C943C921E560FFC1E67DEF2D
:10FB7000FFFF32C601EF60FF60FFC0F6E2E362C93B
:10FB800063C063C063C063C063C063C063C063C05D
:10FB900063C063C063C063C063C063C0A3C0E2C985
:10FBA00001DC60F660FF60FF60FF60FF60FF02D372
:10FBB00022C923C923C923C923C923C923C923C9E6
:10FBC00023C923C923C923C923C923C923C923C9D5
:10FBD00023C923C923C923C923C9E2D260FF60FF17
:10FBE00061ED23C923C923C923C923C923C923C953
:10FBF00023C923C923C923C923C923C923C923C9A5
:10FC000023C923C923C923C923C923C923C923C994
:10FC100023C923C9C1E460FFC0E61CE7FFFFFFFF63
:10FC2000FFFF1BE72AC600EF60FF60FF60FF20FFB9
:10FC3000A1EDC1DB02CAE3C063C063C063C063C09F
:10FC400063C063C063C063C063C063C063C063C09C
:10FC500063C063C063C063C063C063C063C063C08C
:10FC600063C063C063C063C0E3C062D261E480F676
:10FC700060FF60FF60FF40F726CED9DEFFFFFFFF89
:10FC8000FFFFFFFFFFFFFFFF76CE60F760FF80FF03
:10FC900080FF80FF80FF80FF80FF80FF80FF80FF6C
:10FCA00080FF80FF80FF80FF80FF80FF80FF80FF5C
:10FCB00080FF80FF80FF80FF80FF80FF80FF80FF4C
:10FCC00080FF60FF60FF60FFD9DEFFFFFFFFFFFFE7
:10FCD000FFFFFFFFFFFFFFFFFFFFFFFFFFFFFFFF34
:10FCE0007DEF0DC6C1E660FF60FF60FF60FF40F67C
:10FCF00081E442DB22D262C9E3C0C3C0C3C023C9CE
:10FD0000C2C9E2D201DC81ED00FF80FF60FF60FF2D
:10FD100060FF82DE4ECEF2BD80FF60FF60FF80FF9D
:10FD200080FF80FF80FF80FF80FF80FF80FF80FFDB
:10FD300080FF80FF80FF80FF80FF80FF80FF80FFCB
:10FD400080FF80FF80FF80FF60FF60FFC1E67DEFE6
:10FD5000FFFFFFFF96D663D660FF60FF60FF60FF86
:10FD600041F6C1E481DBA2D202D2A2C962C982C932
:10FD7000C2C942D2E2D281DB81E4C0ED00FF80FF44
:10FD800060FF60FF60FF20F7E3C560FF60FF60FF7A
:10FD900080FF80FF80FF80FF80FF80FF80FF80FF6B
:10FDA00080FF80FF80FF80FF80FF80FF80FF80FF5B
:10FDB00080FF80FF80FF80FF80FF60FF60FF60FFAB
:10FDC00060FF80FF80FF80FF80FF80FF80FF80FF5B
:10FDD00080FF80FF80FF80FF80FF80FF80FF80FF2B
:10FDE00080FF80FF80FF80FF80FF80FF80FF80FF1B
:10FDF00080FF80FF60FF60FFC0E61CE7FFFFFFFFA2
:10FE0000FFFFFFFFFFFFB8DE29CEC0E660FF60FF07
:10FE100060FF60FF60FF40FF80F681EDA1E4C2DB80
:10FE200022D382D202D282C942C902C1C3C0C3C096
:10FE3000C3C0C3C0C3C0E3C023C962C902CAA2D23F
:10FE400062DB41E441ED60F640FF60FF60FF60FF70
:10FE500060FF40F725CE74CEBEF7FFFFFFFFFFFF28
:10FE6000FFFFFFFFFFFFFFFF76CE60F760FF60FF41
:10FE700060FF60FF60FF60FF60FF60FF60FF60FF8A
:10FE800060FF60FF60FF60FF60FF60FF60FF60FF7A
:10FE900060FF60FF60FF60FF60FF60FF60FF60FF6A
:10FEA00060FF60FF60FF60FFD9DEFFFFFFFFFFFF25
:10FEB000FFFFFFFFFFFFFFFFFFFFFFFFFFFFFFFF52
:10FEC000FFFFFFFFFADE2CCE81DE60FF60FF60FFE8
:10FED00060FF60FF80FF80FF80FF80FF80FF80FF6A
:10FEE00080FF60FF60FF60FF60FF60FF20F744D687
:10FEF00050CE5CEFFFFF94D680FF60FF60FF60FF95
:10FF000060FF60FF60FF60FF60FF60FF60FF60FFF9
:10FF100060FF60FF60FF60FF60FF60FF60FF60FFE9
:10FF200060FF60FF60FF60FF60FF60FFE1E67CEF65
:10FF3000FFFFFFFFFFFF7DEF2EC662DE60FF60FF69
:10FF400060FF60FF60FF60FF80FF80FF80FF80FF39
:10FF500080FF80FF60FF60FF60FF60FF60FF60FF69
:10FF600040FF62D62BCE98D653CE60FF60FF60FF75
:10FF700060FF60FF60FF60FF60FF60FF60FF60FF89
:10FF800060FF60FF60FF60FF60FF60FF60FF60FF79
:10FF900060FF60FF60FF60FF60FF60FF60FF60FF69
:10FFA00060FF60FF60FF60FF60FF60FF60FF60FF59
:10FFB00060FF60FF60FF60FF60FF60FF60FF60FF49
:10FFC00060FF60FF60FF60FF60FF60FF60FF60FF39
:10FFD00060FF60FF60FF60FFC0E61BE7FFFFFFFF01
:10FFE000FFFFFFFFFFFFFFFFFFFF1BE750CE47CEE6
:10FFF000A1DE40FF60FF60FF60FF60FF60FF60FF09
:020000040801F1
:1000000060FF80FF80FF80FF80FF80FF80FF80FF18
:1000100080FF80FF80FF80FF80FF80FF80FF60FF08
:1000200060FF60FF60FF60FF60FF80FF20F763D626
:100030004BCE97D6DFFFFFFFFFFFFFFFFFFFFFFF66
:10004000FFFFFFFFFFFFFFFFFADE8ED68EDE8EDEA4
:100050008EDE8EDE8EDE8EDE8EDE8EDE8EDE8EDE40
:100060008EDE8EDE8EDE8EDE8EDE8EDE8EDE8EDE30
:100070008EDE8EDE8EDE8EDE8EDE8EDE8EDE8EDE20
:100080008EDE8EDE8EDE8EDE5CE7FFFFFFFFFFFF83
:10009000FFFFFFFFFFFFFFFFFFFFFFFFFFFFFFFF70
:1000A000FFFFFFFFFFFFFFFF5CEF53CE49CE63D69C
:1000B00000EF60F760FF60FF60FF60FF60FF60FFC0
:1000C00060FF60FF20F7A2DE46CE4ECEB8D6BEF768
:1000D000FFFFFFFFFFFFF9DE8EDE8EDE8EDE8EDE9F
:1000E0008EDE8EDE8EDE8EDE8EDE8EDE8EDE8EDEB0
:1000F0008EDE8EDE8EDE8EDE8EDE8EDE8EDE8EDEA0
:100100008EDE8EDE8EDE8EDE8EDE8EDE4FCEBEF795
:10011000FFFFFFFFFFFFFFFFFFFF7DEF54CE4ACE43
:1001200063D6E1EE20F760FF60FF60FF60FF80FFB5
:1001300060FF80FF60FF20F700EF82DE47CE4ECEEB
:1001400096D69DF7FFFFFFFFD9DE8ED68EDE8EDEC0
:100150008EDE8EDE8EDE8EDE8EDE8EDE8EDE8EDE3F
:100160008EDE8EDE8EDE8EDE8EDE8EDE8EDE8EDE2F
:100170008EDE8EDE8EDE8EDE8EDE8EDE8EDE8EDE1F
:100180008EDE8EDE8EDE8EDE8EDE8EDE8EDE8EDE0F
:100190008EDE8EDE8EDE8EDE8EDE8EDE8EDE8EDEFF
:1001A0008EDE8EDE8EDE8EDE8EDE8EDE8EDE8EDEEF
:1001B0008EDE8EDE8EDE8ED64ECE7DEFFFFFFFFF13
:1001C000FFFFFFFFFFFFFFFFFFFFFFFFFFFFDFFF5F
:1001D0005DEF96D650CE2ACE45D682DEE0EE20F7F1
:1001E00040F760FF60FF60FF60FF60FF60FF60FF3F
:1001F00060FF60FF60FF60FF60FF60FF60FF60FF07
:1002000040F700EFA2DE44D62ACE50CEB8D69EF7F5
:10021000FFFFFFFFFFFFFFFFFFFFFFFFFFFFFFFFEE
:10022000FFFFFFFFFFFFFFFFFFFFFFFFFFFFFFFFDE
:10023000FFFFFFFFFFFFFFFFFFFFFFFFFFFFFFFFCE
:10024000FFFFFFFFFFFFFFFFFFFFFFFFFFFFFFFFBE
:10025000FFFFFFFFFFFFFFFFFFFFFFFFFFFFFFFFAE
:10026000FFFFFFFFFFFFFFFFFFFFFFFFFFFFFFFF9E
:10027000FFFFFFFFFFFFFFFFFFFFFFFFFFFFFFFF8E
:10028000FFFFFFFFFFFFFFFFFFFFFFFFFFFF9EF7E7
:100290001AE795D651CE4ECE4CD66CD64CD64DCE16
:1002A00050CE94D6D8DE7DEFDFFFFFFFFFFFFFFFCC
:1002B000FFFFFFFFFFFFFFFFFFFFFFFFFFFFFFFF4E
:1002C000FFFFFFFFFFFFFFFFFFFFFFFFFFFFFFFF3E
:1002D000FFFFFFFFFFFFFFFFFFFFFFFFFFFFFFFF2E
:1002E000FFFFFFFFFFFFFFFFFFFFFFFFFFFFFFFF1E
:1002F000FFFFFFFFFFFFFFFFFFFFFFFFFFFFFFFF0E
:10030000BEF73BE7B7D694D651CE50CE2FCE2FCEE8
:1003100051CE72CE94D6B7DE1BE79EF7FFFFFFFFEC
:10032000FFFFFFFFFFFFFFFFFFFFFFFFFFFFFFFFDD
:10033000FFFFFFFFFFFFFFFFFFFFFFFFFFFFFFFFCD
:10034000FFFFFFFFFFFFFFFFFFFFFFFFFFFFFFFFBD
:10035000FFFFFFFFFFFFFFFFFFFFFFFFFFFFFFFFAD
:10036000FFFFFFFFFFFFFFFFFFFFFFFFFFFFFFFF9D
:10037000FFFFFFFFFFFFFFFFFFFFFFFFFFFFFFFF8D
:10038000FFFFFFFFFFFFFFFFFFFFFFFFFFFFFFFF7D
:10039000FFFFFFFFFFFFFFFFFFFFFFFFFFFFFFFF6D
:1003A000FFFFFFFFFFFFFFFFFFFFFFFFFFFFFFFF5D
:1003B000FFFFFFFFFFFFFFFFDFFF7DF73BE7D8DE1B
:1003C000B6D693D651CE4FCE4ECE4DCE4CD66CD661
:1003D0006CD66BD66CD66DD64ECE4FCE51CE94D653
:1003E000B7D6FADE7DEFDFFFFFFFFFFFFFFFFFFF66
:1003F000FFFFFFFFFFFFFFFFFFFFFFFFFFFFFFFF0D
:10040000FFFFFFFFFFFFFFFFFFFFFFFFFFFFFFFFFC
:10041000FFFFFFFFFFFFFFFFFFFFFFFFFFFFFFFFEC
:10042000FFFFFFFFFFFFFFFFFFFFFFFFFFFFFFFFDC
:10043000FFFFFFFFFFFFFFFFFFFFFFFFFFFFFFFFCC
:10044000FFFFFFFFFFFFFFFFFFFFFFFFFFFFFFFFBC
:10045000FFFFFFFFFFFFFFFFFFFFFFFFFFFFFFFFAC
:10046000FFFFFFFFFFFFFFFFFFFFFFFFFFFFFFFF9C
:10047000FFFFFFFFFFFFFFFFFFFFFFFFFFFFFFFF8C
:10048000FFFFFFFFFFFFFFFFFFFFFFFFFFFFFFFF7C
:10049000FFFFFFFFFFFFFFFFFFFFFFFFFFFFFFFF6C
:1004A000FFFFFFFFFFFFFFFFFFFFFFFFFFFFFFFF5C
:1004B000FFFFFFFFFFFFFFFFFFFFFFFFFFFFFFFF4C
:1004C000FFFFFFFFFFFFFFFFFFFFFFFFFFFFFFFF3C
:1004D000FFFFFFFFFFFFFFFFFFFFFFFFFFFFFFFF2C
:1004E000FFFFFFFFFFFFFFFFFFFFFFFFFFFFFFFF1C
:1004F000FFFFFFFFFFFFFFFFFFFFFFFFFFFFFFFF0C
:10050000FFFFFFFFFFFFFFFFFFFFFFFFFFFFFFFFFB
:10051000FFFFFFFFFFFFFFFFFFFFFFFFFFFFFFFFEB
:10052000FFFFFFFFFFFFFFFFFFFFFFFFFFFFFFFFDB
:10053000FFFFFFFFFFFFFFFFFFFFFFFFFFFFFFFFCB
:10054000FFFFFFFFFFFFFFFFFFFFFFFFFFFFFFFFBB
:10055000FFFFFFFFFFFFFFFFFFFFFFFFFFFFFFFFAB
:10056000FFFFFFFFFFFFFFFFFFFFFFFFFFFFFFFF9B
:10057000FFFFFFFFFFFFFFFFFFFFFFFFFFFFFFFF8B
:10058000FFFFFFFFFFFFFFFFFFFFFFFFFFFFFFFF7B
:10059000FFFFFFFFFFFFFFFFFFFFFFFFFFFFFFFF6B
:1005A000FFFFFFFFFFFFFFFFFFFFFFFFFFFFFFFF5B
:1005B000FFFFFFFFFFFFFFFFFFFFFFFFFFFFFFFF4B
:1005C000FFFFFFFFFFFFFFFFFFFFFFFFFFFFFFFF3B
:1005D000FFFFFFFFFFFFFFFFFFFFFFFFFFFFFFFF2B
:1005E000FFFFFFFFFFFFFFFF000000000000000013
:1005F00001020304060708090000000001020304C9
:1006000000061016000610161B5B481B5B324A1BC7
:100610005B33366D44656B6F646572206B6F647518
:10062000204D6F72736527612056302E32620D0A9D
:100630001B5B33376D4D61792032352032303230DB
:100640002031393A31333A32320D0A7361734065E1
:100650006C706F7274616C2E706C0D0A1B5B33339F
:100660006D2A2A2A205354415254202A2A2A0D0A3C
:100670000000000064656661756C745461736B0002
:100680001B5B343B3330481B5B33346D746F6E3D02
:100690002534646D732070727A3D2534646D732047
:1006A0005B2532642F25645D1B5B353B3330482767
:1006B0002E273D2533646D7320272D273D25336478
:1006C0006D732070617573653D2533641B5B363B2C
:1006D00033304857504D3D2533641B5B7500000097
:1006E000000701080000002028010000043900086C
:1006F0002808010828010020407A01001439000868
:100700000101000000000000000000000000640083
:10071000900158024600D200E7001027F4010000C3
:1007200000000000000000000000000000000000C9
:1007300000000000000000000000000000000000B9
:100740000000000000000000000020C10000204167
:1007500000002041000020C1000020C10000204115
:1007600000002041000020C1000020C1000020C185
:100770000000204100002041000020C1000020C1F5
:100780000000204100002041000020C1000020C1E5
:10079000000020C1000020C10000204100002041D5
:1007A0000000204100002041030001000000101063
:1007B00000000000000000000024F4000100000020
:1007C0001000000000000000000000000000000019
:1007D0000000000000000000000000000000000019
:1007E0000000000000000000000000000000000009
:1007F00000000000000000000000000000000000F9
:1008000000000000000000000000000000000000E8
:1008100000000000000000000000000000000000D8
:08082000AAAAAAAA0000000028
:040000050800019955
:00000001FF
